:020000040000FA
:040000006FD00400B9
:101000006F00907E00000000000000009020002093
:10101000AA220020A9BDF9F56C23002000000000E1
:10102000000000006C230020902000200000000041
:101030000000000090200020000000009020002010
:101040000000000090200020902000209020002030
:101050009020002090200020582F00209424002071
:101060000000000090200020902000201E2400207E
:1010700090200020D22300209020002090200020EB
:101080009020002090200020902000209020002020
:101090009020002001A04111B7170040985F3AC688
:1010A000945F3247E39CE6FE3245410182800111A4
:1010B00013078008F337078093F787083EC20100C3
:1010C0000100B7170040930570052380B70413068D
:1010D00080FA2380C7040100010083C6B70493F699
:1010E000F60DA385D704238007049246F3A6068055
:1010F0000100010093760502D5CEF336078093F602
:10110000860836C4010001002380B7042380C70489
:1011100001000100B70614007D89558D88C70100C4
:1011200001000100010023800704A246F3A6068007
:101130000100010073370780137787083AC6010062
:1011400001002380B7042380C704010001000100CF
:1011500001003727004093061005A303D7802380A2
:101160000704B247F3A70780010001009307800836
:10117000F3B7078093F787083ECE01000100B71749
:101180000040130770052380E704130780FA2380CB
:10119000E7040100010003C7B70413670708A3852C
:1011A000E70423800704F247F3A70780010001004A
:1011B0000561828093760504BDC6F336078093F6F9
:1011C000860836C8010001002380B7042380C704C5
:1011D00001000100B7061400938606047D89558D31
:1011E00088C7010001000100010023800704C246F6
:1011F000F3A6068001000100733707801377870884
:101200003ACA010001002380B7042380C70401000B
:1012100001003727004093062005A303D7802380D1
:101220000704D24781B773370780137787083ACC12
:10123000010001002380B7042380C70401000100DE
:1012400098471367070C98C723800704E24719BF24
:101250000111814601468145114506CE97000000E7
:10126000E780605893078008F3B7078093F78708F3
:101270003EC601000100B717004013077005238028
:10128000E704130780FA2380E7040100010003C785
:101290006704136717002383E70423800704B2471A
:1012A000F3A7078001000100F2400561828041112F
:1012B000814601468145114597000000E780A05214
:1012C00013078008F337078093F787083EC40100AF
:1012D0000100B7170040130670052380C70493066A
:1012E00080FA2380D70401000100FD552396B70240
:1012F00023800704A245F3A5058001000100733790
:101300000780137787083AC6010001002380C704CD
:101310002380D7040100010003C767041367170087
:101320002383E70423800704B247F3A70780010063
:10133000010001A0B1473305F50201007D1575FDDF
:101340008280411122C426C206C6AA8401446317C2
:101350009400B24022449244410182800504130566
:10136000803E420497000000E78000FD4180C5B741
:101370009305000273A04580824573901534924016
:101380002242B2424243D2436244F2440255925551
:101390002256B2564257D2576258F25806499649D9
:1013A000264AB64A464BD64B664CF64C065D965DD1
:1013B000265EB65E465FD65F09617300203041113C
:1013C000B7170040985F3AC6945F3247E39CE6FE49
:1013D000324541018280B71700401307000323887C
:1013E000E702854717170000232AF75473002030BF
:1013F000411122C42D6426C24AC006C637190040D6
:101400001304A4AAB704002023208900976000E0F9
:10141000E780E0389C408297976000E0E7802038C2
:10142000E5B737370040834747009146BD8B639E41
:10143000D702B73600401306F00F973500009385AA
:10144000E52C9737000083D7673C03C7A6001377C6
:10145000F70F1DE3B7E70400BC4F09468945171590
:1014600000000345A5F7829731A099466394D70001
:10147000834757007300203003C786001377F70FA8
:10148000E365F6FC13851700AE9717380000231F9D
:10149000A8362380E70075B7B787004003C7670009
:1014A000098B6309071003C77700930600031377BE
:1014B0000703630DD708174800000348F884174650
:1014C0000000130666810547B30606012380E60087
:1014D00083C577001747000013070782429793F5EB
:1014E000F50F2300B70003C58700973500009385EB
:1014F000A57FC2951375F50F2380A500034707004C
:1015000089451377F703630CB70C63E7E50A6306B5
:10151000071A8545630CB7129737000083C7D77E3B
:101520003307F600034707001377F70F19CB85073A
:1015300093F7F70F3D476363F71A17370000A305CA
:10154000F77CB787004009472383E700B78700404F
:1015500083C77700E207E18763DE0704973700005F
:1015600083C7977A17370000130707773E9785469A
:101570002300D70017370000130707783E9793061C
:1015800000032300D700173700001307E7753E97C5
:10159000A14685072300D70093F7F70F3D47636403
:1015A000F71417370000A301F776B7870040094703
:1015B0002383E70073002030930610026300D70EE8
:1015C000930620026305D70693060002E316D7F4BC
:1015D00003C727021377C70F13672700D5A803C7D0
:1015E00067001377070465CB03C7A702173800000D
:1015F000130808501735000013054547134707081F
:101600002385E70203C7A7021377370F1367870005
:101610002385E702814713070004B305F5008C41D9
:10162000B306F80091078CC2E399E7FEF5B503C74E
:10163000A702134707042385E70203C7A70213770E
:10164000C70F136727002385E702F9B503C76700B3
:101650001377070449C303C767021738000013084C
:10166000E83C17350000130525341347070823838A
:10167000E70203C767021377370F136787002383D7
:10168000E702814713070004B305F5008C41B30658
:10169000F80091078CC2E399E7FEBDBD03C767025E
:1016A000134707042383E70203C767021377C70FB3
:1016B000136727002383E70285B503C76700137705
:1016C000070411CB03C727021377370F136787006F
:1016D0002381E70291B5238006003DBD97370000C6
:1016E000A3840762B9BD97370000A38F076075BD5B
:1016F0002303048015472303E48001002302A48010
:10170000828083076480E3CE07FE23030480828007
:1017100083076480E3CE07FE03454480828083070D
:101720006480E3CE07FE2302A4808280411126C498
:101730004AC24EC006C61377F50BAD47AA892E895B
:101740009544630CF700194597000000E78080FA84
:1017500097000000E78020FB8D444E859700000035
:10176000E78040F9FD59FD1463983401B240A2446A
:101770001249824941018280135509011375F50F01
:1017800097000000E780E0F92209F1BF011126CCA3
:1017900006CEB704080097000000E780C0F61545A4
:1017A00097000000E78000F597000000E78080F6D2
:1017B00097000000E78000F62AC697000000E78047
:1017C00080F432459377150089EB13651500137586
:1017D000F50FF240E24405618280FD14E9F0014515
:1017E000CDBF397126DC4ADA4ED852D656D45AD2F9
:1017F0005ED006DE62CE66CCB7E700E07D5783AAF6
:10180000070022C603AA470023A0E71823A2E7186F
:10181000B7170040130770052380E704130780FA09
:101820002380E70483C74704930B75FFB684E20760
:1018300093FBFB0F8546AA892E8B32893724004003
:10184000E187015763FA76016308D50089461307DB
:1018500000026313D5000157D98F93F7F70FB71C18
:1018600000402382FC0411472303E4801305F00F9A
:1018700097000000E78000E8094C97000000E7802F
:1018800080E863657C15B7050700DA9537870700A0
:10189000795563FEE504B3879500636AF704370B57
:1018A0000800A94733EB65016395F90881E8814495
:1018B00097000000E78020E5268515A8DA85094510
:1018C00097000000E780C0E605090345F9FFFD1415
:1018D000050B97000000E780C0E481C49377FB0FFD
:1018E000E5F797000000E780A0EA69F17D55B7179A
:1018F0000040130770052380E704130780FA238054
:10190000E70403C74704418B2382E704F250B7E79B
:1019100000E023A0571123A24711E2543244525948
:10192000C259325AA25A125B825B724CE24C21615C
:101930008280A547639BF90685691309F00FB306FA
:101940009900B3742B01B6941349F9FFB37499004D
:10195000856B33796901416B9387F9FFB3F72701F1
:1019600099E363FC340193D94900C147E3E637FFAB
:101970003DBF0569C1697D19D9B71305800D63881D
:101980006901130500026384790113051008CA85F3
:1019900097000000E780C0D997000000E78040DF93
:1019A00031D54E99B38434416DBFDA852D4597000A
:1019B0000000E780E0D7CA94E30B99EE0509970091
:1019C0000000E78020D5A30FA9FEFDB79387F9FF9C
:1019D00093F7F70F636DFC0C83C71C0413073008E3
:1019E0006315F706370708006361EB06B3079B0032
:1019F000B706100063FBD704334BEB0089476399AC
:101A0000F9068980D549E38404EADA850945970017
:101A10000000E780E0D111090327C9FF9147232087
:101A2000E48003076480E34E07FE23033481FD173F
:101A3000EDFBFD14110B81C49377FB0FE9FF9700B9
:101A40000000E780E0D461F155B5B717004003C747
:101A50005704B70708001377070219E3B787070091
:101A60007955E376FBE833079B00E3F9E7F841B5E6
:101A70008547E380F9F0DA852D4597000000E7807F
:101A800020CB9389F4FFE38404E297000000E78011
:101A900060C893F7390091EB83260480032709007F
:101AA00093074900E396E6E03E89CE84D9BFB54767
:101AB0006399F9001305900B97000000E78080C33D
:101AC000FDB3B1471305B00AE388F9FE9947639760
:101AD000F904B7050800B365BB002D459700000069
:101AE000E78000C581448D4BA14997000000E78045
:101AF00060C263967401832704802320F900850463
:101B0000E39534FF8327048013172B0163550700E7
:101B10002312F90069BB2322F90051BB9D47639F43
:101B2000F90281451305B00497000000E78040C02A
:101B3000BD442320090023220900FD59970000001D
:101B4000E78040BD93F77400CA9703C70700FD14F0
:101B5000398D2380A700E39334FF91BBA14763979E
:101B6000F90697000000E780A0C28144630D0B00D6
:101B70008D479304C0036308FB00930400056304CE
:101B80008B01930440041375C507E30295D21945F0
:101B900097000000E78000B697000000E780A0B63D
:101BA000054597000000E780E0B426859700000017
:101BB000E78020B7094597000000E78080B69700CE
:101BC0000000E780E0BCE31405CE0DB39147639FAE
:101BD000F9001305600697000000E780A0B19700A8
:101BE0000000E78040B213059009F9B5E38109CC04
:101BF000F1547DB9BD660147173600001306462E25
:101C0000938606A685458347060093F7F70F91C391
:101C100082800507E3F9E6FE973700002382B72CA0
:101C2000DDB77D166206618693178601E18763D46E
:101C3000070001458280931726003307F500AE9711
:101C400018439C4363E7E7007D16E37FF7FC7D556F
:101C5000828005458280FD15E205E18513978501A7
:101C6000618793F7F50F63480700FD15139725006B
:101C70002A97584365D713851700620561858280CE
:101C80003308B5021C4283A80600B335B502C297DB
:101C900033B50701AE98469585486367B5006394F0
:101CA000A50063E3070181480C43C6950CC388C2B5
:101CB0001CC2828081471397870161876343B70005
:101CC0008280139727002A97232007008507E5B70E
:101CD0008147014793968701E18663C5B6001335B6
:101CE0001700828093962700AA9694428507558F05
:101CF000D5B793D755408A07AA979C430545331516
:101D0000B5007D8D828017F3FFDFE702833D2A84D3
:101D100097000000E78060F405C5931725003E9406
:101D20000327C4FF814711EB7D1516053E9542053B
:101D3000418517F3FFDF6700033D05838507E5B79E
:101D40000145C5BF81471397870161876343C7007A
:101D5000828013972700B386E50094422A9785076F
:101D600014C3D5B77D1662066186014793178601B5
:101D7000E18763D50700133517008280931726008B
:101D8000B306F500AE9794429C437D16B58F5D8FE8
:101D9000F1BF8A05AA9501476363B500828083A6D7
:101DA000C5FFF11593D71600D98F9CC11397F60183
:101DB000E5B72A830148014701456343D700828084
:101DC000B387050183A80700B30706019C43C697A4
:101DD000AA976384F80033B517010507B308030118
:101DE000620723A0F80061871108C1BF2A83014759
:101DF0008147014563C3D70082803388E50083288B
:101E00000800330EE600032E0E003388A840330886
:101E1000C8416384080133B508018507B308E300AE
:101E2000E20723A00801E1871107E9B717F3FFDFF5
:101E3000E702232B0111B286B2842E86AA850A8579
:101E400097000000E780C0FA2A84A6850A859700DB
:101E50000000E78020E833348000060413351500C5
:101E6000018D056117F3FFDF6700E32917F3FFDF3B
:101E7000E702A3244111AA89AE8A328BB68402C23A
:101E800002C402C60144131C8401135C8C416349E3
:101E90009C02939B1400FD1B0549138CF4FFF15C1D
:101EA00033048901620461846340740792478E049D
:101EB000CE9423AEF4FE410117F3FFDF67006323E6
:101EC00013192400B30B2B01014A93172A00D6974C
:101ED00083A50B0088437800340050009700000071
:101EE000E78040DA050A93178A01E187F11BE35E78
:101EF000FCFC92474E9905042320F900A2473EC2FC
:101F0000B24702C63EC441B7131A8901135A8A4127
:101F1000131D240093178A01E18763CF970092472E
:101F20000A044E941CC0A24705091379F90F3EC25A
:101F3000B24702C63EC4ADB7B3079A0313152A00D1
:101F400056950841780034005000050AEA97DA9760
:101F50008C4397000000E780E0D26DBF197106C284
:101F600012C416C61AC81ECA22CC26CE2AD02ED219
:101F700032D436D63AD83EDA42DC46DECAC0CEC2C9
:101F8000D2C4D6C6DAC8DECAE2CCE6CEEAD0EED2F9
:101F9000F2D4F6D6FAD8FEDA971500009385859923
:101FA0008841E700050092402242B2424243D243B8
:101FB0006244F244025592552256B2564257D257C5
:101FC0006258F25806499649264AB64A464BD64BBD
:101FD000664CF64C065D965D265EB65E465FD65F45
:101FE0000961730020300000972100209381810156
:101FF000175100201301018117F5FFFF1305C500DC
:102000009705002093850500171600201306C6FDCE
:1020100063FAC5008322050023A055001105910530
:10202000E3EAC5FE170502001305C5FB971500205E
:102030009385C5FB171600201306C66563FAC50015
:102040008322050023A0550011059105E3EAC5FE92
:102050001715002013050564974500209385053466
:102060006377B500232005001105E36DB5FEFD4241
:10207000739002BC8D4273904280B722000093821D
:10208000828873900230970200209382A2F793E235
:10209000320073905230975200009382228A7390DC
:1020A00012346FB0F47573002030397101436EC67D
:1020B00019A0397141536AC866CA62CC5ECE19A0B4
:1020C000397101535AD056D252D44ED64AD826DA54
:1020D00022DC06DE33016140828241114AC026C201
:1020E00022C406C68282B24D4101024D924C224C5E
:1020F000B24B4101024B924A224AB2494101024984
:1021000092442244B240410182803D432A87637356
:10211000C3029377F700BDEFADE5937606FF3D8AE6
:10212000BA960CC34CC30CC74CC74107E36BD7FE30
:1021300011E28280B306C3408A0697020000969699
:102140006780A6002307B700A306B7002306B700E1
:10215000A305B7002305B700A304B7002304B70005
:10216000A303B7002303B700A302B7002302B700FD
:10217000A301B7002301B700A300B7002300B700F5
:10218000828093F5F50F93968500D58D9396050182
:10219000D58D61B7939627009702000096968682A8
:1021A000E78086FA9680C1171D8F3E96E374C3F8C8
:1021B000A5B73367B500FD530D8B79E7B7877F7FF0
:1021C0009387F7F710419441B372F6003363F6003A
:1021D000BE92B3E262006397720C6318D606504158
:1021E000D441B372F6003363F600BE92B3E26200EC
:1021F0006398720A631BD60410459445B372F600C7
:102200003363F600BE92B3E262006391720A631E0A
:10221000D6025045D445B372F6003363F600BE9241
:10222000B3E26200639A72086311D60210499449BE
:10223000B372F6003363F600BE92B3E262006393BA
:1022400072085105D105E30FD6F6131706019397CF
:102250000601631CF7001357060193D706013305E7
:10226000F7409375F50F91E982804183C18333056F
:10227000F7409375F50F91E182801377F70F93F78D
:10228000F70F3305F74082800346050083C605003B
:10229000050585056313D60065FA3305D6408280AF
:1022A00011059105E312D6FE014582802105A105A5
:1022B000E31CD6FC014582803105B105E316D6FC4E
:1022C000014582804105C105E310D6FC01458280AD
:1022D000B717004003C777051377E70FA38BE70411
:1022E000130700F8A38DE7043D47238CE704130789
:1022F0005003A38CE70403C7A7051377D70F238DDB
:10230000E7048280B717004003C7E7020D89411137
:102310001377C70F498F93068008F3B6068093F6AC
:10232000860836C601000100930670052380D70495
:10233000930680FA2380D704010001002387E70277
:1023400023800704B247F3A7078001000100410181
:10235000828041112A83014E930E407E130F001993
:10236000930F400663E56E129308001913034006AD
:10237000B3781503854E0D4FA14F337365020D8958
:102380001335150063EFBE121308F6FF79467298F5
:102390004208135808013307C70213D61700BE07B7
:1023A00032976146B3F6C60213068070B386C60242
:1023B0003697A166F58F42075D8FB716004083C739
:1023C000F60293F70708A303F1000346710083C7E1
:1023D000F60293F70708E394C7FE83477100B71628
:1023E000004093F7F70F6388071293078008F3B74D
:1023F000078093F787083EC401000100B71700402B
:10240000930670052380D704930680FA2380D704AF
:102410000100010023AA070383C6170393E60608F9
:10242000A388D70223800704A247F3A707800100EF
:1024300001001166B71700407D16D45BC85F938515
:102440004703A98EF18EF5FA93068008F3B606804D
:1024500093F6860836C601000100930670052380B6
:10246000D704930680FA2380D7040100010098C1A5
:1024700003C7170313670704A388E7022380070431
:10248000B247F3A7078001000100410182807D135C
:102490003368E3039308E016630E08003368F30320
:1024A0009308D016630808009378330093B8180097
:1024B0009388D81633081E01131E0801135E0E01FF
:1024C00055B56393E5030548638608000148630337
:1024D00003002A8871087298FD15131E0801C205B1
:1024E000135E0E01C18179BD13F8150063F4BF00BE
:1024F0007908D5B713381800E5BF83C7F60293F7FC
:102500000708A303F1000346710083C7F60293F79F
:102510000708E394C7FE8347710093F7F70FF1DFD5
:10252000E9B531714AD966CB06DF22DD26DB4ED70D
:1025300052D556D35AD15ECF62CD6AC96EC7AA8C26
:1025400002D897100000E78020B12A8993078008FD
:10255000F3B7078093F787083EDA01000100B71749
:102560000040130770052380E704130780FA2380D7
:10257000E7040100010003C7F7021377770FA38771
:10258000E70203C7F70213678700A387E7022380E8
:102590000704D257F3A70780010001000545970003
:1025A0000000E78060D6130780C13347E902116A53
:1025B00093070AE893065002BD69930BA004814A71
:1025C000014B13048008930470057D1AB347F90288
:1025D0003307D7023EC0FD873ECC938709A69309F7
:1025E000803E3347F7023AC27D873AC43347390306
:1025F0008549B399990193D93940B306D702B30BF2
:102600007703B3C6F602B3CBFB0236C6FD8636C8E7
:1026100093D6FB4136CEB7460F0093860624334946
:10262000D9028566938606FAB3969601B389E902C4
:10263000130760553309D90293060010B389E902E4
:102640003349D902B3C9F9029316390036CA37198A
:102650000040FD8636D0930D090493D7F9413ED250
:10266000F336048093F6860836DC010001009307F8
:1026700070052380FD00930680FA2380DD000100B1
:1026800001008346390593F6860FA309D9048346D2
:10269000390593E61600A309D90423800D00E256FC
:1026A000F3A6068001000100130C80FA116DF336C9
:1026B000048093F6860836DE01000100930770055A
:1026C0002380FD0023808D01010001008346390530
:1026D000216693E60602A309D90483560905B3E6E9
:1026E000A6012318D90483560905D18E2318D904CD
:1026F00023800D00F256F3A60680010001008346F8
:10270000390593F606026381061A03463905218AC4
:102710006DDE081897100000E7800098733604807B
:1027200013768608B2C20100010023809D00238039
:102730008D0101000100B717004003C6370513766D
:10274000F60DA389C70403C6370513660602A389DD
:10275000C704835609052166B3E6A6012318D904E8
:1027600083560905D18E2318D90423800D0096467F
:10277000F3A60680010001008346390593F60602A0
:10278000638B061483463905A18AEDFE970000206D
:10279000E7806090AA8636D497000020E780A08F5B
:1027A000A256E30AD5FE835609054255B3E6A601B3
:1027B0002318D90497100000E780C08F834639059D
:1027C000A18AEDDE03560905834629058247337643
:1027D000CA00B306DA0293D5F641B296B388F64042
:1027E000E24733B8C6002E983308F840A247B3B684
:1027F00016013308D84063C70701631DF8009247EC
:1028000063FA1701C247634FF80E63950701B24799
:1028100063EAF80E894663E9660FF24693151800DD
:1028200013D3F8015E8613951800B365B30042D642
:1028300046D497C00100E780E0E13258050B137BD6
:10284000FB0F63470001631A0838A25863870838F2
:1028500013081500B336A800B69513D6F5013298C3
:10286000B336C800AE9613581800FE06B3E606014C
:102870007336048013768608B2C6010001002380F7
:102880009D0023808D01010001000356C902B2960C
:10289000C206C1822316D90223800D00B646F3A6D4
:1028A00006800100010021B5F336048093F6860806
:1028B000B6C00100010023809D0023808D0101002E
:1028C00001008346390593E60602A309D904238053
:1028D0000D0086460DB5F336048093F68608B6C41F
:1028E0000100010023809D0023808D010100010073
:1028F0008346390593E60602A309D90423800D0017
:10290000A646BDB5E30B0BF0F336048093F68608BC
:10291000B6C801000100930680FA23809D00238041
:10292000DD00010001008346390593F5FC0F93F6A5
:10293000860FA309D90483463905CD8EA309D9048E
:1029400023800D00C646F3A6068001000100130592
:1029500080FA03463905930639051D8A631C9629BA
:102960007336048013768608B2CC0100010013068A
:1029700080FA23809D002380CD000100010003C662
:1029800006001376F60D2380C60003C60600136604
:1029900006022380C600835609051166D18E2318CE
:1029A000D904835609052166D18E2318D9042380C2
:1029B0000D00E646F3A6068001000100130680FA2A
:1029C0008346390593F60602638006268346390559
:1029D000130C3905A18AFDDA081897000000E7807A
:1029E000A06BF336048093F68608B6D00100010090
:1029F000930680FA23809D002380DD000100010002
:102A000083460C00116693F6F60D2300DC00834626
:102A10000C0093E606022300DC0083560905D18EE4
:102A20002318D904835609052166D18E2318D904A9
:102A300023800D008656F3A60680010001001306D0
:102A400080FA8346390593F60602638A0620834698
:102A50003905A18AEDFE97F0FF1FE780C0632A8C3D
:102A600097F0FF1FE7802063E30C85FF835609057D
:102A700011664255D18E2318D90497000000E780D3
:102A800060638346390513063905A18AFDDAF336FA
:102A9000048093F68608B6D401000100930680FAFC
:102AA00023809D002380DD00010001008346060095
:102AB00093F6F60D2300D60023800D00A656F3A64C
:102AC0000680010001008356090503462905D24707
:102AD000B376DA003306CA021305800C9355F6412B
:102AE0003696330DF6408257333CD6002E9C333653
:102AF000A601330CFC40330CCC40330885039256BE
:102B00004E86B335A5033305A503C29597C00100D2
:102B1000E78040B463468001631E0C16630C0D16FB
:102B2000130615003335A6002E959356F5013696FB
:102B3000B335D600AA959396F50105828585D18E89
:102B40006346B000639D051A638B061A0356C902DB
:102B500015823305D6003336C500B2956348B00000
:102B6000639105241306F00F637DA622894663F363
:102B7000561593078008F3B7078093F78708BED6EA
:102B80000100010037170040930770052300F70488
:102B9000930780FA2300F704010001008356C7025F
:102BA00089678117D58FC207C1832316F7022300D7
:102BB0000704B657F3A7078001000100FA506A54D2
:102BC000DA544A59BA592A5A9A5A0A5BFA4B6A4C49
:102BD000DA4C4A4DBA4D296182801308F5FF33352E
:102BE000A800FD152E951356F5013298B336C8008E
:102BF000AA9695B9F336048093F68608B6CA010002
:102C0000010023809D002380AD0001000100834668
:102C10003905CD8EA309D90423800D00D646F3A62D
:102C200006800100010035B3F336048093F6860870
:102C3000B6CE0100010023809D002380CD0001005D
:102C400001008346390593E60602A309D9042380CF
:102C50000D00F646F3A606800100010095B3F33699
:102C6000048093F68608B6D20100010023809D00FF
:102C70002380CD00010001008346390593E606025A
:102C8000A309D90423800D009656F3A606800100FF
:102C9000010045BB9306F5FF33B5A600FD152E9543
:102CA0009355F501AE96B3B5B600AA951396F50106
:102CB000858269B5F336048093F68608B6D801009C
:102CC0000100930680FA23809D002380DD0001002F
:102CD00001008356C9020566011693F6F60FD18EE0
:102CE000C206C1822316D90223800D00C656F3A660
:102CF000068001000100850A93FAFA0F95B233E6C7
:102D0000B60045C20356C9023305D0403338A0008F
:102D1000B305B040B385054115826345B000D1E1EC
:102D20006371A608894663F0560593078008F3B7D8
:102D3000078093F78708BEDA01000100B71700404B
:102D4000130770052380E704130780FA2380E70444
:102D50000100010003D7C7027D8B2396E702238081
:102D60000704D65781BDF336048093F68608B6DC97
:102D700001000100930680FA23809D002380DD007E
:102D8000010001008356C9020566011693F6F60F8D
:102D9000D18EC206C1822316D90223800D00E656C9
:102DA000B9B793078008F3B7078093F78708BEDEAB
:102DB0000100010037170040930770052300F70456
:102DC000930780FA2300F704010001000356C702AD
:102DD00093975600B297C207C1832316F7022300C8
:102DE0000704F657C1BB914763EEB70217D701003E
:102DF000130787238A05BA959C41BA978287B7172C
:102E0000004003A7470B1345F5FF698F23AAE70A84
:102E100003A7070B698F23A8E70A03A7070A798D81
:102E200023A0A70A8280B717004083A6470B134749
:102E3000F5FFF98E23AAD70A83A6070B558D23A881
:102E4000A70A83A6070A758F23A0E70A8280B7170F
:102E5000004003A7470B498F23AAE70A03A7070BE4
:102E60001345F5FF45BFB717004083A6470B13472F
:102E7000F5FF758F23AAE70A03A7070A598D4DB7F7
:102E8000B717004003A7470B498FEDB7914763EE93
:102E9000B70217D701001307671A8A05BA959C4134
:102EA000BA978287B717004003A7470D1345F5FF70
:102EB000698F23AAE70C03A7070D698F23A8E70CE6
:102EC00003A7070C798D23A0A70C8280B7170040B9
:102ED00083A6470D1347F5FFF98E23AAD70C83A6C7
:102EE000070D558D23A8A70C83A6070C758F23A06B
:102EF000E70C8280B717004003A7470D498F23AA2C
:102F0000E70C03A7070D1345F5FF45BFB7170040B2
:102F100083A6470D1347F5FF758F23AAE70C03A778
:102F2000070C598D4DB7B717004003A7470D498FC0
:102F3000EDB7797122D43714004026D24AD0035914
:102F400024028354040206D64209C2044ECE52CC57
:102F500056CA13590901C1802DE11379F9F793F489
:102F6000F49F4209C20413590901C18093078008E4
:102F7000F3B7078093F787083EC401000100930769
:102F800070052300F404930780FA2300F404010081
:102F90000100231124032310940223000404A247F8
:102FA000F3A7078001000100B25022549254025945
:102FB000F249624AD24A45618280B7F507008146EC
:102FC0003000B105194597000020E7808081A247B5
:102FD00013972701E34A07FC1369090893E40440A7
:102FE00093098008F3B7098093F787083EC0010072
:102FF0000100930A700523005405130A80FA230088
:10300000440501000100231124032310940223002E
:1030100004048247F3A7078001000100294597F0C7
:10302000FF1FE7802031F3B9098093F989084EC268
:1030300001000100230054052300440501000100A4
:103040008357040293E707202310F40223000404AB
:103050009247B9B7B7170040884742054181937737
:10306000050491EB9377F5013755E80113050580C9
:103070003345F50282809377050C130700046397AC
:10308000E7009377F50137459C1CCDB72165130503
:1030900005D0828037E700E01C435443A183E20659
:1030A000D58F1CC1FD572320F7182322F7188280E3
:1030B00013178500B7E700E023A0E710618123A282
:1030C000A7108280B7F700E08847CC47828081470D
:1030D00037370040A14663C4C7003285828003456C
:1030E000B740E38EA6FE3385F5000345050085074E
:1030F0002304A740CDB797070020938727EF9C4371
:1031000017370020130787293E95636EE5001737B0
:1031100000201307274F6368A70017070020232705
:10312000A7EC3E858280FD57EDBF8280411122C40D
:1031300006C62A8497000000E78000F22947B307FB
:10314000E502B2408D83B3D7870222449507B3D7F7
:10315000E70237370040C207C1832316F700410159
:103160008280411137150E0006C697000000E780E7
:1031700020FCB7370040130770F82381E7000D47A4
:10318000A381E70013070004A380E7000547238716
:10319000E700B24041018280373700408347270073
:1031A0001A0593F7F703C98F93F7F70F2301F70079
:1031B0008280B737004003C7170019C9D98DA38093
:1031C000B70003C70700136787002380E7008280EA
:1031D00093C5F5FFF98DA380B7008280AE872A875B
:1031E000B736004021463738004089E71703000012
:1031F0006700E3F383C8B600E30916FF05078348B9
:10320000F7FFFD17C20723041801C183F9BF41115D
:1032100022C406C62A8497000000E780E0E329471D
:10322000B307E502B2408D83B3D7870222449507E6
:10323000B3D7E70237370040C207C1832316F740F0
:1032400041018280716541111305052006C6970072
:103250000000E78000FCB7370040130770F82381B7
:10326000E7400D47A381E74013070004A380E74030
:1032700005472387E740B24041018280CC4141119C
:1032800006C6328503C6150083C5050022064D8E8D
:1032900042068D654186138875A2630C0611634B47
:1032A000C804138845A26300060D634AC8009385CD
:1032B00035A26301B6082390060029464DA0138865
:1032C00055A26305060D938565A2E316B6FE8D45EE
:1032D0001D4663E6E5081146198E63F3C7003E8676
:1032E000B7E704002390C600FC4797D501009385FB
:1032F00025D79DA0138895A263030611634E060D82
:103300001388A5A263000613938505A5E315B6FAF5
:1033100099451D4663E5E504198E63F3C7003E86B3
:10332000B7E704002390C600FC479705002093856B
:1033300025D61DA09D451D4663E3E5022146198E55
:1033400063F3C7003E86B7E70400FC472390C6003E
:103350009705002093858534BA9582970146B2403F
:10336000328541018280AD451D46E3EAE5FE3146E6
:10337000198E63F3C7003E86B7E704002390C600AA
:10338000FC4797D50100938525D0F9B7B1451D4677
:10339000E3E7E5FC3546198E63F3C7003E86B7E7E1
:1033A00004002390C600FC4797D501009385C5CE45
:1033B00065B78D451D46E3E4E5FA1146198E63F3C2
:1033C000C7003E86B7E704002390C600FC4797D5A8
:1033D00001009385A5C949B78D451D46E3E1E5F890
:1033E0001146198E63F3C7003E86B7E704002390A9
:1033F000C600FC4797D501009385C5CBB1BFA54555
:103400001D46E3EEE5F42946198E63F3C7003E86B8
:10341000B7E704002390C600FC4797D501009385C9
:10342000A5C51DBFB5451D46E3EBE5F23946198E2E
:1034300063F3C7003E86B7E704002390C600FC474D
:1034400097D501009385C5C001BFB7E7040003A36A
:103450000713970600209386A6C24146A545170587
:1034600000201305E5B80283797126D252CCAE84D0
:103470002A8A97D501009385E5C517D50100130564
:10348000E5C706D63AC622D44AD0368432894ECE13
:1034900056CA97B00100E7802067A28517D50100C2
:1034A0001305C5C697B00100E7800066294597B0AF
:1034B0000100E780406A83C7840093F70702F9EFB1
:1034C00083C904008947054532476391F90AD4400E
:1034D00083C7160083C60600A207D58FC166138670
:1034E00016FE638DC7028D16638BD7088D66938693
:1034F00026902945639CD706B7E70400A28622548C
:1035000003A34714B250F249D24A4A86A68502590B
:1035100092545285624A8547456102832D4539E7B9
:10352000130A700F354563638A04B7EA040083A762
:10353000CA04C8442286CA8582978149630A440125
:10354000C84483A78A0433068A408145229582971E
:10355000970700209387073D9C43014581CB9C43FF
:1035600091C74E852286CA8582970145B250225462
:1035700092540259F249624AD24A456182802D45ED
:1035800075F79307700F3545E3E287FEB7E7040050
:10359000FC47C8442286CA8582975DBF2145F9B79A
:1035A0002D455DE703C505000947631FE50803A82E
:1035B0004500411106C6034718003285034608003E
:1035C00022074168518F930828FE6307170563E9B6
:1035D000E80005186303070323900600294591A816
:1035E000130648FE630AC7041518E31707FF1546BC
:1035F0003E87637BF600154701A81306700F3E87D0
:103600006374F6001307700FB7E704002390E60019
:10361000FC471316070111A83E8691C30546B7E77C
:103620000400FC472390C6004206CC4541828297A5
:103630000145B24041018280130600083E87E375D0
:10364000F6FC13070008C9B72390060005458280E1
:103650008280416779176304E504411122C406C6DC
:1036600085472A84639FF500B7E70400228522443A
:10367000B24003A38713970500209385E5294101F4
:10368000028389476399F500B7E7040083A7070B16
:103690008545829771D9B24022444101828082805F
:1036A000411122C437E404008327841326C2AA846C
:1036B000416506C697050020938505267D158297EE
:1036C0008327C40A170500001305E5F8858882974B
:1036D00095C0032304132244B2409244970600206D
:1036E000938686AC4146C545170500201305C59A4B
:1036F00041010283B240224492440145410182804B
:1037000019C59707002023AFA720014582804545B2
:103710008280011122CC06CE26CA4AC84EC69147E5
:10372000094463EDA70417D70100130767990A0539
:103730003A951C41AE84B285BA9782879387F4FF8D
:10374000C207C1831307600F61446369F702B7E9D9
:10375000040083A7C904170900201309A9F42686C9
:103760004A8582971306700F01446389C40083A7BA
:103770008904058E81453305990082972285F240A0
:103780006244D2444249B24905618280854761441E
:10379000E396F4FEB7E70400FC4705461705002052
:1037A0001305C5FF82970144D1BF9307700F614491
:1037B000E396F4FCB7E70400FC471306700F170507
:1037C00000201305E5FDF9BF930700086144E39766
:1037D000F4FAB7E70400FC471306000817050020B9
:1037E0001305850BC1B795476144E399F4F8B7E732
:1037F0000400FC47154617050020130525125DB788
:10380000411126C2B7E4040083A7C41322C44AC0EE
:1038100006C62E8497050020938505102A89829775
:10382000058905C5970700209387078783D7A70BCE
:10383000A28503A3440D2310F4002244B240924415
:103840004A850249014641010283B2402244924422
:103850000249494541018280970700202386070CD1
:103860009707002023A4070CB717004003A7070CF5
:10387000B706C0FFFD16758F23A0E70C03A7070D41
:10388000B7064000558F23A8E70C03A7070C3D9B04
:1038900023A0E70C03A7070D1367070123A8E70C74
:1038A0008280B717004003A5470C83A7470C5981B6
:1038B00013451500C18B058999E31365250097070A
:1038C000002083C767066380A70297070020238D27
:1038D000A70411C9970700209387470503A3070092
:1038E0006303030002838280114517F3FFFF670023
:1038F00083C3011122CC06CE3714004026CA4AC821
:103900004EC652C483447405034AB40583498405F2
:103910000349940597F0FFFFE780C09B8347A40508
:1039200093F4F40F137AFA0F93E71700230DF404BE
:1039300093F9F90F1379F90FB717004003C7A705DB
:10394000058B6DFF03D5C705A38D4705238C370570
:10395000A38C2705A38B9704F2406244D2444249CA
:10396000B249224A0561828041119397050122C420
:1039700006C626C2C1872E8463DC0700B7E40400B4
:10398000FC54829719C1BC5482972165218D15A8DA
:1039900093F7150013C515008DE793F725009DC714
:1039A00097000000E78020F0B7E70400BC4F130643
:1039B000000A8945170500200345C5F7829713457E
:1039C0002400B24022449244410182809397250111
:1039D00063D80702B7E4040083A7C41E8297970048
:1039E0000000E780A0F0BC4C3756070013060630F5
:1039F0008965170500200345E5F38297096579B7C6
:103A0000939715010145E3DE07FA17C50100130579
:103A1000E57797B00100E7800027B7E70400BC4FC7
:103A2000130600649165170500200345A5F08297F1
:103A30001165A9BF1D71A2CC37E404005C5C485835
:103A400086CE494697C501009385C56F829711E9D7
:103A500017C501001305457097B00100E780A0224B
:103A600001A0B7F600E0795798CAFD57DCCA056790
:103A7000B7E700E023A0E7101306F00290C223A0EE
:103A8000E71801000100370700201847130600045B
:103A900081459706002023ADE6E84157A38AE74019
:103AA0003C4408088297971700209387A7853EC853
:103AB000856713870740938757D1231AE1002312A4
:103AC000F1021307B00F97F7FFFF9387E75F23100B
:103AD000E1023ED81547970700009387C7E1B7F585
:103AE0000700A30FE1003EDC05479707000093871E
:103AF000E7DF81463000E10519452301E1023EDEA2
:103B000097F0FF1FE780E0CD180881479946300005
:103B10003E960346060085070507A30BC700E398FA
:103B2000D7FEC24791C70357410185676373F7000A
:103B300001A0B7E7040083A7470A08088297AA856F
:103B400011C917C501001305656297B00100E78030
:103B5000A0FB01A0F640664425618280411126C287
:103B6000B7E4040083A7040806C622C417050000B2
:103B70001305C5DF8297170400201304A4DB23007C
:103B8000A40097000000E780800297000000E78013
:103B9000E0CC03450400224403A38405B2409244D0
:103BA00013060032896541010283797106D622D459
:103BB00013078008F337078093F787083EC2010098
:103BC0000100B7170040930570052380B704130662
:103BD00080FA2380C7040100010083C6F70293F630
:103BE000A60FA387D702238007049246F3A6068078
:103BF0000100010073370780137787083AC401007A
:103C000001002380B7042380C7040100010003C71B
:103C1000F70213672700A387E70223800704A24760
:103C2000F3A7078001000100054597E0FFFFE7804B
:103C3000A06D97000000E78060CB01478146814777
:103C4000054685451305407E97E0FFFFE780A0709D
:103C500037E404003C446800514681458297B70729
:103C6000C0A83EC8B787E803938707D03ECA97E746
:103C7000FF1F9387C7743EC67C5868008297B25076
:103C8000225445618280411197D50100938545B248
:103C900017C501001305854606C697B00100E780E9
:103CA000A0E617D50100130565C997B00100E780AC
:103CB000A0E5B2402945410117B301006700A3E91F
:103CC000411197D501009385E5AF17C50100130594
:103CD000E54206C697B00100E78000E317D5010072
:103CE000130585C497B00100E78000E2B240294582
:103CF000410117B30100670003E6411122C406C663
:103D0000834705002A849DC797D50100938545B157
:103D100017C501001305853E97B00100E780C0DE9E
:103D20004C4017D501001305A5D397B00100E780DB
:103D3000A0DD3DA058410DEF97D50100938545AE1C
:103D400017C501001305853B97B00100E780C0DB74
:103D500017D50100130545D297B00100E780C0DAFE
:103D60002244B2402945410117B301006700A3DE98
:103D7000A1679386D7036313D70297D50100938574
:103D800025AA17C501001305653797B00100E78024
:103D9000A0D717D50100130525CF7DBFED0797D517
:103DA00001009385E5A717C5010013052535631BA1
:103DB000F70097B00100E78020D517D50100130563
:103DC000E5CD59BF97B00100E78000D44C4017D52E
:103DD00001001305A5CE91BF411197D50100938530
:103DE000A59F17C501001305653106C697B00100F0
:103DF000E78080D1B2402945410117B30100670037
:103E000083D5797122D426D24AD02E842A8981453D
:103E1000B2844800714606D697E0FFFFE780202F66
:103E200097F7FF1F93874759DC4783D70700231471
:103E300021012313F10097500000E78000E485473B
:103E4000A305F1009307401F3EC6FD572305A100BF
:103E5000230AF10097500000E78060F62686A285CD
:103E6000480097500000E78020E4B250225492545A
:103E70000259456182809727002023980798972749
:103E8000002023810788B7E70400BC47411106C61C
:103E900041468145170500201305453582971707D0
:103EA00000200347A7369307F00A6315F70293072C
:103EB000F0F8894517050020130545351707002040
:103EC0002306F73497070020A38207349760000089
:103ED000E78000A097600000E78020CC814537058F
:103EE00004009707002023A1073097070020239B99
:103EF000072E970700202388072E97070020239777
:103F00000726970700202395072497070020239A68
:103F1000072C970700202393072E97300000E78097
:103F20000029014597600000E78080A397D5010034
:103F30009385058D17C501001305451C97B0010039
:103F4000E78080BC17D50100130585BD97B001003F
:103F5000E78080BBB2402945410117B301006700EB
:103F600083BF4111814617F6FF1F13062642854580
:103F7000170500200355851D06C697C00000E78081
:103F8000602A15C997D501009385458817C501009A
:103F90001305C51697B00100E78000B717D50100DB
:103FA000130505A897B00100E78000B6294597B032
:103FB0000100E78040BA97D501009385258517C594
:103FC00001001305A51397B00100E780E0B317D5F2
:103FD0000100130525A697B00100E780E0B229454E
:103FE00097B00100E78020B797F7FF1F9387C73C82
:103FF000DC47054797D50100938545812390E7006D
:1040000017C501001305850F97B00100E780C0AF09
:1040100017D50100130545A397B00100E780C0AE96
:10402000B2402945410117B301006700C3B24111F5
:1040300022C497C501009385E57F2A8417C5010036
:104040001305C50B06C697B00100E780E0AB4C40F6
:1040500017D501001305459A97B00100E780C0AA63
:10406000294597B00100E78000AF0347040093079C
:10407000F00F631FF70297C501009385A57B17C555
:1040800001001305A50797B00100E780E0A74C40A9
:1040900017D501001305459797B00100E780C0A62A
:1040A0002244B2402945410117B301006700A3AA89
:1040B000B240224441018280411122C426C22A8496
:1040C000AE8417C501001305650397C501009385EC
:1040D000257206C697B00100E78000A317D501003E
:1040E000130585A297B00100E78000A2294597B08B
:1040F0000100E78040A697C501009385656F97078B
:1041000000202395870417C50100130525FF0544EA
:1041100097070020239A970297070020239787028A
:10412000971700202393976E97B00100E780C09DFA
:104130009715002083D5656D17D501001305459DA2
:1041400097B00100E780409C294597B00100E780C7
:1041500080A0971700202387875A97F7FF1F938720
:10416000A725DC4703D70700C167FD176312F702D5
:104170002244B7E70400B240924403A3870517F531
:10418000FF1F0345A57B1306000A854541010283F5
:10419000B2402244924441018280B1C1411122C403
:1041A00017C50100130585F52E8497C50100938579
:1041B000656306C697B00100E7800095A28517D514
:1041C00001001305A59397B00100E780E093224416
:1041D000B2402945410117B301006700C3978280AF
:1041E000011122CC06CE26CA4AC84EC693F7150046
:1041F0002E84B1CF97000000E780E0D6930710F837
:10420000170700202304F7009707002083D7C7F380
:1042100017070020A30CF7FE17050020130505FF64
:10422000A1839145170700202303F7FE970700207D
:10423000A38F07FC97500000E780806913451400A6
:10424000F2406244D2444249B2490561828093F708
:1042500005108DC7054597500000E7806070171561
:1042600000200355855A97500000E780C03B9720F7
:104270000000E780C00B13450410D9B793F7250061
:10428000E9CF170700200357E7F569C7AD64B719F1
:1042900000409384A4AA23A0990097060020938647
:1042A000A6F4944297D701009387878917060020C8
:1042B000034666F3814517050020130525F3977023
:1042C0000000E780E01123A0990097F7FF1F2399D2
:1042D000A7FE2A8941C197C501009385E55917C5F5
:1042E00001001305A5E197B00100E780E081CA85D0
:1042F00017C50100130545F897B00100E780C0809D
:10430000294597B00100E780008597070020239B8F
:1043100007EC930710F8170700202309F7EE97071B
:10432000002083D767E217070020A301F7EEA183DF
:1043300017070020230DF7EC91458D471705002046
:104340001305C5EC17070020A303F7EC97500000F6
:10435000E780005813452400E5B593F74500D1C325
:1043600097C501009385455117C50100130505D96F
:1043700097A00100E780407917C50100130585F17A
:1043800097A00100E7804078294597A00100E780C9
:10439000807C930720F8170700202309F7E697078A
:1043A000002083D7A7DC17070020A301F7E6A1832D
:1043B00017070020230DF7E4854717070020A308FF
:1043C000F7E497500000E780809F17050020130551
:1043D000E5E3914597500000E780804F1345440086
:1043E00085B593F78500A9C797C501009385C54892
:1043F00017C50100130585D097A00100E780C070A4
:1044000017C50100130545EA97A00100E780C06FBA
:10441000294597A00100E7800074970700202393A7
:1044200007DC97700000E780800B1345840009BD0E
:1044300093F70501D1C3854517050020035505D322
:1044400097600100E78040C197C501009385C54290
:1044500017C50100130585CA97A00100E780C06A4F
:1044600017C50100130585E597A00100E780C06925
:10447000294597A00100E780006E930730F81707E1
:1044800000202305F7D89707002083D727CE1707EA
:104490000020A30DF7D617050020130525D7A1830B
:1044A0008D45170700202304F7D697500000E780BA
:1044B00020421345040169B393F70502D1C797C59C
:1044C00001009385653B17C50100130525C397A01F
:1044D0000100E780606317C50100130565E097A040
:1044E0000100E7806062294597A00100E780A0668F
:1044F000930740F817070020230AF7D097070020FA
:1045000083D707C517070020A302F7D0A183170799
:104510000020230EF7CE854717070020A309F7CE0A
:1045200097070020239607C297500000E780208954
:1045300017050020130585CD914597500000E780B1
:10454000203913450402EDB993F70504FDC397C55F
:1045500001009385653217C50100130525BA97A0A0
:104560000100E780605A17C501001305E5D897A040
:104570000100E7806059294597A00100E780A05D10
:104580009707002083C787C81307700A6386E7066A
:104590001307800A638CE7081307600A6393E70434
:1045A000930760F8170700202302F7C6970700203B
:1045B00083D727C317070020A30AF7C4A1831707CF
:1045C00000202306F7C4854717070020A305F7C47A
:1045D000B14517050020130565C397500000E7801B
:1045E000202F97400000E780807D13450404970743
:1045F0000020239807BEA9B1930770F81707002081
:104600002306F7C09707002083D7A7BD1707002010
:10461000A30EF7BEA18317070020230AF7BE854724
:1046200017070020A306F7BE994565B7930780F8E2
:10463000F1B793F705080145E38407C097C501006A
:104640009385852317C50100130545AB97A001008D
:10465000E780804B17C50100130585CB97A00100AB
:10466000E780804A294597A00100E780C04E930764
:10467000A0F817070020230BF7B89707002083D76F
:10468000E7B717070020A303F7B8A1831707002097
:10469000230FF7B6854717070020A30AF7B6970739
:1046A0000020239D07B497400000E7804071170564
:1046B00000201305A5B5914597500000E7804021E3
:1046C00013450408B5BE011122CC37E404005C5C3C
:1046D00006CE354697C501009385852717D501007D
:1046E000130505F6829711E917C501001305C5A644
:1046F00097A00100E780205901A097F7FF1F93873B
:10470000A7243EC4B7F507008567938707808146D5
:1047100017F6FF1F1306C622E10519453EC697E0AE
:10472000FF1FE780000C7C44194697F5FF1F938517
:104730002521170500201305A5A38297340017F63D
:10474000FF1F1306E61F97C501009385E57117C586
:1047500001001305E57297700000E780609D2A84D0
:104760001DCD97C501009385251017C501001305C0
:10477000E59897A00100E7802039A28517C50100C0
:104780001305051E97A00100E7800038294597A072
:104790000100E780403CF24062440561828097E07E
:1047A0000000E780600317C50100130565129760DC
:1047B0000000E780A09197A00000E780A0579760D5
:1047C0000100E78020BC17F5FF1F130565BB97604C
:1047D0000100E780C0A417C50100130565109760AC
:1047E0000100E780A0BC2A8497600000E780E0F722
:1047F00097100100E780009497800100E780202D4A
:1048000097700000E780C05397600000E780E06D7C
:1048100097300100E780605597C501009385C50476
:1048200017C501001305858D19C897A00100E78001
:10483000A02DA28517C501001305C514A1B797A027
:104840000100E780602C17C501001305E51597A04E
:104850000100E780602B294597A00100E780A02F89
:1048600097300100E780403197F00000E78000506A
:104870007DC185453705040097300000E78020930F
:1048800097C50100938545FE17C5010013050587EF
:1048900097A00100E780402717C5010013054512C6
:1048A00097A00100E7804026294597A00100E780F6
:1048B000802A97F7FF1F9387A79F83D707001717B3
:1048C00000202314F7F4854717170020230CF7E284
:1048D00097F7FF1F938747AEDC4703D70700C167F1
:1048E000FD176316F70097F0FFFFE780C06797702A
:1048F0000000E78000CF1305C51497700000E78023
:1049000000CF97200000E78040B497200000E780A8
:1049100000A217150020035545EF97500000E780CF
:1049200080D0054597500000E780800397C50100BF
:10493000938585F317B501001305457C97A0010009
:10494000E780801C17C501001305C50997A0010069
:10495000E780801B25BD97C501009385E5F017B55D
:1049600001001305A57997A00100E780E01917C59C
:1049700001001305E51A97A00100E780E01829451A
:1049800097A00100E780201D014569BF411122C4A5
:1049900037E404008327041A06C682979750000064
:1049A000E78020CC832704081705000013058583C2
:1049B000829797F7FF1F2383A7F817F5FF1F1305AB
:1049C000A59F97400000E78020722244B240410139
:1049D00017030000670063CFB7E70400FC471171BD
:1049E000A2DDCAD986DFA6DBCED72E8432892E86F9
:1049F000AA851705002013056581829717070020F7
:104A00001307C78083470700930680029387E70751
:104A100093F7F70FE3ECF610BA898A0717B701008E
:104A200013070777BA979C43BA9782878D4797C534
:104A300001009385A5E517B501001305256C630FEB
:104A4000F40097A00100E780200C17C501001305B2
:104A5000A5A297A00100E780200BBDA497A00100AC
:104A6000E780800A17C50100130585A297A0010001
:104A7000E7808009294597A00100E780C00D9307D2
:104A800020F8114697F5FF1F938545784A8517F75B
:104A9000FF1F230DF77697F7FF1FA38A077697F07E
:104AA000FFFFE78040362A841DC997C50100938522
:104AB000E5DD17B501001305656497A00100E780E7
:104AC000A004A28517C50100130545A097A0010009
:104AD000E7808003294597A00100E780C00797C5BC
:104AE00001009385A5DA17B501001305256197A08C
:104AF0000100E780600117C501001305659E97A0BE
:104B00000100E7806000294597A00100E780A0042C
:104B10004165930730FA054697F5FF1F9385056FAA
:104B20007D1517F7FF1F2303F76E97F0FFFFE78050
:104B3000802D2A841DC997C50100938525D517B5F9
:104B400001001305A55B97A00100E780E0FBA285AB
:104B500017C501001305859797A00100E780C0FAEB
:104B6000294597A00100E78000FFB7E70400BC4F8C
:104B70000566130606C8A14517F5FF1F034505DCAA
:104B80008297FE506E54DE544E59BE591161828098
:104B900091476303F40297C50100938525CF17B5AC
:104BA00001001305A55597A00100E780E0F517C5A2
:104BB00001001305259671BDB7E70400FC4F914530
:104BC00017F5FF1F034585D7829797C50100938589
:104BD000E5CB17B501001305655297A00100E780EA
:104BE000A0F217C501001305A59497A00100E78066
:104BF000A0F1294597A00100E780E0F5974000006B
:104C0000E780E01B914535A485476303F40297C50F
:104C100001009385A5C717B501001305254E97A080
:104C20000100E78060EE17C501001305E59115B599
:104C300097F7FF1F239C2753B7E704000566BC4F77
:104C4000130606C8C1450DBF8D476303F40297C51F
:104C500001009385A5C317B501001305254A97A048
:104C60000100E78060EA17C501001305A58FD5B3E1
:104C7000930740F8114697F5FF1F938525594A85FC
:104C800017F7FF1F2304F75897F7FF1FA381075853
:104C900097F0FFFFE78020172A84E30405EE97C50D
:104CA00001009385A5BE17B501001305254597A002
:104CB0000100E78060E5A28517C5010013050581A5
:104CC00097A00100E78040E4294597A00100E78014
:104CD00080E845BD9147E31CF4F6B7E70400FC4FBC
:104CE0009305000217F5FF1F034545C5829797C539
:104CF00001009385A5B917B501001305254097A0BC
:104D00000100E78060E017C5010013052587F1BDAC
:104D1000894763E3870297C50100938525B717B5D7
:104D200001001305A53D97A00100E780E0DD17C550
:104D300001001305E58531BB97F4FF1F83C4244DA3
:104D400097F7FF1F83C7974C97C50100938505B45C
:104D5000A20417B501001305653ADD8C97A0010088
:104D6000E78080DAA28517C501001305A58397A007
:104D70000100E78060D9C204294597A00100E780BF
:104D800080DDC1849305D4FF93960401C1824A86D5
:104D900093F5F50F17F5FF1F1305754797200000D2
:104DA000E780A044E35F90DC930750F817F7FF1FFC
:104DB000230EF74483C73900228697F5FF1F93859A
:104DC000E54485074A8517F7FF1FA302F74497F0CC
:104DD000FFFFE78040032A84E30505DA97C5010059
:104DE0009385C5AA17B501001305453197A00100A9
:104DF000E78080D1A28517C50100130525CFC9B56D
:104E0000894763E3870297C50100938525A817B5F5
:104E100001001305A52E97A00100E780E0CE17B58D
:104E200001001305E57935B197400000E78020F9CE
:104E3000A28517F5FF1F1305653D97500000E78019
:104E400020A981B38D476303F40297C501009385C0
:104E5000E5A317B501001305652A97A00100E780B7
:104E6000A0CA17B5010013056577E5B6B76602005D
:104E70000146B7750200054597E0FF1FE780609681
:104E8000930760F817F7FF1F2302F73897F7FF1F04
:104E9000A38F07369307000617F7FF1F230AF7367D
:104EA000894717F7FF1FA305F73697F7FF1F2382E0
:104EB000073697F7FF1FA38E0734C14717F7FF1F69
:104EC000230AF734930720F917F7FF1FA304F734D9
:104ED000314697F7FF1FA380A73497F5FF1F9385EF
:104EE000E5324A8597F7FF1F2387073297F0FFFFC8
:104EF000E78060F12A84E30605C897C50100938521
:104F0000E59817B501001305651F97A00100E7801C
:104F1000A0BFA28517B501001305C56D55B3B147F4
:104F20006303F40297C501009385459617B5010008
:104F30001305C51C97A00100E78000BD17B501004F
:104F40001305056D39B6B7E70400FC4F930500045F
:104F500017F5FF1F0345859E829797400000E78065
:104F600000E6B145F9B5914763E3870297C50100B3
:104F70009385C59117B501001305451897A0010049
:104F8000E78080B817B501001305456AD9B497F4D6
:104F9000FF1F83C4E42797F7FF1F83C75727A20487
:104FA000DD8C8E04B77702006D14BE942286A68530
:104FB00017B501001305C56897A00100E780C0B4CC
:104FC000B7E70400FC47228697F5FF1F9385552419
:104FD0002800829793160401C1823000A6850945F6
:104FE00097D0FF1FE780E07F2A8409C917B5010029
:104FF0001305C56697A00100E780E0C8930770F825
:10500000194697F5FF1F938565204A8517F7FF1FFF
:10501000230EF71E97F7FF1FA38C871E97F0FFFF45
:10502000E78060DE2A84E30E05B497C5010093850E
:10503000E58517B501001305650C97A00100E78011
:10504000A0ACA28517B501001305456295B9994733
:10505000630BF41297C501009385458317B50100D2
:105060001305C50997A00100E78000AA17B5010044
:1050700013054561F9BA914763E3870297C50100BB
:105080009385C58017B501001305450797A001005A
:10509000E78080A717B50100130545605DBA97F456
:1050A000FF1F83C4E41697F7FF1F83C75716A20498
:1050B000DD8C8E04B77702006D14BE942286A6851F
:1050C00017B501001305C55E97A00100E780C0A3D6
:1050D000B7E70400FC47228697F5FF1F9385551319
:1050E0002800829793160401C1823000A6850D45E1
:1050F00097D0FF1FE780E06E2A8409C917B5010029
:105100001305C55C97A00100E780E0B7930780F81E
:10511000194697F5FF1F9385650F4A8517F7FF1FFF
:105120002306F70E97F7FF1FA384870E97F0FFFF64
:10513000E78060CD2A84E30605A497B50100938536
:10514000E57417B50100130565FB97A00100E78022
:10515000A09BA28517B501001305855895B6994700
:105160006303F40297B501009385457217B50100FA
:105170001305C5F897A00100E780009917B5010055
:1051800013058557F9B0B7E70400FC4F93050004F9
:1051900017E5FF1F0345857A829797400000E78057
:1051A00000C2994579B18D476303F40297B50100B8
:1051B0009385C56D17B50100130545F497A001004F
:1051C000E780809417B501001305855459B017B5D1
:1051D00001001305E55497A00100E780C0AA13055C
:1051E000C01297D0FF1FE780C015014597E0FFFF71
:1051F000E78080EA0D4597100000E780A0A02945D0
:1052000097D0FF1FE780E01397D0FF1FE78040048F
:105210008DBA99476303F40297B50100938505673A
:1052200017B50100130585ED97A00100E780C08D3B
:1052300017B501001305854F29B817F7FF1F03475E
:1052400037FD97F7FF1F83C7A7FC22075D8F916685
:10525000BA96C2061166C1821306F6EF8D476365E2
:10526000D60297E7FF1F938727159C4B17F6FF1F62
:105270000346F6F99386C7002DC203D6070069CA14
:105280008907E39CD7FE89471307A0F8114697F5D5
:10529000FF1F9385A5F74A8597F6FF1F2388E6F63B
:1052A00017F7FF1FA305F7F697F0FFFFE780A0B5FC
:1052B0002A84E308058C97B501009385255D17B511
:1052C00001001305A5E397A00100E780E083A28514
:1052D00017B501001305C546E5B203D60700630EF6
:1052E000E60A8907E39BF6FE8D4779BF9147630481
:1052F000F40297B501009385655917B501001305B0
:10530000E5DF97A00100E780208017B501001305B5
:10531000A5446FF00FF4B7E70400FC4F93050008B5
:1053200017E5FF1F034585618297C9B897B501004E
:105330009385C55517B50100130545DC979001000D
:10534000E780807C17B50100130585426FF06FF090
:105350002390E70017E5FF1F1305050697300100AE
:10536000E78000A797B501009385455217B5010066
:105370001305C5D897900100E780007917B50100A3
:105380001305054097900100E78000782945979024
:105390000100E780407C8147C5BD2390070017E5E9
:1053A000FF1F1305650197300100E78060A297B5E4
:1053B00001009385A54D17B50100130525D49790DD
:1053C0000100E780607417B501001305E53C5DBF7F
:1053D000411122C406C6834705002A849DC797B59C
:1053E00001009385654617B50100130525D19790F7
:1053F0000100E78060714C4017B501001305457549
:1054000097900100E7804070E1A05841B707CF00B6
:105410009387777D631DF70697B501009385C54295
:1054200017B50100130585CD97900100E780C06D89
:105430001C448356E4008355C40003C6070017B517
:1054400001001305657297900100E780E06B294524
:1054500097900100E78020700357E4009707002031
:1054600083D7A73A6309F7008355C400084497E03F
:10547000FFFFE780E0D60356E4008355C4000844EC
:105480002244B240410117F3FFFF67002355B707DD
:10549000CC009387777D6315F70497B5010093855A
:1054A000A53A17B50100130565C597900100E7807F
:1054B000A0651C448356E4008355C40003C607005E
:1054C00017B501001305456A97900100E780C06396
:1054D0002244B24029454101179301006700A367A8
:1054E000B707CE009387777D6304F70297B5010075
:1054F0009385853517B50100130545C097900100C8
:10550000E78080604C4017B501001305255BCDBDD9
:10551000B240224441018280411122C44AC006C6E1
:1055200026C29307D00D2A892E841306D00D63E37B
:10553000B7002E86B7E70400FC4742064182CA85C1
:1055400017F5FF1F130585CC829797B5010093854A
:10555000A53517B50100130565BA97900100E780DE
:10556000A05A97F5FF1F83C565CA17B5010013053B
:10557000A5DB97900100E78020592945979001000D
:10558000E780605D97F4FF1F938444C883C70400DD
:1055900041479387070693F7F70F636CF75A17B7DE
:1055A0000100130727C98A07BA979C43BA978287D5
:1055B000994763E7870297B501009385E52E17B5F4
:1055C00001001305A5B397900100E780E05317B5DC
:1055D00001001305E5D597900100E780E0528DA406
:1055E00097F7FF1F83C797C2DDCB17F7FF1F03474E
:1055F00017C297F7FF1F83C787C122075D8F97F7F1
:10560000FF1F83C7E7C0C2075D8F97F7FF1F83C7E0
:1056100037C0E207D98F17F7FF1F2327F7BC83C7CF
:10562000640097B501009385252817B5010013057F
:10563000E5AC17F7FF1F2308F7BA97900100E78042
:10564000A04C97F7FF1F938727BA8C4317F6FF1FCD
:10565000034666B917B50100130545CF97900100C1
:10566000E780804A294597900100E780C04E97F770
:10567000FF1FA38D07B82244B2409244024993070A
:1056800000F817F7FF1F2303F7B89D4517F5FF1F15
:105690001305C5B7410117430000670063239760F6
:1056A0000000E78040F397F7FF1F2382A7B69357C8
:1056B000850017F7FF1FA30CF7B4935705012A8441
:1056C00017F7FF1F2306F7B493578501014517F716
:1056D000FF1FA30FF7B297600000E78020F497F751
:1056E000FF1F2388A7B297B501009385E51B17B567
:1056F00001001305A5A097900100E780E04017F690
:10570000FF1F034606B1A28517B50100130585C525
:10571000B1B7C94763E3870297B501009385C51800
:1057200017B501001305859D97900100E780C03DE6
:1057300017B50100130585C479BD37E404007C4426
:10574000414697F5FF1F938575AC17F5FF1F1305AD
:10575000E5A9829797F7FF1F83C767AC17F7FF1F6D
:105760000347D7ABA20703238405D98F17F7FF1F81
:10577000231AF7A61306000A89452244B240924430
:10578000024917E5FF1F0345651B41010283894755
:1057900063E3870297B501009385051117B50100F2
:1057A0001305C59597900100E780003617B50100F5
:1057B000130585CC0DB517F4FF1F034444A597F7D7
:1057C000FF1F83C7B7A497B501009385E50D220499
:1057D00017B50100130585925D8C97900100E78055
:1057E000A032A28517B501001305C5BA9790010034
:1057F000E7808031294597900100E780C0350D464C
:1058000097F5FF1F938585A0228597E0FFFFE7802E
:10581000805FAA8421C197B501009385E50817B57B
:1058200001001305A58D97900100E780E02DA68566
:1058300017B50100130545B797900100E780C02C0C
:105840002244B24092440249294541011793010084
:105850006700633097F7FF1F239A8790B7E704002C
:10586000116603A38705130606E8914539B78947F2
:1058700063E3870297B501009385050317B501001F
:105880001305C58797900100E780002817B5010030
:10589000130545CD89B317F4FF1F0344449797F7C9
:1058A000FF1F83C7B79697B501009385E5FF2204D4
:1058B00017B50100130585845D8C97900100E78082
:1058C000A024A28517B50100130545AF97900100EC
:1058D000E7808023294597900100E780C0270D4687
:1058E00097F5FF1F93858592228597E0FFFFE7805C
:1058F0008051AA841DC197B501009385E5FA17A5CB
:1059000001001305A57F97900100E780E01FA685A1
:1059100017B501001305C5AB05B797F7FF1F23990E
:105920008782B7E70400116603A38705130606E81C
:105930009305000299B5894763E3870297B5010093
:10594000938585F617A501001305457B9790010007
:10595000E780801B17B50100130585C3ADB997F427
:10596000FF1F83C4C48A97F7FF1F83C7378A97B581
:105970000100938565F3A20417A5010013050578BE
:10598000DD8C97900100E7802018A68517B50100EF
:10599000130585A597900100E7800017294597908A
:1059A0000100E780401B228697F5FF1F938505863F
:1059B000268597E0FFFFE78000452A84630C051ADF
:1059C00097B50100938545EE17A5010013050573F2
:1059D00097900100E7804013A28517B501001305D9
:1059E000E5A199BD854763F78718834519002244CF
:1059F000B24092440249B335B00097E7FF1F2381BC
:105A0000B77817B501001305A5A041011793010050
:105A10006700830FA2852244B24092444A8502491E
:105A200041011703000067002324954763E38702C1
:105A300097B50100938545E717A501001305056C8F
:105A400097900100E780400C17B50100130505CEC3
:105A500059B617E4FF1F0344847B97E7FF1F83C7F2
:105A6000F77A97B50100938525E4220417A5010074
:105A70001305C5685D8C97900100E780E008A2855A
:105A800017B501001305459A97900100E780C007FC
:105A9000294597900100E780000C194697E5FF1F04
:105AA0009385C576228597E0FFFFE780C035AA84FD
:105AB0001DC197B50100938525DF17A501001305CA
:105AC000E56397900100E7802004A68517B50100E3
:105AD0001305859695B397E7FF1F23918772B7E764
:105AE0000400116603A38705130606E89305000862
:105AF00069B197B50100938525DB17A50100130552
:105B0000E55F11E897900100E780000017B50100FC
:105B10001305C593C9B497900100E780E0FE17B55F
:105B200001001305259497900100E780E0FD2945C9
:105B300097900100E78020022244B240924402493B
:105B400097E7FF1F2390076A410117630000670072
:105B5000039997B50100938525D517A50100130575
:105B6000E55997900100E78020FA17B50100130569
:105B700025C095B4B240224492440249410182803A
:105B8000411106C622C497E0FFFFE780C02721CD60
:105B900097E7FF1F83D7E75E85072A8417E7FF1F74
:105BA0002311F75E97B50100938585D197E7FF1F15
:105BB000239AA75C17A5010013054554979001008F
:105BC000E78080F4A28517B50100130525F29790B0
:105BD0000100E78060F32244B24029454101179358
:105BE0000100670043F797E7FF1F83D7C759B2400B
:105BF0002244850717E7FF1F2317F75841018280CA
:105C0000411122C491462A8417E6FF1F1306066E2F
:105C10009D652D4506C697D0FF1FE78080BCB7F76E
:105C2000070003C70701A5476313F70001A0930608
:105C3000001001469D65254597D0FF1FE78060BA9B
:105C400097E7FF1F2384876A2244B240914617E6F4
:105C5000FF1F1306A6699D652945410117D3FF1F44
:105C6000670023B81171CED7B7E9040083A7C90430
:105C7000CAD917E9FF1F13096959A2DD2E8686DFED
:105C8000A6DB2E84AA854A85829797E7FF1F83C7E4
:105C9000E7571307700A6385E710636DF700130772
:105CA000600A6385E704FE506E54DE544E59BE59B7
:105CB000116182801307800A6385E7161307900A33
:105CC000E393E7FE8D476306F41C97B501009385C7
:105CD00025F517A501001305654297900100E7809F
:105CE000A0E217B501001305E5F025A08D47630C70
:105CF000F40297B501009385A5F217A501001305DD
:105D0000E53F97900100E78020E017B501001305FB
:105D1000A5E797900100E78020DF294597900100D3
:105D2000E78060E349B7854717B50100130585E7AC
:105D300017E7FF1F2306F74497900100E780A0F4C0
:105D4000B7750200B76602000146054597D0FF1FF0
:105D5000E78020A9930760F817E7FF1F2308F74A99
:105D600097E7FF1FA385074A9307002617E7FF1F42
:105D70002320F74AE5779387072117E7FF1F231BA7
:105D8000F748B14597E7FF1F2387074897E7FF1FAD
:105D9000A383A7484A8597000000E780E01621B753
:105DA000914763E3870297B50100938565E717A5DF
:105DB00001001305A53497900100E780E0D417B5E2
:105DC0000100130525E0B1B797E4FF1F83C44444E5
:105DD00097E7FF1F83C7B743A204DD8C83A7C904DD
:105DE0006D14228697E5FF1F9385954228008297C0
:105DF0008E0493160401B7750200C1823000A69587
:105E0000094597D0FF1FE780C09D930770F817E7FB
:105E1000FF1F230DF73E994597E7FF1FA38AA73E73
:105E200095BF914763E3870297B50100938545DFEE
:105E300017A501001305852C97900100E780C0CCC1
:105E400017B50100130585D9E9B597E4FF1F83C491
:105E5000243C97E7FF1F83C7973BA204DD8C83A7F1
:105E6000C9046D14228697E5FF1F9385753A2800B3
:105E700082978E0493160401B7750200C182300028
:105E8000A6950D4597D0FF1FE780A095930780F852
:105E9000BDBF17B50100130525D797900100E78016
:105EA00080DE930790F82304F100834719008D45A5
:105EB0002800A304F100834729002305F10097007F
:105EC0000000E78060041305C01297C0FF1FE78041
:105ED0004047014597D0FFFFE780001C0D45970024
:105EE0000000E78020D2294597C0FF1FE78060456A
:105EF00097C0FF1FE780C0357DB397E7FF1F23AF33
:105F0000A73E828097E7FF1F9387473F03A30700C1
:105F1000630303000283174300006700639B411182
:105F20004AC09706002083D6468E328917D6FF1FB7
:105F30000356A64A22C426C206C62A84AE84970007
:105F40000000E780C05B35C12DC0994763FF97040F
:105F50008347140003470400A207D98F13978700D3
:105F6000A183D98FC2073167C1831307C755639EC9
:105F7000E70297D7FF1F83D74746A301F400A18309
:105F80002302F4009707002083D7278891C7A30234
:105F9000F400A1832303F400A68517B501001305BF
:105FA00025CC97900100E78020B697F7FF1F83C7A5
:105FB0006775A5C797D5FF1F83D5254217B5010083
:105FC0001305C5CB97900100E78000B42686A28513
:105FD00017D5FF1F0355654097000000E78080BA82
:105FE0006306090497F7FF1F83C7C771A1E397E70B
:105FF000FF1F83C7E7309DCB95C897E7FF1F83C777
:1060000027188DE722852244B2400249A685924492
:106010004101174300006700A38B17B5010013056A
:10602000E5C697900100E78000C65DBFB2402244FC
:1060300092440249410182808347550083454500CF
:1060400017B50100130585C0A207DD8D1793010068
:10605000670083AB17B50100130545BE1793010018
:10606000670063C28D4763FBB70A011126CA06CEDB
:1060700022CC0344350097E4FF1F83C4742897B5EE
:106080000100938565C1B337800017E7FF1FA3099F
:10609000F72609C497B501009385C5C017B501005F
:1060A0001305C5C097900100E78000A697E7FF1F82
:1060B00083C717256386970097000000E780E02CD0
:1060C00097E7FF1F83C7D7238DC785472306F100B6
:1060D000B7E7040083A747177000854513055030C4
:1060E000829717B50100130565BD97900100E78001
:1060F00080B99967938757EE2316F10068008547AA
:106100009145A30781002307F10097000000E78075
:10611000A0DFF2406244D2440561828082808947D8
:1061200063F7B708011122CC06CE26CA83442500A6
:1061300085472A84639DF404914763F5B7040345BA
:1061400045008347340022055D8D97D7FF1F2396B6
:10615000A72897000000E78060439967938767EE60
:106160002314F1008347340023059100A305F100B7
:1061700083474400954528002306F100970000005E
:10618000E78080D8F2406244D24405618280FDF805
:106190009967938767EE2314F10097D7FF1F83D782
:1061A000C723A305F10023050100A183E1B7828085
:1061B0000111996722CCD51717F4FF1F13048454DB
:1061C0002314F1008347040026CA97F4FF1F938429
:1061D000C4632305F10083D7040028009545A30577
:1061E000F100A18306CE2306F10097000000E780AE
:1061F000A0D103D604008345040017B501001305A0
:1062000065AD97900100E7802090F2406244D2444F
:10621000056182809D677971D9172316F10097F780
:10622000FF1F83C7274E06D62307F100A9C3B7E790
:106230000400FC47414697E5FF1F938525FB1305A6
:10624000F10082976800CD4597000000E780C0CB41
:1062500097F5FF1F83C5054B17B50100130585AAE8
:1062600097900100E780408AB25045618280B7E78D
:106270000400BC47414681451305F1008297D9B718
:1062800045C5411106C622C4930750FA2300F50004
:106290009307A005A300F50089472301F500914766
:1062A000A301F5009307C003A302F50097F7FF1FB2
:1062B0009387474583C70700230205002A842303E9
:1062C000F50097E7FF1F9387B70383C70700414691
:1062D00097E5FF1F938585F1A303F50097F7FF1F4F
:1062E00083D7A7522304F500A183A304F50097D711
:1062F000FF1F83D7870E2305F500A183A305F500B3
:10630000B7E70400FC47310582972285F1459700E5
:106310000000E780C01A230EA4002181A30EA40070
:10632000B240224441018280828079710A8506D67A
:1063300097000000E78000F50A86F945014597D0EF
:10634000FFFFE780403DB25045618280411122C489
:1063500026C24AC02A84AE843289AA85856601464F
:10636000254506C697C0FF1FE780A047A2852244A7
:10637000B240CA862686024992442945410117C384
:10638000FF1F670003460111B7C7A55A22CC9387A8
:10639000C73317E4FF1F1304B4F63EC48347040059
:1063A0002C002146196506CE3EC697000000E78006
:1063B00020FA8345040017B501001305A5A39780B3
:1063C0000100E7806074F24062440561828001113F
:1063D000A146300099652D4522CC06CE97C0FF1FFF
:1063E000E7802040A24737C4A55A1304C4336395FD
:1063F0008702B24517B5010013050593B335B00008
:1064000097E7FF1FA38EB7EE97800100E780C06F6C
:10641000F2406244056182809165A1463000938517
:1064200005F02D4597C0FF1FE780A03BA247E38200
:1064300087FC97E7FF1FA38507EC814517B501008F
:106440001305C590D1B77971D146700091652D457E
:1064500022D406D697C0FF1FE780A038B24737C4C2
:10646000A55A1304F43563988702B7E70400FC4784
:1064700017E5FF1F130585D741460C08829717B50E
:1064800001001305A59297800100E780C07FB250FC
:106490002254456182809165D1467000938505E85C
:1064A0002D4597C0FF1FE780C033B247E38F87FABF
:1064B00017B5010013058591F9B7C1676976814663
:1064C000FD1705061397060141836364B7003E85F7
:1064D00082803307D50003470700B98F214713F89F
:1064E0001700858363050800B18FC207C1837D173C
:1064F0001377F70F6DF78506F1B741C5A547054737
:1065000063F2B70883471500034705003168A20707
:10651000D98F13978700A183D98FC207C18313082E
:10652000C855054763900707411106C622C426C215
:1065300003442500914763F087049307540063ECFC
:10654000F502A301C50021822302C5009304340093
:1065500091C6A302D500A1822303D5002A84A68573
:1065600097000000E780A0F526942300A400218175
:10657000A300A4000147B240224492443A8541015D
:10658000828005473A8582800111B7C7A55A22CC7F
:106590009387E7342A842AC621462C00156506CE47
:1065A0003EC497000000E780A0DAA28517B501007D
:1065B0001305458697800100E7800055970000008D
:1065C000E780E0D6F2406244056182800111A14675
:1065D000300095652D4522CC06CE97C0FF1FE78081
:1065E0004020A24737C4A55A1304E43463958702B8
:1065F000B24517A501001305657797D7FF1F239EA6
:10660000B7DCC205C18197800100E780E04FF2400E
:106610006244056182809165A1463000938505EE54
:106620002D4597C0FF1FE780C01BA247E38287FC70
:10663000D14717D7FF1F2312F7DAD14517A501005D
:106640001305C574C9B721C1411126C206C622C4AB
:10665000AE848DC52A8497000000E780806697E7A6
:10666000FF1F83C7E7C999CB22852244B240A68584
:10667000924441011733000067008325B240224451
:10668000924441018280828001114AC806CE22CC08
:1066900026CA4EC693F715002E899DCBAD673717D6
:1066A00000409387A7AA1CC3B7E70400BC4F13069A
:1066B0000019854517D5FF1F034505D2829713455D
:1066C0001900F2406244D2444249B24905618280D5
:1066D00093F72500638A071C17F7FF1F0357C7129C
:1066E000954763F9E70C014417F6FF1F1306C6012F
:1066F0009306300513055004130810049308B004E2
:1067000013039005930764006374F7043A84FD59FA
:1067100097F4FF1F83C444FF97F7FF1F83C7D7FE7B
:10672000A204DD8CAD679387B755638BF41463E3E4
:10673000970AA9679387A755638EF414A28517F566
:10674000FF1F130565FC97000000E78000F031A2F1
:10675000B307860083C50700639AD50483C5170075
:106760006396A50483C527006392050583C537009A
:10677000639ED50283C54700639A150383C75700FC
:1067800063966702A2890DE897F5FF1F83D5C507B9
:10679000B3853541C20517F5FF1F1305E5F6C18125
:1067A0004E9597000000E78040EAE1A0050442040E
:1067B000418089BF3A84FD598547E3EB87F45DC486
:1067C000854517F5FF1F130525F497000000E780A6
:1067D000C0E769A8B1679387C7556380F404B567BC
:1067E0009387D755E39CF4F4A28517F5FF1F130593
:1067F000A5F197300000E780A00D8947630FF404EE
:106800009305E4FFC205C18117F5FF1F1305E5EFEE
:1068100097000000E780E04A89A097200000E78009
:10682000C0F797000000E780204911C9A28517F53D
:10683000FF1F130565ED97000000E78080480546BF
:10684000A28517F5FF1F130525EC97F0FFFFE780E2
:10685000406D97200000E78040F4A68517A5010051
:106860001305055D97800100E780002AFD57E39D31
:10687000F9F097F7FF1F239907F81345290091B501
:10688000A28517F5FF1F130525E897F0FFFFE780A6
:10689000E07AE1B7A28517F5FF1F1305E5E697F04B
:1068A000FFFFE780607B55BF93F745000145E38A12
:1068B00007E017A501001305E55897800100E78060
:1068C000803C97300000E780002F13454900D5BB7E
:1068D000411122C437E404005C5C06C6354697A526
:1068E00001009385E50617B50100130565D582976C
:1068F00011E917A501001305A55597800100E78050
:10690000803801A08327041C82972A84054597C0FC
:106910000000E780C0EB97600100E780E0709760BF
:106920000100E780E04597B00000E78040FD228548
:10693000B2402244410182804111054506C622C46D
:1069400026C297C0FFFFE780005F1305A00497B041
:10695000FF1FE780C075757585457D1597C0FFFFE2
:10696000E780A0487D7585451305F53697C0FFFF84
:10697000E7800052371400408327840A8D451305B1
:10698000002093E707202324F40A97C0FFFFE78045
:10699000C045B7E4040097D0FFFFE780E08AC858FD
:1069A00097800100E780202E17B50100130545C927
:1069B00097800100E780202D8327840C8545414581
:1069C00093E707082324F40C97C0FFFFE780404CAF
:1069D0008D451305000897C0FFFFE780604B97C007
:1069E000FFFFE780407837A507001305051297C021
:1069F000FFFFE780E073014597C0FFFFE780007A63
:106A000095450545894717F7FF1F2301F7E097C014
:106A1000FFFFE780407AB7E700E013070006238D09
:106A2000E7403707000423A0E71097D0FFFFE78077
:106A3000A00097D0FFFFE780A01297000000E7803A
:106A400060E997000000E780C09897000000E780A9
:106A500020B897E0FFFFE780A0F397000000E780F1
:106A6000802797000000E780801083A7040817059F
:106A700000001305A5C1829797D7FF1F238EA79407
:106A8000BC4C130600648545829797C0FF1FE780C2
:106A9000209601458280AD67371700409387A7AAEB
:106AA0001CC3B7E700E03707400023A0E718010048
:106AB0000100B7F7070003C70701A5476316F700F2
:106AC0009397450191C301A04111AE860146AA8565
:106AD000254506C697C0FF1FE780A0D0B240B7E7A4
:106AE00000E03707400023A0E710410182804111F8
:106AF000B2862E86AA852D4506C697C0FF1FE78061
:106B000040CEB2400145410182809307000463EC0E
:106B1000C7041D71A2CC2A840808A6CACAC886CE9A
:106B200032C697800100E780C0F2AD67371700409A
:106B30009387A7AA1CC3B7E400E03709400023A04D
:106B4000241901000100B2461008A285294597C00A
:106B5000FF1FE78000C9F640664423A02411D644F5
:106B60004649256182803955828041110D658D45E8
:106B700006C697C0FFFFE7804027B71700408D6625
:106B800023A6D70A17F5FF1F130585C81387C70A61
:106B90009387870A1CC15CC5856689675CC958C133
:106BA00014C518C9B7E70400B24003A3871E41010A
:106BB00002838145B307B5008387070089E7172360
:106BC0000000670023C48505C205C181E5B797A70A
:106BD00001009387E7411357C5003E97034707001D
:106BE000011106CE2304E100135785003D8B3E972B
:106BF0000347070023060100A304E10013574500E3
:106C00003D8B3D893E97AA970347070083C707003E
:106C100028002305E100A305F10097000000E780AC
:106C200080F9F24005618280411126C2E97797F42C
:106C3000FF1F938464CE22C49387A7552E8423819B
:106C4000B4002E86AA8517F5FF1F130525CD06C6AD
:106C50002390F400A381040097800100E78060DFA7
:106C600093052400C205C18117F5FF1F1305E5CA6E
:106C700097000000E780A084B38784002382A700E8
:106C80002181A382A700930564002244B240268597
:106C90009244C205C181410117230000670083B6F9
:106CA00009C99307800263E6B70017030000670075
:106CB000E3F7828017F5FF1F034505B7828097F73A
:106CC000FF1F83C727C589E717230000670083B329
:106CD000828097F7FF1F83C707C799EF411106C648
:106CE00097200000E780E0A9B240854717F7FF1F13
:106CF000230BF7C44101828082806307054A6385C4
:106D0000054A5D71CAC04EDE86C6A2C4A6C252DC68
:106D100056DA5AD85ED662D466D26AD0B9472A8982
:106D2000AE8963F9B706394697A501009385051A20
:106D300097800100E78080CF31ED8347E90013079A
:106D400010036394E702854717F7FF1F2304F7BC7E
:106D500017A501001305851897F7FF1F239B07BA96
:106D600097000000E78020E571A01307000317A536
:106D700001001305A519E395E7FE97F7FF1F238B85
:106D800007B897F7FF1F239607B817A5010013054B
:106D90006516F9B797F7FF1F83C7C7B76387072241
:106DA000BD6AB96B938CFA55014A17FBFF1F130B91
:106DB000EBA7138CEB65938AFA6605A8B307490124
:106DC00083C6070097F7FF1F83D7A7B4B1E39307E4
:106DD000A005639BF600854717F7FF1F231BF7B23B
:106DE00097F7FF1F2384D7A4050A93170A01C183CD
:106DF000E3E637FDB640264496440649F259625A06
:106E0000D25A425BB25B225C925C025D616182801D
:106E1000054D639BA7039307500A639EF6008947BD
:106E200017F7FF1F2317F7AE930750FA17F7FF1F47
:106E3000A30EF79E55BF9307A005E387F6FA97F7D1
:106E4000FF1F239807AC4DB7138717004207DA9747
:106E500041832380D70017F6FF1F231CE6AA8D4726
:106E6000E3F4E7F817F4FF1F0344749C97F7FF1F40
:106E700083C7E79B22045D8C9307F4FFC207C1839D
:106E80009306F00DE3EDF6FA93076400C207C183A1
:106E9000E31CF7F493052400C205C18117F5FF1F19
:106EA0001305E59897F0FFFFE780606133078B00DB
:106EB0008347570003474700A207D98F17F7FF1FE3
:106EC000231907A46318F50E8144630CA40197F4F9
:106ED000FF1F83C4E495A20497F7FF1F83C757954C
:106EE000DD8C170500001305E5DB97F0FFFFE78059
:106EF000000163878407636D9C029387EB5563826F
:106F0000F40497F7FF1F83C7A79205476389E70635
:106F100081CB1387A7051377F70F8D4663F2E60839
:106F20001307F0072300E100A300F10089459DA0AD
:106F300063829405E39754FD97F0FFFFE780C02D2F
:106F400011A8A28517F5FF1F1305858E97F0FFFF87
:106F5000E7808011014597F0FFFFE78040FA69B5AF
:106F6000A28517F5FF1F1305A58C97F0FFFFE7809B
:106F7000401BCDB797F0FFFFE780C023E1BF930729
:106F800010F8130511002300F10097F0FFFFE780D0
:106F9000602FFD450A8597000000E78020C95DBF8E
:106FA000A28517F5FF1F1305A58897F0FFFFE7805F
:106FB000A0CB4DB79307F00789450A852310F10050
:106FC00097000000E78080C605B5BD4763F8371716
:106FD000414697A501009385A5F54A859780010054
:106FE000E780C0A4631C051417A50100130585F5EF
:106FF00097000000E78020BC17F5FF1F0355E580D0
:1070000097000000E780E0BC97E7FF1F83C7876F0A
:1070100017A50100130585EA89E717A501001305E7
:1070200065EA97000000E78000B917A50100130585
:10703000E5F297000000E78000B817C5FF1F035571
:10704000653797000000E780C0B817A50100130559
:1070500025F197000000E78000B617C5FF1F035514
:10706000C53797000000E780C0B617A501001305DB
:10707000A5EF97000000E78000B417D5FF1F035568
:10708000851097000000E780C0B417A50100130524
:1070900025EE97000000E78000B217D5FF1F0355CB
:1070A000450E97000000E780C0B217A50100130548
:1070B000A5EC97000000E78000B017D5FF1F03552F
:1070C000650C97000000E780C0B017A5010013050C
:1070D000E5EA97000000E78000AE17C5FF1F0355E3
:1070E000251E97000000E780C0AE17A5010013051C
:1070F00065E997000000E78000AC97D7FF1F83C7C2
:10710000E70EA20717D5FF1F0345550E5D8D9700AB
:107110000000E78000AC97D7FF1F83C7470DA20789
:1071200017D5FF1F0345B50C5D8D97000000E78064
:1071300040AA17950100130525591DB1C14763FEEB
:107140003705414697A50100938505E44A85978058
:107150000100E780A08D31E1834709011307100387
:10716000639CE700854717E7FF1F230FF76A17A502
:1071700001001305A5E2EDB61307000317A50100F2
:107180001305C5E4E39EE7BC97E7FF1F238E07685E
:1071900017A50100130505E2E1B6CE854A8597C023
:1071A000FFFFE780E003B9B18280411126C2AE84BF
:1071B0008D4522C406C62A8497C0FFFFE78040CDD4
:1071C000B717004099C803A5C70C418D23A6A70C8B
:1071D000B240224492444101828003A5870C418D34
:1071E00023A4A70CF5B78347050003471500A207A2
:1071F000D98FC2076177C18713072720639AE700F9
:10720000834525003705040017030000670023FAB3
:10721000828017E6FF1F130666738147B286130349
:10722000F00FA9483308F6000348080013F7F70FDA
:107230006307A80C630668008507E39517FF2947D5
:10724000B387E6002380A70097E7FF1F9387C770E7
:107250005DA8411113D765001347170006C693F6C2
:107260003500058B954791CA054699476387C60047
:1072700009469D476383C600A14713F64500333690
:10728000C00093F68503050685C2A145638BB6044D
:10729000E145638AB604930580026388B6049305CA
:1072A00080036393B600914697F5FF1F238BF590FB
:1072B00097F5FF1F2386C59097F5FF1FA382D590F2
:1072C000BE8517A501001305A5D697800100E780AC
:1072D000A083B240854717F7FF1FA304F78E410133
:1072E00082808546D1B78946C1B78D4675BF17A53F
:1072F0000100130565D6178301006700E38017E7D7
:10730000FF1F13076765BA972380B700E147E302C1
:10731000F5F493077002E30CF5FC82802A87238042
:107320000500814717E5FF1F130545621308F00F9D
:107330002946B306F50083C606006396E60297E683
:10734000FF1F93866661B69783C7070005452380B4
:10735000F5009947636EF7029D4763FDE700E1473B
:10736000630DF7008280638506018507E393C7FC00
:107370000145C5B7238005008280B737004003C7A9
:10738000370083C7050093F70704D98F2380F500E2
:1073900082805D7152DC56DA5ED6716A97FBFF1F00
:1073A000938B4B938D6AA6C24EDE62D486C6A2C46E
:1073B000CAC05AD866D26AD06ECEC1495E8C97E4F4
:1073C000FF1F9384245A130A0A20938A7ADC17F940
:1073D000FF1F03492993B3872B0183C7070093F746
:1073E000F70FC9EFB787004003C76700058BE310AD
:1073F000077C03C76700118BE30D077E83C7570027
:10740000918B99E36F10200317F7FF1F0347A78F96
:1074100085476304F7006F10400197E7FF1FA382C1
:10742000E77A97E7FF1F238F075E97E7FF1F238DFC
:10743000076A97E7FF1F238B077697E7FF1F2388CD
:10744000077697E7FF1FA38F075C97E7FF1FA38DC2
:10745000076897E7FF1FA38B077497E7FF1FA388B1
:10746000077497E7FF1FA38F077497F7FF1FA38C7D
:107470000788B787004011476F007077930719009E
:1074800093F7F70F3D476364F70617F7FF1F230BCA
:10749000F78697F7FF1F9387E785CA9783C707008B
:1074A0001307100293F7F703638EE71E6366F70472
:1074B00005446385871CE38C07620947638EE710E8
:1074C00013070002E384E74EB7E700E03707400008
:1074D00023A0E71801000100629923000900FD19AB
:1074E00023A0E71093F9F90FE39309EEE5BD97F7B1
:1074F000FF1F2389078071BF130730026388E70CE1
:1075000063E8E71613074002638CE70A13070003DA
:10751000E39CE7FA97E7FF1F9387C77CCA9703C7E7
:107520000700A1471377F70FE31BF71483C7640025
:1075300097E6FF1F238EF66697E7FF1F83C7F74284
:1075400091C7FD5797E6FF1F2384F66697E5FF1F57
:1075500083C5554197E7FF1FA38CB76497E7FF1FCB
:1075600083C7474013FB07089306000493F70706F9
:10757000639FD74C9307A009638DF51663EAB71292
:107580009307F0056386F54A930750096384F52A4B
:10759000014497E7FF1F83C7B7611547E392E736BA
:1075A000B7E700E03707400023A0E718010001001B
:1075B000B786004023808602130680FC6F00500EC1
:1075C000FD5717E7FF1F2304F75EFDBDFD5717E7C3
:1075D000FF1F230DF75CCDBD17A50100130545B9AD
:1075E00097700100E780206A97E7FF1F9387876FF6
:1075F000CA9703C40700014B97ECFF1F938C0C4FF5
:107600001374F40F17AD0100130D0DB763478B040E
:10761000294597700100E7800054854717E7FF1F51
:10762000A304F74C17E7FF1F2301874C17E7FF1F41
:10763000230AF75837E700E0B70640002320D718A1
:1076400001000100378600408347A60293F7370FF9
:107650002305F6022320D71085BDB3876C0183C5AF
:1076600007006A85050B97700100E780E04979BF44
:10767000854717E7FF1F2309F746B9B517E7FF1F2F
:10768000130747664A970347070097E6FF1FA38B38
:10769000F63897E6FF1F2388E63817E7FF1F230316
:1076A000F7521DB5854717E7FF1F230DF73629BD94
:1076B0009307400A6389F5349307200B6384F536FA
:1076C0009307100AE396F5EC838724000144E3D284
:1076D00007EC97E7FF1F83C7172993F63700638AE4
:1076E000061A0546638AC62209466395C61A1D47CF
:1076F00055A217E5FF1F03450527C94797ECFF1F54
:1077000083CC7C2697E5FF1F83C5052617E4FF1F62
:10771000034494256315F510CD476392FC1093073D
:107720007008639CF5021307300FB7170E0063084B
:10773000E4001307900DB7B704006314E40817E7DB
:10774000FF1F232DF746BE8517A50100130545A38E
:1077500097700100E780403B25BD93078008639D3B
:10776000F500B307804013F4F70FB777460093870F
:1077700087CDB3D78702E1B793079008639AF500E6
:10778000B307804013F4F70F91679387C766D5B7A7
:107790009307A008639BF500B307804013F4F70F2D
:1077A000B7173D0093870790E9B79307B008639A2E
:1077B000F500B307804013F4F70F9167938797D0D4
:1077C0004DBF93F5F5078D47639BF500B3078040E8
:1077D00013F4F70FB7975B00938707D859BF894712
:1077E000639BF500B307804013F4F70FB7770B00E6
:1077F0009387071BBDBF8547639AF500B307804099
:1078000013F4F70FDD67938767E3A5B7D28785F990
:10781000B307804093F7F70FB3D7FA020DB797007D
:107820000000E780409FA285668597000000E78002
:10783000809EB9BB9305610017E5FF1F0345A512A4
:1078400017E4FF1F0344341297000000E78040ADA7
:1078500093057100228597000000E78060AC3C0032
:1078600017E7FF1F2326F746834761002304F10033
:1078700083477100A304F100894717E7FF1F23091D
:10788000F7328357810017E7FF1F231DF70C0944C8
:1078900009B3154793F64700B336D00093F7870333
:1078A000850685C32146638BC7066146638AC70682
:1078B000130680026388C706130680036393C7001C
:1078C000914717E6FF1F230DD62E97E6FF1FA389CA
:1078D000F62E97E7FF1F2386E72E17E7FF1F0347C4
:1078E000A7089376070497E7FF1F83C7F7078DEE76
:1078F0001377770C93067008630CD7021377F7079A
:107900008D466312D70CB307F040B7955B0093F731
:10791000F70F938505D849A81947ADBF854755B7D7
:10792000894745B78D4771BF930670086311D70229
:107930001307300FB7150E006389E7021307900D88
:10794000B7B504006383E7021307700845BF9306C9
:10795000800C6311D702B307F040B775460013F7E8
:10796000F70F938785CDB3D5E70297E7FF1F23A7CE
:10797000B724D9BB9306900C631CD700B307F04023
:1079800093F5F70F91679387C766B3D5B702F1BF39
:107990009306A00C631DD700B307F040B7153D0058
:1079A00093F7F70F93850590B3D5F5027DBF930646
:1079B000B00CE315D7F4B307F04093F5F70F9167D8
:1079C000938797D0D9B78946631BD700B307F04098
:1079D000B7750B0093F7F70F9385051BF1B7854635
:1079E000631AD700B307F040DD6593F7F70F93856F
:1079F00065E35DBFD28535FBB305F04093F5F50F28
:107A0000B3D5BA029DB783C72400C18B99C78547F8
:107A100017E7FF1F2301F71AA5BE97E7FF1F238C67
:107A20000718BDB6854717E7FF1FA30CF7188DB6DB
:107A30003C0017E7FF1F232DF72809479307000392
:107A40002314F10097E6FF1F2384E6162DBD6394EF
:107A50000756A94763E5B742179701001307875AEE
:107A60008A05BA959C41BA97828717E4FF1F0344A1
:107A700094EF894C6306940D63E68C068547630397
:107A8000F4089307F00F17E7FF1F0347671263F629
:107A9000E70017E7FF1F230DF71097ECFF1F83CCBC
:107AA0002C119307000413F4FC0F63F497011304E3
:107AB000000497E7FF1F9387A72103AD07002286E5
:107AC0002685EA85B38C8C40229D97700100E78063
:107AD00040F897E7FF1F238D970D97E7FF1F23A916
:107AE000A71F45BC8D47630CF40A9947E31BF4F8C4
:107AF000979701009387875717E7FF1F232AF71CE3
:107B0000A94751B717E7FF1F0347E71F97E7FF1F75
:107B10009387070C4946979501009385255E630678
:107B2000870097950100938565593E859770010000
:107B3000E78020F217E7FF1F232CA718C947A1B73A
:107B400097E6FF1F83C6261C054797E7FF1F93870D
:107B500027086394E6023E8513067002979501009C
:107B60009385455797700100E780A0EE17E7FF1F48
:107B70002320A7169307700239B73E8513063004F9
:107B8000979501009385454F97700100E78060EC61
:107B900017E7FF1F232EA71293073004EDB597E5D3
:107BA000FF1F83C545DC179501001305A55E97707F
:107BB0000100E78060F5054D97EDFF1F83CDAD1403
:107BC00097E5FF1F83C525DA179501001305855C2E
:107BD0006398AD0B97700100E78000F397E7FF1FF4
:107BE00083C767D8B5CBE36EF4E81794010013049C
:107BF0002455638CB701179401001304E454638681
:107C00009701179401001304A45522859770010071
:107C1000E780A0081375F50F93071500860717E78F
:107C2000FF1F2307F7FA8D4717E7FF1FA302F7FA95
:107C300097E7FF1F9387C7F90147BE861376F70FB3
:107C400089076365A60297E7FF1F23A3D70897E775
:107C5000FF1F83C7E7F705BD979701009387474745
:107C600017E7FF1F2326F706914731BD3306E400CF
:107C700003460600A380070005072380C7007DBFD9
:107C800097700100E78040E897E7FF1F83C7A7CD03
:107C9000E1D7E368F4DE1794010013046447638CB2
:107CA000A7011794010013042447638697011794D2
:107CB00001001304E447228597700100E780E0FD8E
:107CC0001375F50F93071500860717E7FF1F2301AC
:107CD000F7F08D4717E7FF1FA30CF7EE97E7FF1F9D
:107CE000938707EF0147BE861376F70F8907E37C7A
:107CF000A6F43306E40003460600A3800700050748
:107D00002380C700D5B797E5FF1F83C5C5C5179565
:107D100001001305E54897700100E780E0DE97E772
:107D2000FF1F83C7B7EA93E7470017E7FF1FA30FBB
:107D3000F7E883C7240017E7FF1FA307F7E889B810
:107D4000179501001305054797700100E780A0F320
:107D500097E7FF1F938747E783C7070017E7FF1FD2
:107D60002302F7C017E4FF1F034484E43334800088
:107D70000DB0179501001305254597700100E780A8
:107D800080F097E7FF1F83C777E493E7070117E7C2
:107D9000FF1FA30DF7E283C7240017E7FF1F23058A
:107DA000F7E26FF0EFFE179501001305254397707A
:107DB0000100E78040ED03C704007D8B51EFB787DA
:107DC000004003C767021377C70B1367270023839D
:107DD000E70203C7A7021377C70B136727002385A2
:107DE000E70203C7E7021377C70B13672700238750
:107DF000E70203C727031377C70B136727002389FD
:107E0000E702854717E7FF1F230EF7C017E7FF1F9D
:107E1000230CF7CC17E7FF1F230AF7D817E7FF1F3C
:107E20002307F7D897E7FF1FA38E07BE97E7FF1F2B
:107E3000A38C07CA97E7FF1FA38A07D697E7FF1F00
:107E4000A38707D697E7FF1FA38E07D697E7FF1FE5
:107E5000A38B07EA6FF0CFF389476312F70297E726
:107E6000FF1F83C767B09146638CD70863E0F604B1
:107E7000638EE70C6369F70A05476380E70EFD57D9
:107E800017E7FF1FA306F7D237074000B7E700E068
:107E900023A0E71801000100B78600401306F0FC9C
:107EA0002381C60223A0E7106FF00FE2130720081A
:107EB0006382E7086362F70213071008E391E7FCA7
:107EC000378700408347670293F7C70B93E7270084
:107ED0002303F7026FF0CFEB130730086389E70243
:107EE00013074008E39DE7F83787004083472703DF
:107EF00093F7C70B93E727002309F7026FF04FE9C9
:107F0000378700408347270393F73707F5B737874D
:107F100000408347E70293F7C70B93E72700230747
:107F2000F7026FF0EFE6378700408347E70293F7E9
:107F30003707F5B7378700408347A70293F7C70B8A
:107F400093E727002305F7026FF08FE4378700409F
:107F50008347A70293F73707F5B737870040834772
:107F6000670293F73707ADB717950100130505288A
:107F700097700100E78020D197E7FF1F2384079EB9
:107F8000D5B3179501001305652797700100E780A9
:107F900080CF97E7FF1F2397079C97E7FF1F9387E3
:107FA00027C103C40700894763F38700094413749A
:107FB000F40F6FF00FDE13070002E392E7EC631B90
:107FC0000B0A638FF500930720026383F50817956A
:107FD00001001305252697700100E780E0B245B542
:107FE000179501001305452297700100E780A0C98D
:107FF0000144179D0100130D6D22A14CB38784002D
:1080000083C507006A85050497700100E780C0AF4B
:10801000E31694FF178501001305057197700100A1
:10802000E78060C617E4FF1F0344049401E897E764
:10803000FF1F238B0790014B6FF0AFD58947E310EB
:10804000F4E4854717E7FF1F2300F7906FF04FD444
:1080500017E6FF1F0346369197E5FF1F83C5A590DE
:10806000179501001305051C97700100E780C0A952
:108070006FF00FD26380F50693071002E399F5F4D1
:1080800097E5FF1F83C5458E179501001305851BD6
:1080900097700100E78040A797E7FF1F23AA97C2C8
:1080A00097E7FF1F938787B1944383D7470017E76C
:1080B000FF1F034707B117E6FF1F2325D68A1D447C
:1080C00097E6FF1F2392F68A97E7FF1F238FE78823
:1080D0006FF02FCC97E5FF1F83C505891795010029
:1080E0001305C51797700100E78000A297E7FF1FEF
:1080F000238C078497E7FF1F239607866FF02FF9DD
:108100002547638FE7C89946378700406394D702B5
:1081100023008702B7E700E0B706400023A0D71886
:1081200001000100130600FC2301C70223A0D710A1
:108130006FF08FB99306100A639FD7002300870260
:10814000B7E700E0B706400023A0D7180100010000
:10815000130680FCD1BF9306A009E381D7FE9306E6
:10816000400AE38DD7FC93062002639DD700B7E752
:1081700000E0B706400023A0D7180100010023004B
:108180008702F9B78546E384D7FE93070008E3002A
:10819000FBFEB7E700E0B706400023A0D7180100B8
:1081A0000100130620FC23008702BDBF17E7FF1F55
:1081B000034717A06302F71E63E7E70295476300D2
:1081C000F7109947630AF704B78600402380060238
:1081D000B7E700E03707400023A0E71801000100DF
:1081E0001306A0FC75B99307F005630AF70093071F
:1081F00050096306F70093071002E317F7FCB7E78F
:1082000000E03707400023A0E71801000100B7860F
:108210000040130620FC69B117EBFF1F034B4B997D
:10822000930700045A8D63F46701130D000497E768
:10823000FF1F9387E7A983AC07001374FD0F228605
:10824000E685268597700100E780A080B3078B4004
:10825000669417E7FF1F230DF79497E7FF1F23A9E5
:1082600087A6B7870040630C0B022380A703B7E6FD
:1082700000E03706400023A0C6180100010003C734
:108280002702134707042381E70203C72702137756
:10829000C70F2381E70223A0C6106FF0EFA223804F
:1082A000070237E700E0B70640002320D718010097
:1082B0000100130620FC2381C7026FF0AFB9378796
:1082C00000408347370097E6FF1F83C6F68F93F77A
:1082D0000708D58FA301F700B7064000B7E700E015
:1082E00023A0D718010001001306A0FC35BD97E7B5
:1082F000FF1F9387279FCA9783C7070093F7F70F3E
:10830000C1CF97E7FF1F83C707A0D9E717E7FF1F74
:108310000347178A930700026310F70883AD040030
:1083200017DDFF1F034D4D6497DCFF1F83CCDC631B
:1083300017DBFF1F034B6B63E6876A87DA866E865F
:1083400097D5FF1F83C5456017950100130585F27A
:1083500097600100E780407B97E7FF1F23A0B78766
:1083600097E7FF1F238EA78597E7FF1FA38A9785AF
:1083700097E7FF1F2387678597D7FF1FA385875C34
:10838000B7E700E03707400023A0E718010001002D
:10839000B78600406FF04FA2B7E700E03707400014
:1083A00023A0E71801000100B786004015BD97E63D
:1083B000FF1F83C646950547639CE6042947238132
:1083C000E70209472383E7022385E70297D7FF1FC8
:1083D000A38A077E97E7FF1FA3870792B78700400E
:1083E000A381070017D7FF1FA300077E054723833C
:1083F000E700B640264496440649F259625AD25ADA
:10840000425BB25B225C925C025DF24D61618280F4
:1084100029472381E70209472383E7022385E702EF
:108420002387E7022389E70255B717D7FF1FA30C5D
:10843000F7506FE01FFF854717D7FF1F2304F75E34
:1084400017D7FF1F2302F76A17D7FF1F2300F776FE
:1084500017D7FF1F230DF7746FE0BFFE854717D7AF
:10846000FF1F2301F75C17D7FF1F230FF76617D7EE
:10847000FF1F230DF77217D7FF1F230AF77217D7B5
:10848000FF1FA301075A17D7FF1FA30F076417D7B2
:10849000FF1FA30D077097D7FF1FA38A0770828065
:1084A000411106C697000000E78080FBB7870040B7
:1084B00023800700130740FC2386E7001307C0044E
:1084C000A386E70017D7FF1F1307C7492398E700C4
:1084D00017D7FF1F1307074D239AE70017D7FF1F72
:1084E00013078758239CE70017D7FF1F130707645C
:1084F000239EE70029472381E70209472383E702F8
:108500002385E7022387E7022389E702A381070087
:10851000930600F8A380D700930690022380D7002B
:10852000FD562383D7002381E7009306000537E734
:1085300000E0230BD740B70640002320D71003C725
:10854000170013671700A380E700B24097D7FF1FFB
:10855000239C076641018280411106C697000000F6
:10856000E78000F0B787004023800700130700FC76
:108570002386E7003147A386E70017D7FF1F1307BD
:10858000673E2398E70017D7FF1F1307A741239AD9
:10859000E70017D7FF1F1307274D239CE700294744
:1085A0002381E70209472383E7022385E702A381AA
:1085B0000700930600F8A380D7009306900223805B
:1085C000D700FD562383D7002381E70093060005DB
:1085D00037E700E0230BD740B70640002320D71031
:1085E00003C7170013671700A380E700B24097D7AF
:1085F000FF1F239B075C41018280F167938707205F
:1086000017D7FF1F232CF75A854717D7FF1F2319AA
:10861000F75AA14717D7FF1F2305F75A97D7FF1F10
:10862000A381075A97D7FF1F238E075897D7FF1F9D
:10863000238C073097D7FF1FA3870730814717D5B3
:10864000FF1F1305A530FD5517D6FF1F1306C630B3
:108650002947B306F5002380B600B306F600238051
:1086600006008507E397E7FE97D7FF1FA38307540C
:1086700097D7FF1FA381075497D7FF1F238C07525B
:1086800097D7FF1F2387075297D7FF1F23860752CD
:1086900097D7FF1FA380075297D7FF1F238D07503F
:1086A000814717D6FF1F1306E6624147B306F6005F
:1086B000238006008507E39BE7FE828017D7FF1F14
:1086C0000347676485476316F700170300006700D8
:1086D000E3E8170300006700E3DC411122C406C68B
:1086E00017D7FF1F0347276285472E8613F4F50F20
:1086F000AA856317F70417D5FF1F1305E53A97609E
:108700000100E780003597D7FF1F238F073CB7870D
:10871000004023848702B7E600E03706400023A02C
:10872000C6180100010003C7A7021377C70F2385EE
:10873000E702B240224423A0C610014541018280D5
:1087400017D5FF1F1305052A97600100E7806030E9
:1087500097D7FF1F2388072CB78700402382870203
:10876000B7E600E03706400023A0C618010001006C
:1087700003C767021377C70F2383E7025DBF411169
:1087800006C697000000E78080E7B240410117036A
:1087900000006700E3F2411106C697F0FFFFE78093
:1087A00080BF97D7FF1F83C7F727A1CB97D5FF1FA0
:1087B00083C5652789C917D5FF1F1305E52697E0EF
:1087C000FFFFE780C05397D7FF1FA38D072497D7DC
:1087D000FF1F2389073E37E700E0B706400023204C
:1087E000D71801000100378600408347660293F7DF
:1087F000370F2303F6022320D710B24041018280B5
:1088000041C9D9C597D7FF1F83C7073CD1C3011101
:1088100022CC4AC84EC656C25AC006CE26CA52C438
:108820002E89AA890144930A0004371B0300637749
:108830002403B3078940C207C183BE8463F4FA00EE
:1088400093040004C204C180130A1BD497D7FF1FEE
:1088500083C7471D9DE37D1A631C0A00F2406244F2
:10886000D2444249B249224A924A024B056182806F
:1088700097F0FFFFE78020B2D1BF338589002694AF
:10888000A685420497000000E78060E5418045B777
:10889000828097D7FF1F9387A74A18429C4383D6AD
:1088A00045000345070083C5C7000356460063968D
:1088B000A50083D5E700638DD502011106CE23867E
:1088C000A7002397D700B705CF00DC4B9385757DB4
:1088D00005077D162EC2230001003AC42316C100ED
:1088E0002317D10099C30A858297F24005618280DF
:1088F0008280DC4DDC4B81CFB7E70400904503A3B9
:108900008705914517D5FF1F0345C5430283828024
:108910006D713C083EC6B707E500232291103EC8A2
:10892000AA843C083285232611103ECA23248110D4
:10893000232021112E8997300000E78040672A8488
:108940009795010093858596177501001305057BA2
:1089500097600100E780401BA28517950100130571
:1089600065A597600100E780201A294597600100FE
:10897000E780601EB705CB009385757D6800971072
:108980000000E780C06CA285680097300000E78097
:108990006054014781467000CA85268597200000F3
:1089A000E780409005CD2A84979501009385059036
:1089B000177501001305857497600100E780C014E6
:1089C000A285179501001305A59F97600100E78018
:1089D000A013294597600100E780E0178320C110AC
:1089E00003248110832441100329011051618280E6
:1089F00097D7FF1F9387C73418429C43797122D4BD
:108A000006D60348070083C807012A8483D6450099
:108A1000035546006396080183D82701638DD80269
:108A20002388070105072399D7003708CC00DC4BC2
:108A30001308787D3ACC1307F5FF42CA23080100DA
:108A4000231EE100231FD10099C7080832C62EC497
:108A500082973246A245228597000000E78080EB8E
:108A6000B2502254456182806D713C083EC0B70708
:108A7000E5003EC23C083EC4232611102324811089
:108A8000232291102317010023180100231901004C
:108A9000231A0100231B010097B7FF1F83D74796B6
:108AA00099E3C167FD172316F10097B7FF1F83D71E
:108AB000479591EB97D7FF1F938787289C439C434B
:108AC000DC4783D7070017B4FF1F13046493584C87
:108AD0002317F10083574400484B2318F10031E17C
:108AE000979501009385858317750100130505612E
:108AF00097600100E7804001179501001305458349
:108B000097600100E7804000294597600100E780F9
:108B100080048320C11003248110832441105161FB
:108B2000828097B7FF1F83C7178E89EBB7E70400D2
:108B3000BC5782975C4C23AA0700E1BFFD1797B68C
:108B4000FF1FA382F68C03560701834704014C479D
:108B50000A85230BF10097300000E780C03497D7D7
:108B6000FF1F9387E71D9C430147814688430A8680
:108B70006C0097100000E780E072AA8429C19785F5
:108B800001009385A5791775010013052557976096
:108B90000100E78060F7A685178501001305057AB7
:108BA00097600100E78040F6294597600100E78063
:108BB00080FA584CB7E70400BC57484B9DBF97B7A5
:108BC000FF1F83C75784F5D7B7E70400BC4F104495
:108BD000854517D5FF1F0345E51682971DBF5C4EDF
:108BE000DC4BB9CFB1CD411122C41775010013057B
:108BF000E5502E84978501009385857006C69760A1
:108C00000100E78060F0A285178501001305C57596
:108C100097600100E78040EF294597600100E780F9
:108C200080F3B7E704002244B24003A3870517D5B9
:108C3000FF1F03452511130640069145410102839C
:108C40008280411122C417A4FF1F130424791C4CF5
:108C500006C689C7DC4399C34C488297584CB7E78E
:108C60000400BC57484B82975C4CB240224423AA74
:108C700007004101828017A7FF1F1307277883474A
:108C800007009306F00B850793F7F70F63E9F600EB
:108C900097A6FF1F2384F67603450700828093077B
:108CA00000F8FDB7835745006386071001114AC8D5
:108CB00017A9FF1F1309C97452C4032AC90106CE9C
:108CC00022CC03274A0126CA4EC656C2F15735E3C5
:108CD0001307D00DFD57636EC704B7E9040083A7DF
:108CE00009072A841305860042054181B284AE8AB1
:108CF0008297232AAA000325C9015C49A9E7978521
:108D000001009385E55D177501001305253F976008
:108D10000100E78060DF178501001305256D97606E
:108D20000100E78060DE294597600100E780A0E24E
:108D3000DD57F2406244D2444249B249224A924A43
:108D40003E850561828093874400B705CF002319D3
:108D5000F5009385757D310597100000E780202F81
:108D60000325C90183456400310597300000E78081
:108D700060160325C9012686D68531059730000087
:108D8000E78060127146A2854A8597600100E780FE
:108D900040CC504419CA83A78905854517D5FF1FC4
:108DA000034545FA8297814769B797000000E7803D
:108DB000E0CBD5BFFD573E858280411126C297A4E6
:108DC000FF1F9384E463D84C22C437E404003C546E
:108DD000484B06C68297DC4C0323C4052244B240AC
:108DE000924423AA070017D5FF1F0345A5F5854523
:108DF00041010283411126C297D4FF1F938444F49A
:108E00009C4006C622C44AC0D5C3DC43C5C35CC16E
:108E10002300B5002A84978501009385A54717751F
:108E200001001305A52D97600100E780E0CD2945DD
:108E300097600100E78020D29C4023A4070023A272
:108E4000070097A7FF1F93876759DC4FDC4B91C73B
:108E5000295597000000E78000DF97A7FF1F938741
:108E6000275ADC4FDC4B89C797000000E78020F5CC
:108E700037E904008327C905894517D5FF1F034536
:108E800065EC82978327C905914517D5FF1F0345D8
:108E900065EB82979C4003A3470163090300228589
:108EA0002244B2409244024941010283B24022442A
:108EB00092440249410182800111328506CE22CCC2
:108EC00026CA2E8497300000E780600EAA8497851A
:108ED00001009385653F17750100130525229760F2
:108EE0000100E78060C203078400035664008355D5
:108EF0004400A68617850100130505499760010007
:108F0000E78080C0294597600100E780C0C497A72B
:108F1000FF1F83C7074D639D970001459700000021
:108F2000E78060D281450A8597000000E780C0ECA9
:108F3000F2406244D244056182806D712324811025
:108F4000232611102322911093F745002E84638766
:108F500007143C083EC0B707E5003EC23C083EC4CB
:108F6000231701002318010023190100231A01000F
:108F7000231B010097A7FF1F83D7474699E3C167CB
:108F8000FD172316F10097A7FF1F83D7474591EBE5
:108F900097D7FF1F9387C7DA9C439C43DC4783D74F
:108FA000070017A7FF1F130767432317F100544F4C
:108FB000835747002318F100DC4AA1E79785010099
:108FC0009385C5341775010013054513976001009B
:108FD000E78080B317850100130585359760010090
:108FE000E78080B2294597600100E780C0B613454D
:108FF00044008320C1100324811083244110516157
:10900000828097A7FF1F83C7D73D2555D9C3FD177A
:1090100017A6FF1FA307F63C03D6060183470701E7
:10902000CC460A85230BF10097300000E780A0E7CB
:1090300097D7FF1F9387C7D09C4317A7FF1F13071E
:10904000E739978601009386A63188430A866C002B
:1090500097100000E7800025AA8451D99785010068
:109060009385C52A1775010013054509976001000E
:10907000E78080A9A685178501001305252C976038
:109080000100E78060A8294597600100E780A0AC57
:10909000268597000000E78000BB91BF93F725006D
:1090A0009DC7B7E70400BC47414681452808829721
:1090B000255597000000E78000B928089305F00FB8
:1090C00097000000E78040D3134524001DB793F7B5
:1090D0001500014599DF97000000E78020991345AE
:1090E000140001BF5C4D411106C688C317D7FF1F8E
:1090F0002328F7C4B7E7040083A707081705000073
:109100001305E5E38297B24097D7FF1F238CA7C2D0
:1091100001454101828001113335A000A307A10060
:10912000B7E7040083A7471706CE1306F10085456D
:10913000130550308297F240056182808280411190
:1091400022C406C697D7FF1F83C747C1014489EFD2
:1091500097B7FF1F83C7D71A054499E717B4FF1FB6
:109160000344041A13441400228597000000E7808A
:10917000C0FA178501001305653209E4178501005F
:109180001305C5322244B240410117630100670054
:10919000A397797122D426D206D64AD04ECEA30701
:1091A000010097B7FF1F83C7A715AE84328489CB10
:1091B000B7E7040083A747172E86A285829735A8B4
:1091C00037E9040083278917AA899305F10013055D
:1091D000503082978347F10085CB0145970000000E
:1091E000E780A0F3832749172686A2854E858297BC
:1091F000054597000000E78040F2B2502254925497
:109200000259F24945618280832749172686A28543
:109210004E856DB741119397050122C406C626C23B
:10922000C1872E8463D40702B7E40400FC5417A559
:10923000FF1F0345E51F829719C1BC548297216522
:10924000218DB240224492444101828093F715005F
:109250008DC7B7E7040083A7471A17A6FF1F130699
:10926000261C97D5FF1F9385A5AE17A5FF1F0345A5
:10927000251C829713451400E9B793F7250099CF71
:10928000B7E70400BC4F13060064894517A5FF1F0C
:109290000345051A82971345240065B793F78500A7
:1092A00085CF97D7FF1F83C727AC85E7B7E70400B3
:1092B00003A8871A1307401F97A7FF1F83C74717E5
:1092C000814613064006994517D5FF1F035545A94A
:1092D000029813458400B5B793F745000145B5D30F
:1092E000B7E4040083A7041817D5FF1F035545A74B
:1092F0008297BC4C13060064914517A5FF1F0345D8
:1093000025138297134544002DBF97D7FF1F83D79E
:1093100027A56398A70217D7FF1F2314B7A417D751
:10932000FF1F2311C7A417D7FF1F231ED7A22E8606
:10933000178501001305051EBE8517530100670040
:10934000A37C178501001305651E176301006700E4
:1093500083930357450097D7FF1F83D767A0631CEC
:10936000F706C167F917411117D7FF1F232AF79E88
:1093700022C497D7FF1F23A7079E97D7FF1FA38F4E
:10938000079C97D7FF1F2381079E37E404007C4C7E
:1093900006C6894517A5FF1F0345850982977C4CA2
:1093A000914517A5FF1F0345A508829797C7FF1F83
:1093B00083C7473591CB854717A7FF1FA301F70840
:1093C00097A7FF1F238E07062244B24041011703CF
:1093D0000000670003D717850100130525151763E3
:1093E00001006700438A7D15954763E2A71C178734
:1093F0000100130727090A053A951C41011122CCE7
:1094000006CEBA972E848287178501001305851230
:1094100097600100E7802087A1A203C72500994734
:109420006311F7022E8597000000E780C0F28345A4
:109430006400178501001305E51097500100E780CF
:10944000A06C97B7FF1F238D07EA1785010013054E
:1094500025117DBF03C7250095476319F702C16732
:1094600017D7FF1F0357C78FF91703D5A500630947
:10947000F702B7E7040083A7C71782971785010093
:109480001305050F97500100E780E07F854717B768
:10949000FF1F2307F7E6178501001305E50F8DBFB2
:1094A00097D7FF1F239EA78A83D7E50097D6FF1F74
:1094B0002399F68A83D7050197D6FF1F2394F68A4E
:1094C00083D7250197D6FF1F239FF68897D7FF1FC5
:1094D000A3860788631BE502B7E70400BC4F096653
:1094E00013060690A14517A5FF1F034565F4829753
:1094F0000356E4008355A400178501001305850871
:1095000097500100E780406051B79307700F231612
:10951000F100B7E7040083A7870D17A6FF1F0346D6
:1095200026F16C0082974DF9854717D7FF1FA307D7
:10953000F7825DB7178501001305C506D1BD83C548
:10954000250091476392F502178501001305050771
:1095500097500100E780207397000000E78060BE0D
:10956000F24062440561828099476392F502228548
:1095700097000000E78020DE834564001785010026
:10958000130545FC97500100E7800058D1BF95476F
:10959000639AF50083471400E1F317850100130572
:1095A0002504BDB51785010013050504E1BF8280C0
:1095B0003757315F97A7FF1F9387C7E8130777D502
:1095C00098C39356C50017870100130767F1BA9631
:1095D00083C5060093568500BD8ABA9603C6060069
:1095E00093564500BD8A3D89BA962A9783C60600E0
:1095F00003470700238407002383D700A383E700E2
:109600002382B700A382C70097A7FF1F938787E431
:109610002383B700A383C7002384D700A384E70074
:109620008280411106C697000000E780A0F8B7E7E6
:10963000040083A7871417A6FF1F1306A6E0D545CD
:1096400001458297B2404D4697A5FF1F938585E05F
:10965000130570304101170300006700C3B3617147
:109660002324811A37E40400832704082326111ACF
:109670002322911A2320211B232E311917050000C4
:10968000130585B9829717A9FF1F130969DA99474E
:1096900085442300A900231CF100978501009385D0
:1096A00025E39307400617750100130525A5231C24
:1096B000F1082308910097C9FF1F93890915975056
:1096C0000100E780604483D5090017850100130578
:1096D00025DF97500100E78020432945975001007E
:1096E000E780604703D50900896997000000E7809B
:1096F00060EC832744171008854513055030829786
:109700008327441717A6FF1F1306C6D4CD4513059C
:10971000703082978327441717A6FF1F130686D140
:10972000B545130560308297832744173008894573
:109730001305103182978327441730098945130593
:109740002031829783274415938509900D45829790
:10975000832744159385099011458297A3059100AD
:109760002306910002CD23080100230C010083276A
:10977000841630099145130570408297832784161B
:109780001306B10085451305004082978327841690
:109790007000854513051040829783278416300892
:1097A0008545130520408297832784161008854538
:1097B000130550408297832704157D558297832790
:1097C00044137D5582977D5597A0FFFFE78080ED7C
:1097D0008327440C829797A0FFFFE78040C7832729
:1097E000841417A6FF1F1306E6C5D54501458297C9
:1097F00089471306700F814528092306F1009790C9
:10980000FFFFE780C0908D471306000881452808B8
:10981000230CF1089790FFFFE780608F9147230C9E
:10982000F100976701009387E77E984383C747005D
:109830003AC8230AF10097D0FFFFE78040AF7000DD
:109840008545054597A0FFFFE780E0EC30099305CB
:10985000700F094597A0FFFFE780E0EB3008930504
:1098600000080D4597A0FFFFE780E0EA1008954546
:10987000114597A0FFFFE78000EAC16717C7FF1FE8
:109880001307074EF9171CC32322070017A5FF1F54
:109890001305C5B997A0FFFFE780C0E68327C41D65
:1098A00017C5FF1F1305454A82973C480345090029
:1098B000854582978320C11A0324811A8324411A83
:1098C0000329011A8329C1195D618280C16717C804
:1098D000FF1F0358E848F9176301F8083DCDB5CDDF
:1098E000011126CAB7E4040083A7841222CC2E8675
:1098F0002315B10006CE2A8401478146ED454285F5
:1099000082972AC611ED178501001305A5BE975051
:109910000100E7804037F2406244D2440561828012
:10992000FC440356A100A28582972C0017C5FF1F97
:109930000355054397A0FFFFE780C0EC69DD17855D
:109940000100130565BC97500100E780C03383A771
:10995000C412ED45280082977DBF828015C98547D6
:1099600017A7FF1FA30DF7AC97A7FF1F238A07AC0C
:1099700097B7FF1F83C7C7988DE3354697A5FF1F8D
:10998000938545AB13056030170300006700A38083
:1099900097A7FF1FA38507AAC1BF828097C7FF1F94
:1099A00083C7873CA9EFC16717C7FF1F0357473B12
:1099B000F9176306F7044111854722C417C7FF1F33
:1099C0002304F73A37E404007C4C06C6A14517A5EA
:1099D000FF1F0345E5A582970323841A2244B24062
:1099E00097A7FF1F83C7C7A417C5FF1F0355453798
:1099F0001307401F81463146994541010283828009
:109A00006D7123248110232611102322911032849A
:109A100001CD8947630AF5028320C1100324811018
:109A2000832441105161828017850100130585BC94
:109A3000AE8497500100E7800025A285268597C057
:109A4000FFFFE780A0ADC9BFB7E70400FC472800CF
:109A50008297178501001305A5BA97500100E7808A
:109A600080228347810039C41307000B6380E7021B
:109A70001387A7051377F70F8D4663EDE602A285DE
:109A8000280097C0FFFFE780201E79B78547E3F5E0
:109A900087F8834591001775010013056597B33565
:109AA000B00097A7FF1F238DB76C97500100E78088
:109AB000A0059DB703479100A207D98F356713070B
:109AC000D7556385E7086368F7022D671307B75515
:109AD0006387E70631671307C755638AE704296779
:109AE0001307A7556394E702A285280097C0FFFFDC
:109AF000E780805615B739679306E7656381D70815
:109B000063E9F6001307E7556384E706A28528009A
:109B10003DB73D679306F755638AD7061307F76687
:109B2000E396E7FE97C0FFFFE780006FF5B50146BB
:109B3000A285280097C0FFFFE780A03EF1BDA28567
:109B4000280097C0FFFFE780604FF9B58947E3F52C
:109B500087EC97000000E780A0E49305E4FFC205CE
:109B6000C1811305A1009790FFFFE78060676DB585
:109B7000A285280097C0FFFFE780004F71BDA28536
:109B8000280097C0FFFFE780C05979B597C0FFFF55
:109B9000E780406251B5C16717C5FF1F0355451CDB
:109BA000F9176307F500B7E7040003A3C71702839B
:109BB0008280854717C7FF1F2302F71A014517F355
:109BC000FFFF670083551783FFFFE702A34F2A8437
:109BD00008452E89B28919C900C1971500009385DF
:109BE000A586610597300100E780200581447D5AF4
:109BF00097100000E780E03963C7A4048144971000
:109C00000000E780003A63C8A40497C7FF1F93874A
:109C1000E7159C43DC47B307F94091872302F40022
:109C2000638309048327C900B307F4409587A3021F
:109C3000F4001C4C89C79C4799C3228582971783DF
:109C4000FFFF6700634B5C44139714008504BA97C9
:109C50002390470171BF1C48139714008504BA97DD
:109C60002390070069BF832789000547B307F440A5
:109C70009587A302F40083570400638EE7028DC327
:109C800009476384E7040D47E395E7FA97870100E6
:109C90009387C7E91CCC97870100938727EA11A80F
:109CA00097870100938707B01CCC978701009387A3
:109CB00067B05CC8BDBF978701009387A79B1CCC8A
:109CC000978701009387079CEDB7978701009387DB
:109CD000A7EA1CCC97870100938707EBD9BF95E5CE
:109CE0001783FFFFE702A33F004618448347940011
:109CF00075839D8B6317F70097100000E78060B4B1
:109D000048C41783FFFF6700C33F82801783FFFFAC
:109D1000E702433B13893500C16442094111AA8916
:109D20000144F11413590901054A2EC69710000089
:109D3000E7802026B2456348A4000145410117830E
:109D4000FFFF6700633B83A7090013171400BA974E
:109D500083D707006388B7006394970063742A0170
:109D60000504E1B70545D9BF1783FFFFE702A33418
:109D7000AA892E89328BB6843A8ABE8A97A00000BF
:109D8000E780C0FE71C9268597200000E780C00CDF
:109D90008D4763E7A7007D551783FFFF67002335D5
:109DA00083DB440097100000E780A0242A849710EA
:109DB0000000E78040259307740031443305850295
:109DC00063CDA70297100000E780A0229710000043
:109DD000E78020222A8497100000E780C0229307A2
:109DE000740031443305850263C3A7049710000053
:109DF000E78020209307450029A897100000E780FE
:109E00008020330585021307F0179307C017E35F1F
:109E1000A7FA2D55E3C277F963040B02D686528662
:109E2000A6854A8597200100E780C0BDB5B7971089
:109E30000000E780401D330585029307C5FFD1BFB1
:109E4000832749001385C90083D5270097000000A8
:109E5000E78000EC61F581B769553DBF97C7FF1FEB
:109E60002398A7F097C7FF1F938747F09043814738
:109E70000C463307F500420741836393B7008280A5
:109E80005446139847008507C2962390E600D5B73D
:109E900097C7FF1F938787ED9C4303C58700828088
:109EA00017C5FF1F0355C5EC82801783FFFFE7022C
:109EB0000323C1671387D7FF630BE502636AA7001B
:109EC000F1176300F50201451783FFFF6700632365
:109ED0001387E7FF6302E502FD171D8D133515009B
:109EE000E5B797500000E780602A7D15C5BF975001
:109EF0000000E780E0FED5BF97500000E78000FD3E
:109F0000EDB71783FFFFE702831D4111AA840144C7
:109F10002EC697100000E780C008B2456348A40031
:109F2000014541011783FFFF6700A31D9C481315DE
:109F300014003E9583570500E385B7FE0504C9BFAD
:109F400003485500814693F7F60F63E50701814703
:109F50003E858280584593975600BA9703D72700CD
:109F60006316B70003D70700E304C7FE8506E1BF09
:109F70008346450001479377F70F63E4D700814795
:109F800011A81C45131657000507B29703D6070002
:109F9000E313B6FE3E8582801783FFFFE70283123C
:109FA00093170501C18797CAFF1F938A2ADC635B59
:109FB000F00883A70A00C0479C4703570400198D87
:109FC000420541816368F500014422851783FFFF44
:109FD0006700831212052A94CDBFDC471394490011
:109FE000014A3E94834744006341FA02014A834791
:109FF00054006349FA028509C20993D9090183A76C
:10A000000A009847E3EBE9FCC1B71C4413195A0056
:10A01000A6853E994A8597000000E780C0EE05E1DD
:10A02000050AC9B75C4413195A00A6853E994A85AA
:10A0300097000000E78020ED19E1050A4DBFE30C11
:10A0400009FA61B7AA8481495DBF1783FFFFE70260
:10A0500003091C452A8481E79307C5001CC51C44DD
:10A06000231204001CC09307F00F63EDB70093F5B3
:10A07000F50F228597200000E780C0E51783FFFFDA
:10A080006700230893940501C167C18063F9F50057
:10A09000A685228597200000E780E0E8C5B7C1814A
:10A0A00093F5F50F228597200000E780A0E2A685B2
:10A0B000228597200000E780E0E3C9B797C7FF1F1C
:10A0C0009387C7CA884382801C4599C797C7FF1FDB
:10A0D00023AEA7C8014582807D55828097C7FF1FA8
:10A0E0009387C7C8984383474500484792073E95E2
:10A0F00082801783FFFFE70283FE617100451C1811
:10A100003EC6B70780013EC81C183ECA83574400AC
:10A1100002CE02D002CC231EF100834784002A899C
:10A1200002D22301F1023C083ED402D6970000007F
:10A13000E78000FB835705002316F10297500000CB
:10A14000E78000C82307A1025C4003556400F18347
:10A1500013F717008347F10252055181F99BD98FFC
:10A16000A307F10297100100E780207939CDAA8476
:10A170000355050097A00000E78020C083D70400A6
:10A180002AD26800231CF10083D72400231DF1008C
:10A190001C4803D647008C4397200000E780A0D0DE
:10A1A0008347B400CA861776010013062646811736
:10A1B000A305F4006C00481097200100E78080841C
:10A1C0005D611783FFFF6700C3F32155D5BF1C45B1
:10A1D000B1CF03C5A700894613576500630BD702AB
:10A1E0008D46630ED70285466300D70213074006EB
:10A1F0003305E50203C7B700418B15CB83C7B70012
:10A20000BD8B3355F54082801375F5031307803EEF
:10A21000C5B709671375F50313070771D1BF372752
:10A2200009001375F5031307077CD9B70145828030
:10A230001783FFFFE702A3EA03A98500630C090463
:10A240008347B900AE8493F7070E85C30345990091
:10A25000930520030D810505B305B502884461050A
:10A2600097300100E78080AD35A02E859700000073
:10A27000E78020F62A8419CD97000000E780605C13
:10A280008325C900B307B54063FA87002E94B30550
:10A29000A440E9F51783FFFF6700A3E685457DBF6E
:10A2A0001783FFFFE702A3E32A8403D5050001110A
:10A2B00032C636C43AC22EC002CA02CC02CE97A021
:10A2C0000000E78080AB82452ACA22852ECC970009
:10A2D0000000E780E0E003570500231EE1009750EF
:10A2E0000000E780E0ADA24632469247230FA1006E
:10A2F00036874C08B2862285014697000000E78029
:10A30000E0A605611783FFFF6700A3DF1783FFFF48
:10A31000E702E3DC61711C183EC6B70780013EC846
:10A320001C183ECA3C0800453ED4AA8402CC02CE8A
:10A3300002D002D202D697000000E78060DA83578D
:10A34000050035592316F10297500000E78040A719
:10A350002307A10209C48357440081EB21594A8590
:10A360005D611783FFFF6700C3D903556400520581
:10A37000518197100100E78040582A8965D18347B1
:10A38000B40093F7070E99C71305840197300100B5
:10A39000E780009D83574400231EF100834784001B
:10A3A0002301F1025C4003550900D98313F7070824
:10A3B00083471102231CA10093F7F707D98FA3004D
:10A3C000F10283572900231DF1005C40F18313F74C
:10A3D00017008347F102F99BD98FA307F10297A0D9
:10A3E0000000E78080992AD235D98347940068001D
:10A3F000139757008347B400FD8BD98FA305F40052
:10A400001C4803D647008C4397200000E780A0A992
:10A41000A687177701001307671F740005464C10C5
:10A42000268597000000E78060942A890DD983472C
:10A43000B400A685FD8BA305F40097000000E7801B
:10A4400060DF31BF1783FFFFE70263C9832485FE06
:10A450002A844111268597000000E78080D7834732
:10A4600034FF93F7070E8DCB2AC626859700000090
:10A47000E78060C809CD834734FFB245FD8BA3094F
:10A48000F4FE91C5228597300100E780208B4101C1
:10A490001783FFFF6700E3C67DD98327C4FF2685A6
:10A4A000829775F5834734FF93F7070E91C722858E
:10A4B00097300100E780C08A032584FE97000000E2
:10A4C000E78000E5E9B71783FFFFE70243BE9C4141
:10A4D00041112A8903C7070089472E8493566700D4
:10A4E0006380F6040D466388C6049307F00763048F
:10A4F000F7022E8597200000E78060ABAA8481498F
:10A50000C16B130C490097C7FF1F938727869C4395
:10A51000984763E4E90441011783FFFF6700E3BC48
:10A5200003D745008547E3F8E7FE2E859720000016
:10A53000E78040ADE1B703D74500E3FEE7FC2E8599
:10A5400097200000E780A0A6AA842285972000001B
:10A55000E78000A8C204C98C5DB7DC470355A90099
:10A56000139A49003E9A93170501C187635DF00075
:10A5700083570A006397A70263E774038327CA001F
:10A58000034D5A002DA0A1672167A98F1307F7EF8C
:10A59000E374F7FE6397090097000000E7802091BD
:10A5A00061FD85098DB783278A00034D4A00835DCD
:10A5B000A90003576900216A138BC7003AC6814A74
:10A5C00033CA4D01631E5D0197B7FF1F9387877ADA
:10A5D0009C43E1DBA2866286814526858297D1B7BE
:10A5E000A1679387F7EF930C4BFF63F24703B245E4
:10A5F0005A8597F0FFFFE780A0710DC103278B00FC
:10A60000104709CE10436382C4023107D5BFEE85DF
:10A61000668597000000E780008F71F993861A0025
:10A6200093FAF60F130B0B0271BF835644005C4381
:10A63000E3E9F6F622853AC697200000E7802081FC
:10A64000A1679387D7042A8A035D4400324763E8F1
:10A6500097008347D90093E707F8A306F9001C4742
:10A6600066852286E2858297C1670844FD17337AA2
:10A67000FA00529508C02312A40125B797B7FF1F0F
:10A680009387C76E9843814715C31447814763FF7B
:10A69000D500939745004C47BE9519C903C755008F
:10A6A00081476375E600DC451606B2973E858280D9
:10A6B00003C745008147E37BE6FE16069C45F5B7D8
:10A6C0001783FFFFE70203A0AA892E8A814497BA65
:10A6D000FF1F938AAA6983A70A00984763E6E400EC
:10A6E0001783FFFF670043A1DC471394440001492F
:10A6F0003E9413BB140083474400634BF9000149A7
:10A7000013BB140083475400634FF9008504E1B77D
:10A710000844931759005287DA860146A2853E9570
:10A7200082990509C9BF4844931759005287DA86B0
:10A730000546A2853E9582990509E9B71783FFFF73
:10A74000E702E399814517F5FFFF1305054897B721
:10A75000FF1F239F076097000000E780A0F6178384
:10A76000FFFF6700039A97B7FF1F938727609C43FB
:10A7700095C31783FFFFE7028396814517F5FFFF17
:10A780001305A54497000000E780C0F31783FFFF7F
:10A790006700239782801783FFFFE702A39237E4C5
:10A7A00004008327841241112315E100AE89328908
:10A7B000368A3A8681460147ED45AA8482972AC6A1
:10A7C00021C90356A100D28597400100E780602887
:10A7D0008327C413CE8526858297058905C98327DB
:10A7E000440D2314210101462C00268582972A84DA
:10A7F00001C9B7E7040083A7C712ED452800829777
:10A80000228541011783FFFF6700038F4944D5B7B5
:10A810006554FDB75C41FD175CC182801783FFFF63
:10A82000E702E38BB7E70400FC5F829795473305A7
:10A83000F50281450D811783FFFF6700838C178325
:10A84000FFFFE702C389B7E70400FC5F82979547E3
:10A850003305F5020D811783FFFF6700838A178395
:10A86000FFFFE702C387B7E7040083A7870B035501
:10A87000050082971783FFFF6700A3881783FFFFF8
:10A88000E702E385035505003287AE861796FF1F62
:10A89000035666C297B5FF1F9385054E97000000CB
:10A8A000E780A0EF1783FFFF6700A3851783FFFFF3
:10A8B000E702E382B7E7040083A7C71782971783ED
:10A8C000FFFF670003841783FFFFE7024381B7E7B9
:10A8D000040083A7871397B5FF1F9385E5498297E7
:10A8E00001451783FFFF6700C3811773FFFFE7026E
:10A8F000037FB7E7040083A7C71F81451795FF1F94
:10A90000035565B782971773FFFF6700837F17733F
:10A91000FFFFE702C37CB7E7040083A7871397B55F
:10A92000FF1F93856546829701451773FFFF6700F8
:10A93000437D1773FFFFE702837AB7E7040083A71D
:10A94000C71F81451795FF1F0355E5B882971773F9
:10A95000FFFF6700037B1773FFFFE70243782E8535
:10A9600097800000E78080B397800000E78080F048
:10A970001773FFFF6700E3781773FFFFE702237683
:10A9800097800000E78080FA1773FFFF6700637706
:10A990005C49E1175CC95CC583572501A1072319F0
:10A9A000F50083570501A1072318F5008280F147C0
:10A9B0003305F50297B7FF1F9387073F9C433E95EA
:10A9C00082808D476315F60803D74600854763F0FC
:10A9D000E7081773FFFFE7028370368536842E89F8
:10A9E00097100000E780A05C29C9835744009314A6
:10A9F0000501C18063E39704228597100000E7807A
:10AA0000005BFD14231294009307A0026300F5027B
:10AA10009307B0026307F50293079002631FF500E6
:10AA2000228597000100E780608901A80146CA8558
:10AA3000228597A00000E78000B41773FFFF67002E
:10AA4000436C228597100000E7806007FDB7828085
:10AA500097B6FF1F938686359C42014599CF984350
:10AA6000D44217B6FF1F2323E6346396D70097B668
:10AA7000FF1F23AFE6321385C7FE82801773FFFFE7
:10AA8000E702E36597000000E780A04B71443305BF
:10AA90008502914597900000E780C0EC11E565556F
:10AAA0001773FFFF6700E36597B7FF1F23ACA72E5F
:10AAB00097000000E780E0483305850291459790B4
:10AAC0000000E78020EA61DD97B7FF1F23AEA72CC7
:10AAD00097000000E780E04697B7FF1F239EA72A54
:10AAE00097000000E780E04597B7FF1F2397A72A4C
:10AAF000977701009387C7B617B7FF1F2322F72A5E
:10AB000097070000938707E917B7FF1F2328F72847
:10AB1000014579B71773FFFFE702635CAA8517B594
:10AB2000FF1F1305652797100000E780605F17730C
:10AB3000FFFF6700035D1773FFFFE702435A9700AB
:10AB40000000E78060FD97100000E780E05E97B7A7
:10AB5000FF1F9387A7259C4391CF1387C7FE19CB6F
:10AB600083D5C7FF17B5FF1F1305C5249720010024
:10AB7000E780C01C1773FFFF6700A3581773FFFF20
:10AB8000E702E35597000000E780C0EC09CD83475A
:10AB900085002A8493F7070499EB0355E500970095
:10ABA0000000E78080F91773FFFF67008355834734
:10ABB000C5009304450117B9FF1F1309291F85E339
:10ABC000832709005CC997B7FF1F23A1971E83271E
:10ABD0004900F1FB97B7FF1F23AC971CE9B7FD179E
:10ABE0002306F500610597800000E78060DA83079F
:10ABF000840063CB07048347840093E707F82304AA
:10AC0000F400B7E704009C5F82974205A9474181A1
:10AC10003375F5028347840093F707FCC98F23043B
:10AC2000F4008347D4003E951C402318A40089CF2C
:10AC3000984319CB8347C4005040814585073305AD
:10AC4000F502420541810297832709005CC897B746
:10AC5000FF1F23AD97148327490089E797B7FF1F8C
:10AC600023A897148347C4009DDF8355040117B5BB
:10AC7000FF1F1305251497200100E780200C25B73E
:10AC80001773FFFFE702A34597B7FF1F9387C737E7
:10AC90009C4701448583858B85E3AE84B2853A86E3
:10ACA00097100000E780204F2A8419C597100000F4
:10ACB000E7806045829408CC22851773FFFF670008
:10ACC00043441773FFFFE702E33F41112E8932C669
:10ACD000AA8997000000E780C031324713060502B9
:10ACE000CA86970500009385C5CC17B5FF1F1305CD
:10ACF000A50A97000000E780E0F82A8425C993049C
:10AD0000C50097000000E780E0411946AA85268526
:10AD100097100000E78020198545268597100000D0
:10AD2000E780001517750100130545914E95834581
:10AD30000500268597100000E780C0195C48314661
:10AD40008145A1075CC85CC483572401E11723191E
:10AD5000F40083570401E1172318F4001C4C3E85CE
:10AD60009770FFFFE780A03AA304250122854101E7
:10AD70001773FFFF670043381773FFFFE70223369F
:10AD80004111AA842EC632C497100000E780003A11
:10AD9000004DB2452246834784000CC050C093F753
:10ADA000F70393E707042304F4002318040026851F
:10ADB00097100000E780203583479400A9462317A9
:10ADC000A40013D7370005073307D7029D8B8507EB
:10ADD0002306F400A306E40083C70401D8488507CE
:10ADE000230FF7FE17B7FF1F130747FC5843232A0B
:10ADF00004009307440129E317B7FF1F232AF7FA3A
:10AE000017B7FF1F2324F7FA17B4FF1F130484FAA0
:10AE1000228597200100E780A0E41C44858B5D8D8E
:10AE200019E58145228597200100E78020F1410145
:10AE30001773FFFF6700E32C1CC317B7FF1F2329FD
:10AE4000F7F6D9B71773FFFFE702632997050000EC
:10AE5000938565B7014597000000E78000B0014584
:10AE60001773FFFF6700E3291773FFFFE70223272C
:10AE700097000000E78080B01773FFFF670063282A
:10AE80008347C500A5E31773FFFFE70243252A8424
:10AE90000355E50097000000E78000C821C1834703
:10AEA000840093F7F7FB2304F4001C4091C7DC43B4
:10AEB00081C74C400145829797000000E78080B928
:10AEC00017B5FF1F130505EF97200100E78040E944
:10AED0000355E40097000000E78020C61773FFFFCA
:10AEE0006700232282801773FFFFE702431F97B793
:10AEF000FF1F9387A7EB97050000938565C817B5DB
:10AF0000FF1F130525EB23A0070023A207009720AE
:10AF10000100E78080D21773FFFF6700831E1C4D7E
:10AF200091CFDC4381CF1773FFFFE702431B8345BB
:10AF3000070082971773FFFF6700A31C828097B7F3
:10AF4000FF1F938767E99C4303C50700828097B77B
:10AF5000FF1F938767E89C4303C51700828097B75C
:10AF6000FF1F938767E79C4303C52700828097B73D
:10AF7000FF1F938767E69C4303C54700828097B70E
:10AF8000FF1F938767E59C4303C53700828097B70F
:10AF9000FF1F938767E49C4303C55700828097B7E0
:10AFA000FF1F938767E39C4303C56700828097B7C1
:10AFB000FF1F938767E29C4303C57700828097B7A2
:10AFC000FF1F938767E19C4303C58700828097B783
:10AFD000FF1F938767E09C4303C59700828097B764
:10AFE000FF1F938767DF9C4303C5A700828097B745
:10AFF000FF1F938767DE9C4303C5B70011E11D4522
:10B00000828097B7FF1F938727DD9C4303C5C70046
:10B01000828097B7FF1F938727DC9C4303C5D70027
:10B02000828097B7FF1F938727DB9C4303C5E70008
:10B03000828097B7FF1F938727DA9C4303D50701C8
:10B04000828097B7FF1F938727D99C4303C52701A9
:10B05000828097B7FF1F938727D89C4303D547016A
:10B06000828097B7FF1F938727D79C4303D567013B
:10B07000828097B7FF1F938727D69C4303D587010C
:10B08000828097B7FF1F938727D59C4303C5A701ED
:10B09000828097B7FF1F938727D49C4303C5B701CE
:10B0A000828097B7FF1F938727D39C4303C5C701AF
:10B0B000828097B7FF1F938727D29C4303C5D70190
:10B0C000828097B7FF1F938727D19C438857828040
:10B0D00097B7FF1F938747D09C4303D5C702828051
:10B0E00097B7FF1F938747CF9C4303D5E70219E12A
:10B0F0001305800C828097B7FF1F9387E7CD9C4391
:10B1000003C50703828097B7FF1F9387E7CC9C4353
:10B11000C85B828097B7FF1F938787CB8843828065
:10B1200097B7FF1F938707CB8843828019E17D552E
:10B130008280F5DE984265DFFDD917B7FF1F130740
:10B14000A7EC1847AA877155058B631D072403C513
:10B1500007001547E37DA7FC03C737001305F0057B
:10B160007D171377F70FE364E5FC03C35700E30093
:10B1700003FC83C86700E38C08FA03C777004945DE
:10B1800079171377F70FE364E5FA03C7A7001148AF
:10B190001305F7FF1375F50FE36BA8F803CE9700BF
:10B1A0000D481305FEFF1375F50FE362A8F803C8F9
:10B1B000B7006309080065181378F80F1305600DD0
:10B1C000E36705F703C5C700794879151375F50FCF
:10B1D000E36FA8F403C8D7000D457D181378F80F66
:10B1E000E36705F503D80701930E4017511842088D
:10B1F00013580801E3ED0EF303C8E7007D18137838
:10B20000F80FE36605F303C827017D181378F80FDC
:10B21000E36F05F103C88700C54E75181378F80F62
:10B22000E3E70EF103D86701856E938EBEE06D18DB
:10B23000420813580801E3EC0EEF03D847016D18DC
:10B24000420813580801E3E40EEF03D88701791888
:10B25000420813580801E36C05ED03C8A7017D18E7
:10B260001378F80FE36505ED03C5B7011D487D159B
:10B270001375F50FE36DA8EA03C5D7017148791579
:10B280001375F50FE365A8EA03D5E7011308E00F8E
:10B290007D1542054181E36CA8E803C507024948D2
:10B2A00079151375F50FE364A8E8C85301C937C8C9
:10B2B00034005915130858BFE36BA8E603A88702AA
:10B2C00037C53400130555BF5918E36205E717B5B4
:10B2D000FF1F2321C5B003C6050117B5FF1F232D8E
:10B2E000F5AE0545E375C5E403D82501D0493376AD
:10B2F0000603E31E06E203C61501E30A06E217B6DB
:10B30000FF1F2327B6AC83C5270001466387A5002E
:10B3100003C61700F1453306B60283C7070393053A
:10B32000C00272971A071307C70516031A979608E3
:10B330004697B387B70241553E97329742074183FC
:10B340006362E8061773FFFFE70263D936859780CB
:10B350000000E780406C97000100E780C04B2A8422
:10B3600097A00000E780205E2A9497F00000E78015
:10B37000002A2A9497900000E78040852A9497F04D
:10B38000FFFFE780E06F2A9497400000E780009776
:10B390002A9497700000E78040A022951773FFFF62
:10B3A000670023D682801773FFFFE70243D3411162
:10B3B000A307A10097A00000E78040C99305F10012
:10B3C000170500001305E5B597F0FFFFE780802F14
:10B3D000014541011773FFFF6700A3D21773FFFFF9
:10B3E000E70263CD17B4FF1F130404C203288400CF
:10B3F00079599368180097B4FF1F23AB14C11378D1
:10B40000180063100802BA84BE89368B328A2E89EE
:10B41000AA8A97F0FFFFE780E0A77D15269519E53A
:10B4200031594A851773FFFF670063CC97F0FFFF20
:10B43000E78040A67D152695A167E353F5FE97B7F3
:10B44000FF1F938727F398433E8C814B01CB014527
:10B4500097F00000E780C047933B15004A85DA86E5
:10B460005686D28597900000E78060512A8911CDD9
:10B470001C44F99B17B7FF1F232CF7B883270C0038
:10B48000CDD3E3800BFA829769BF268597B7FF1F5C
:10B4900023AE07B697F0FFFFE780809C4146CE853C
:10B4A00017B5FF1F1305C5BF97300100E780605A2D
:10B4B00097D00000E780E09C0325040B97D00000A4
:10B4C000E780A0A0054597D00000E780A0A705452C
:10B4D00097000000E78060EDA9B797B7FF1F93873B
:10B4E000A7B29C47858BEDC71773FFFFE70223BF09
:10B4F00017B5FF1F130505B997B7FF1F23A607B0A0
:10B5000097B7FF1F23A407B097B7FF1F23A207B069
:10B5100097200100E780C08497500000E78080F901
:10B5200097100100E780405097100100E7804056D7
:10B5300097B7FF1F9387C7AB9C4391C7054597807B
:10B540000000E780E02397B7FF1F938727949C4371
:10B5500099C741657D1597700000E780E0A597F0D9
:10B560000000E780804197D00000E780209397B7E4
:10B57000FF1F938727BE9C4313971701635607004D
:10B5800097F00000E780A0B097B7FF1F23AA07B08D
:10B5900097B7FF1F23A807B097B7FF1F23A607B0D1
:10B5A00097B7FF1F23A407B097000000E780008C27
:10B5B00097000000E780A07597F0FFFFE780401834
:10B5C00097F00000E780E0D91773FFFF670063B3CF
:10B5D000828097B7FF1F938727A38843828097B7FE
:10B5E000FF1F938767A2C8438280B7E7B0009387A5
:10B5F000075063E1A70297B7FF1F9387E7A0D843DF
:10B60000FD576367E50097B7FF1F23A1A7A08147F8
:10B610003E858280B957EDBF1773FFFFE70223AC69
:10B6200097800000E780607597800000E780C07712
:10B630001773FFFF6700E3AC1773FFFFE70283A8F0
:10B640002A849304140201112E85B289A68521460D
:10B6500036C63A8997300100E780403D0DE9B24691
:10B6600038082686CE851305940497500000E7809D
:10B67000604121462C084A8597300100E780003B55
:10B680001335150005611773FFFF6700E3A6014539
:10B69000D5BF1773FFFFE70283A49305450617A5DF
:10B6A000FF1F1305A57397100100E780206917732A
:10B6B000FFFF670003A51773FFFFE70243A24111D5
:10B6C0002EC697F0FFFFE780C017B24588C1410141
:10B6D0001773FFFF6700E3A21773FFFFE702839E64
:10B6E000AA842E8497800000E780006CAA89854593
:10B6F000228597000000E780E07D83C7E40113897D
:10B70000940899E313890403CE85228597000000ED
:10B71000E780407C214693051902228597000000AE
:10B72000E780607897B7FF1F9387078E8C43228549
:10B7300097100000E780C08221469385840222850D
:10B7400097000000E78020761773FFFF6700C39A19
:10B750001773FFFFE7022396397197F00000E78027
:10B76000E0B49305400661E997800000E78000603F
:10B770006302051497A7FF1F83C7076813B7170055
:10B7800097A6FF1F238AE666014499CFC16417B9C3
:10B79000FF1F130969879309400EFD1497000000ED
:10B7A000E78020836342A40A97F0FFFFE7806009E7
:10B7B0004169B7290900096AFD7A2A8B81447D19FC
:10B7C0009389F97B130A0A71938A8AC7970000004C
:10B7D000E780208063D7A4041304400EB38784025B
:10B7E00017B7FF1F130747820324070B3E948357A5
:10B7F000C4016382270B18403307EB4063EAE9007A
:10B80000834744008507B3874703D6976365F708E6
:10B8100001468145094597F0FFFFE780C04AAA8BA2
:10B8200029E597400000E780808385476317F50688
:10B8300089659385057117A5FF1F1305255A971074
:10B840000100E780A04F95A0B30734030327090B3D
:10B85000BA9703D7C7016308970003C75700A382AD
:10B8600007002382E700050415BF9305C500228564
:10B8700097000000E78080E65E85228697650100DC
:10B88000938505DD97F0FFFFE780404F5E859710B9
:10B890000000E780608A850415BF97A7FF1F938784
:10B8A000A7769C478D83858BC1F721611773FFFFB6
:10B8B0006700E38301468545094502D002D202D4E0
:10B8C00002D697F0FFFFE7800040AA8479DD97F069
:10B8D0000000E780E09C1389C4002A8481454A85E2
:10B8E00097000000E780005F0C4041464A859700C2
:10B8F0000000E780405B832944006385090C4E8586
:10B9000002D802DA02DC02DE97300100E780E0387C
:10B910002ACE141005462C0808184ECC975000006B
:10B92000E780E00A1375F50F51ED8355840093E528
:10B9300025004A8597000000E780E05E11460C1064
:10B940004A8597000000E780005601469765010090
:10B95000938585D0268597F0FFFFE78020422685D6
:10B9600097000000E780407D5C40A1D301468545FB
:10B970000D4597F0FFFFE7800035AA841DD54840AC
:10B980001389C40097300100E78020312AC64A8518
:10B9900097000000E780404C3246636FC5004C4082
:10B9A0004A8597000000E7800050014681452685C2
:10B9B00097F0FFFFE780803C268597000000E78036
:10B9C000A077E5B583558400ADB71763FFFFE702A5
:10B9D000037197A7FF1F938727639C471DC193E7B8
:10B9E000870017A5FF1F1305653F17A7FF1F23211A
:10B9F000F76297100100E78040321763FFFF67008E
:10BA00004370DD9B17A7FF1F2324F76097300000CA
:10BA1000E780E0647DF117A5FF1F1305253C971013
:10BA20000100E780E033D1BF1763FFFFE702A3689F
:10BA30004169AA892E8AB28A368BBA8B814417ACA7
:10BA4000FF1F130C6C5C930C400E7D1997F0FFFFE9
:10BA5000E780205863C4A40001443DA033849403CC
:10BA600083270C0B3E948357C401638627055A87AE
:10BA7000D6865286CE851305040397000000E78022
:10BA8000E0BB01C923800B0022851763FFFF67001D
:10BA900003668347F40185C35A87D6865286CE85CE
:10BAA0001305940897000000E78040B909C5854751
:10BAB0002380FB00D1BF850451BF835745006380BD
:10BAC000071E1763FFFFE702E35F01112A84970057
:10BAD0000000E780C04D09C985476309F506056187
:10BAE0001763FFFF6700436197E00000E780007C79
:10BAF0007DF5835744004947ED9BE392E7FEC1453E
:10BB0000228597000000E7804033AA8422859700B1
:10BB10000000E780204F0357440002CE91472A8956
:10BB2000631AF700228597000000E780A0513C08C7
:10BB30002ACC3ECE97E00000E78080765C55C5D3E6
:10BB400074084A86A6850545829751BF035744006D
:10BB5000D147E3F6E7F8032A0400C169014997AA2F
:10BB6000FF1F938A6A4A130B400EFD1997F0FFFFDF
:10BB7000E7802046634FA90E2285032A0400970020
:10BB80000000E780C042A1452A8922859700000075
:10BB9000E780A02AAA84228597000000E780804AD7
:10BBA00014402A86AA8978082685CA85970000004D
:10BBB000E780C0E7AA8405D503C7F4018947631568
:10BBC000F7008347C10181DF5546D28513856400A4
:10BBD00097300100E780E0E7014597800000E780AB
:10BBE000C01901C583D7C401A5E797A7FF1F938795
:10BBF000A7419C4793551900858913D73700058BBA
:10BC000001CF8983858B6399B70001452EC69700C4
:10BC10000000E780C0DBB2454E8597800000E780DA
:10BC2000601F0346C1012A849375190026859790E9
:10BC30000000E780E03935C1268597800000E78065
:10BC4000E018268511C0014597800000E780004C70
:10BC500097300000E780A0408547E312F5E883C7EE
:10BC600054001307F00FE38CE7E68507A382F40086
:10BC7000BDB5B304690383A70A0BBE9483D7C4017F
:10BC8000638B37015546D2851385640097300100D8
:10BC9000E780C0D955DD0509D1BD5DD86DB782807B
:10BCA0001763FFFFE702034297800000E780000C64
:10BCB00005C1C164014417A9FF1F1309E9349309A1
:10BCC000400EFD1497F0FFFFE780A030634EA40004
:10BCD00017A5FF1F1305851097100100E780E003EB
:10BCE0001763FFFF67004341330534038327090BC4
:10BCF0003E958357C50163889700231205009780FE
:10BD00000000E780A00C050475BF97A7FF1F93876D
:10BD1000A72F9C478D83858B8DE31763FFFFE70279
:10BD2000033C17A5FF1F1305650B97100100E78063
:10BD300020031763FFFF6700C33C82801763FFFF88
:10BD4000E702E339970500009385C5A017A5FF1FFB
:10BD50001305C50897100100E78020EE1763FFFF69
:10BD60006700233A1763FFFFE70263378841B7E7AD
:10BD70000400BC5B050542054181829709C58547E2
:10BD80002300F50005051763FFFF6700833783C7AE
:10BD9000F5FF2E858507A38FF5FE828083C7F5FF0B
:10BDA000FD1793F7F70FA38FF5FE99EF1763FFFFCA
:10BDB000E702E332B7E70400BC571385F5FF82972B
:10BDC0001763FFFF6700E33382801C410357450080
:10BDD0008D8FBA951CC12312B5003E85828093D702
:10BDE0008500A2051441DD8D835745001387E6FFCA
:10BDF00018C189072312F50013D685004111238F3E
:10BE0000B6FEA38FC6FE4101828018419307F7FF5B
:10BE10001CC18357450085072312F500A30FB7FE09
:10BE20008280835745008D8F2312F5001C41BE95FB
:10BE30000CC12E858280AA8703D7470008410D8F49
:10BE4000AA952392E7008CC38280184108453305E8
:10BE5000A740828083574500035765001D8F1C4112
:10BE600008453385A7403305A74082801763FFFF4D
:10BE7000E702E32641112EC62A8497000000E780DE
:10BE8000A0FDB2456373B50001A08357440008408C
:10BE9000BE952312B4003E9541011763FFFF670072
:10BEA00043261763FFFFE702832341112E84B285E7
:10BEB00032C697000000E780A0FB3246A28597308B
:10BEC0000100E78000B941011763FFFF67006323AA
:10BED0001763FFFFE702A3202E848545970000002B
:10BEE000E78000F9230085001763FFFF67006321E7
:10BEF0001763FFFFE702A31E41112317B100894515
:10BF000097000000E780C0F68347E1002300F500BA
:10BF10008347F100A300F50041011763FFFF6700AD
:10BF2000431E1763FFFFE702831B93D78500A2051B
:10BF30004111DD8D2317B100894597000000E7808E
:10BF400020F38347E1002300F5008347F100A300BD
:10BF5000F50041011763FFFF6700A31A1763FFFF96
:10BF6000E702E3171397850193D78501C16693868E
:10BF700006F0D98F13D78500758FD98FA2053707A3
:10BF8000FF00F98D4111DD8D2EC69145970000000F
:10BF9000E78000EE6C00114697300100E78060AB4F
:10BFA00041011763FFFF6700C3151763FFFFE70237
:10BFB00003131C41854503C4070097000000E78078
:10BFC00080E622851763FFFF6700A3131763FFFF57
:10BFD000E702E3101C414111894503C7070083C7ED
:10BFE00017002307E100A307F10097000000E78096
:10BFF00080E30355E10041011763FFFF6700631011
:10C000001763FFFFE702A30D1C414111894503C7D8
:10C01000070083C717002307E100A307F10097007B
:10C020000000E78040E08357E100410113D587001D
:10C03000A2075D8D420541811763FFFF6700630C16
:10C040001763FFFFE702A3090C4141112A8411463F
:10C05000680097300100E780C09F914522859700D6
:10C060000000E78040DCB247C166938606F0139774
:10C07000870113D58701598D13D78700758F598D87
:10C08000A2073707FF00F98F5D8D41011763FFFF9E
:10C09000670023071C45BE950CC18280AE87944380
:10C0A00091E6584101EF0CC15CC1828003C7570083
:10C0B00013671700A382E700B687D5B70CC3EDB7A7
:10C0C000AA87084119CD1841D44398C36313D500FA
:10C0D000D8C32A87034657009376160081E62320AB
:10C0E00007008280944381CA8C4203A847008CC316
:10C0F00063930601CCC3799A14C3A302C7003687A1
:10C10000D1BF1C45DC471D8DB777DBB6938777DB46
:10C1100009853305F502420541818280F147B385E7
:10C12000F50248452E958280834745008507230206
:10C13000F50082801763FFFFE70263FA2A8409E4AF
:10C140001763FFFF6700E3FB83474400F5DBFD1740
:10C1500093F7F70F2302F400E5F71C4403D72700F9
:10C1600005072391E700DC4399C3228582974C4859
:10C1700089CD83475400898B99E71C4422859C47CD
:10C180009C439C478297232A0400004023200400FC
:10C190007DB71763FFFFE70283F483572500411142
:10C1A0002EC681EB0144228541011763FFFF670022
:10C1B00043F5035705008147F146E305F7FEB385D4
:10C1C000D702404585072E948345440008C4F5F501
:10C1D000B247AA8481E7232A040009A81C456C0001
:10C1E00022859C439C43829748C84DDD8547231296
:10C1F000F400B24723200400231804002319F4009C
:10C200005C485CC483D72400FD172391F40061BF10
:10C210001763FFFFE702A3EC97A7FF1F938707BEF3
:10C2200088432326050023240500410597100100BB
:10C23000E78000B31763FFFF6700A3EC1763FFFFFE
:10C24000E702E3E917A4FF1F130444BB1C4041119C
:10C2500099CF9C472300B5002AC65CC19700000017
:10C26000E78040FB1C40DC4399C332458297410183
:10C270001763FFFF6700E3E80347450029E3584DD4
:10C28000AA877D551DCF1763FFFFE70243E51CC357
:10C29000DC4797A6FF1F23A3E6B6F1561305070157
:10C2A0002390D700970500009385050297100100A1
:10C2B000E780A09801451763FFFF670083E47D5581
:10C2C000828082801763FFFFE70263E1011161460C
:10C2D000814528009760FFFFE78060E397A7FF1F75
:10C2E0009387C7B19C4328009305F00FDC473EC6F7
:10C2F00097000000E780C0F405611763FFFF670047
:10C3000043E097A7FF1F938767AF9C43D847A16778
:10C310009387C702631EF70A397106DE22DC26DA2C
:10C3200080004AD84ED652D456D23285B284970075
:10C330000000E780C0C7AA89268597000000E78033
:10C3400020C92318A4FC268597000000E78040C878
:10C350002319A4FC268597000000E78060C783D7D7
:10C3600044000A8A231AA4FC858393F7F70F230E4F
:10C37000F4FC8607BD0793F7073F3301F1408A8A33
:10C3800001498347C4FD6367F902CE85130584FC28
:10C39000232C54FD97000000E78080EA52811301AE
:10C3A00004FCF2506254D2544259B259225A925A61
:10C3B00021618280268597000000E78060C1931785
:10C3C0001900D69705092390A7001379F90F55BFD7
:10C3D000828097A7FF1F938767A29C43D847A167D6
:10C3E0009387A702631AF70A397106DE22DC26DA80
:10C3F00080004AD84ED652D456D23285B2849700A5
:10C400000000E780C0BAAA89268597000000E7806F
:10C4100020BCFD572318A4FC26852319F4FC9700A3
:10C420000000E780E0BA83D744000A8A231AA4FCFC
:10C43000858393F7F70F230EF4FC8607BD0793F768
:10C44000073F3301F1408A8A01498347C4FD63678E
:10C45000F902CE85130584FC232C54FD97000000BF
:10C46000E78000DE5281130104FCF2506254D25482
:10C470004259B259225A925A2161828026859700E8
:10C480000000E780E0B493171900D69705092390C0
:10C49000A7001379F90F55BF828097A7FF1F9387D5
:10C4A000E7959C43D847A16789076310F70A39715C
:10C4B00006DE22DC26DA80004AD84ED652D456D286
:10C4C0003285328997000000E78060AEAA894A85EC
:10C4D00097000000E780C0AF835749000A8A2318FD
:10C4E000A4FC858393F7F70F230CF4FC8607BD07A4
:10C4F00093F7073F3301F1408A8A8144834784FDE3
:10C5000063E7F402CE85130584FC232A54FD9700CB
:10C510000000E780E0D25281130104FCF250625423
:10C52000D2544259B259225A925A216182804A8584
:10C5300097000000E780C0A993971400D697850460
:10C540002390A70093F4F40F55BF828097A7FF1F95
:10C550009387C78A9C43D847A1679387E704631EE4
:10C56000F70A397106DE22DC26DA80004AD84ED678
:10C5700052D456D23285B28497000000E78020A3BF
:10C58000AA89268597000000E78080A42318A4FCD0
:10C59000268597000000E780A0A3231AA4FC268527
:10C5A00097000000E780C0A283D744000A8A2319BD
:10C5B000A4FC858393F7F70F230EF4FC8607BD07D1
:10C5C00093F7073F3301F1408A8A01498347C4FD4D
:10C5D0006367F902CE85130584FC232C54FD970074
:10C5E0000000E780E0C55281130104FCF250625460
:10C5F000D2544259B259225A925A216182802685D8
:10C6000097000000E780C09C93171900D697050992
:10C610002390A7001379F90F55BF82809797FF1FCA
:10C620009387C77D9C43D847A1679387C704631A44
:10C63000F70A397106DE22DC26DA80004AD84ED6A7
:10C6400052D456D23285B28497000000E7802096FB
:10C65000AA89268597000000E7808097FD57231858
:10C66000A4FC2685231AF4FC97000000E78040967E
:10C6700083D744000A8A2319A4FC858393F7F70F14
:10C68000230EF4FC8607BD0793F7073F3301F14003
:10C690008A8A01498347C4FD6367F902CE85130581
:10C6A00084FC232C54FD97000000E78060B9528180
:10C6B000130104FCF2506254D2544259B259225A26
:10C6C000925A21618280268597000000E780409081
:10C6D00093171900D69705092390A7001379F90F2E
:10C6E00055BF82809797FF1F938747719C43D84718
:10C6F000A167DD076317F7041763FFFFE702239EB7
:10C7000079713285328497000000E780408A2AC61A
:10C71000228597000000E780A08B2311A1022285CB
:10C7200097000000E780A088B2452300A1022808F6
:10C7300097000000E780C0B045611763FFFF670006
:10C74000439C82809797FF1F9387476B9C43D847F2
:10C75000A167938787046317F7041763FFFFE70256
:10C76000039879713285328497000000E780208435
:10C770002AC6228597000000E78080852311A10248
:10C78000228597000000E7808082B2452300A10245
:10C79000280897000000E780A0AA45611763FFFF03
:10C7A0006700239682809797FF1F938727659C4396
:10C7B000D847A1679387A7046312F7021763FFFFA7
:10C7C000E702E39101112800814597000000E7800E
:10C7D00020A705611763FFFF6700A39282809797E8
:10C7E000FF1F9387A7619C43D847A1679387570290
:10C7F0006319F7021763FFFFE702638E01113285A9
:10C8000097F0FFFFE780A07A2308A1008145280068
:10C8100097000000E780C0A205611763FFFF670073
:10C82000438E82809797FF1F9387475D9C43D8472D
:10C83000A1679387E702631BF7041763FFFFE70213
:10C84000038A01113285328497F0FFFFE780407838
:10C85000AA84228597F0FFFFE7808077854709E962
:10C86000228597F0FFFFE78080744205B337A00070
:10C8700028008145231891003ECA97000000E780F8
:10C88000209C05611763FFFF6700A387828097974D
:10C89000FF1F9387A7569C43D84799476313F70810
:10C8A0001763FFFFE702A38379713285328497F023
:10C8B000FFFFE780C06F2AC6228597F0FFFFE78061
:10C8C00020712310A102228597F0FFFFE780206EE0
:10C8D0002301A102228597F0FFFFE780406DA301AD
:10C8E000A102228597F0FFFFE780606C2302A1027E
:10C8F000228597F0FFFFE780806B2313A10222853A
:10C9000097F0FFFFE780A06AB2452314A102280830
:10C9100097000000E780C09245611753FFFF670052
:10C92000437E82809797FF1F9387474D9C43D8474C
:10C93000A1679387C7036313F7081753FFFFE70245
:10C94000037A79713285328497F0FFFFE7802066A1
:10C950002AC6228597F0FFFFE78080672310A10297
:10C96000228597F0FFFFE780A0662311A1022285B0
:10C9700097F0FFFFE780A0632302A102228597F0D2
:10C98000FFFFE780C062A302A102228597F0FFFFAC
:10C99000E780E0612303A102228597F0FFFFE78093
:10C9A0000061B245A303A102280897000000E780B8
:10C9B000208945611753FFFF6700A37482801753D6
:10C9C000FFFFE702C37101112A8497F0FFFFE780A0
:10C9D000005EAA84228597F0FFFFE780605F2285D2
:10C9E00097F0FFFFE780C05E035744008D4763F771
:10C9F000E700228597F0FFFFE780805D228597F0B2
:10CA0000FFFFE780E05C2800A68597000000E78034
:10CA1000208305611753FFFF6700A36E9797FF1FE1
:10CA20009387C73D9C43D847A167FD07631FF70065
:10CA30001753FFFFE702A36A328597000000E780E3
:10CA400040F81753FFFF6700C36B82809797FF1F63
:10CA50009387C73A9C43D847A167E5076315F70852
:10CA60001753FFFFE702A36779713285328497F08D
:10CA7000FFFFE780C0532AC6228597F0FFFFE780BB
:10CA80002055228597F0FFFFE78080542310A102F4
:10CA9000228597F0FFFFE780A053520551812311B3
:10CAA000A10222852302010297F0FFFFE7802050B8
:10CAB000A302A102228597F0FFFFE780404F2303E6
:10CAC000A102228597F0FFFFE780604EB245A303E5
:10CAD000A102280897F0FFFFE78080764561175391
:10CAE000FFFF6700036282809797FF1F93870731DC
:10CAF0009C43D847A1679387E703631FF700175349
:10CB0000FFFFE702C35D328597000000E78060EB1E
:10CB10001753FFFF6700E35E82809797FF1F93879D
:10CB2000E72D9C43D847A16793874704631EF7020C
:10CB30001753FFFFE702A35A79713285328497F0C9
:10CB4000FFFFE780C0462AC6228597F0FFFFE780F7
:10CB50002048B245280897F0FFFFE780606E4561E6
:10CB60001753FFFF6700E35982809797FF1F938752
:10CB7000E7289C43D847A167938787026310F7048F
:10CB80001753FFFFE702A35579713285328497F07E
:10CB9000FFFFE780C0412AC6228597F0FFFFE780AC
:10CBA0000041B2452300A102280897F0FFFFE7806B
:10CBB000206945611753FFFF6700A3548280175314
:10CBC000FFFFE702C351011197F0FFFFE780203E0E
:10CBD000AA85280097F0FFFFE7808066056117535C
:10CBE000FFFF670003529797FF1F938727219C43FE
:10CBF000D847A167D107631FF7001753FFFFE7026C
:10CC0000034E328597000000E780A0FB1753FFFF1B
:10CC10006700234F82809797FF1F9387271E9C43AF
:10CC2000D847A167C507631FF7001753FFFFE70247
:10CC3000034B328597000000E780A0F81753FFFFF1
:10CC40006700234C82809797FF1F9387271B9C4385
:10CC5000D847A167B907631FF7001753FFFFE70223
:10CC60000348328597000000E780A0F51753FFFFC7
:10CC70006700234982809797FF1F938727189C435B
:10CC8000D847A167AD07631FF7001753FFFFE702FF
:10CC90000345328597000000E780A0F21753FFFF9D
:10CCA0006700234682809797FF1F938727159C4331
:10CCB000D84789476318F7021753FFFFE70223425B
:10CCC0000111328532C897F0FFFFE780402EAA8518
:10CCD000280097F0FFFFE780A05605611753FFFF7C
:10CCE0006700234282809797FF1F938727119C43F9
:10CCF000D847A1678D076311F7041753FFFFE702B9
:10CD0000033E01113285328497F0FFFFE780202A2D
:10CD100013066100AA844C00228597300000E7804A
:10CD2000C0232800A68597F0FFFFE78060510561CA
:10CD30001753FFFF6700E33C82809797FF1F93879D
:10CD4000270C9C4381CFDC4391CB1753FFFFE702B5
:10CD5000033982971753FFFF6700A33A8280175366
:10CD6000FFFFE702C33779713C08AE843ED2A1656C
:10CD7000B7070A002A843ED448103C08DD053ED699
:10CD800036C432C63AC297D0FFFFE780402C124724
:10CD90004810BA8597F0FFFFE780C013324648106D
:10CDA000B28597F0FFFFE780E014A2464810B685F1
:10CDB00097F0FFFFE7800012501001478146A685DB
:10CDC000228597D0FFFFE780E04D45611753FFFFB5
:10CDD000670023331753FFFFE702633001117C0024
:10CDE0000329C501AE843ECAA165B70707002A849E
:10CDF0003ECC48087C00C5053ECE97D0FFFFE780BB
:10CE000000258345D900480897F0FFFFE780800C94
:10CE1000500801478146A685228597D0FFFFE7800D
:10CE2000604805611753FFFF6700A32D1753FFFFED
:10CE3000E702E32A83C7950093F7F707A384F50079
:10CE400097000000E78040F91753FFFF6700632B4E
:10CE50001753FFFFE702A32879713C08AE843ED246
:10CE6000A165B70709002A843ED448103C08938581
:10CE700045043ED632C636C497D0FFFFE780201D5A
:10CE8000A2464810B68597F0FFFFE780A00432461F
:10CE90004810B28597F0FFFFE780C00550100147AA
:10CEA0008146A685228597D0FFFFE780A03F456198
:10CEB0001753FFFF6700E3241753FFFFE702232206
:10CEC00083C7950041112A8493F7F707A384F500DF
:10CED00032852EC697F0FFFFE780800F85672AC452
:10CEE0006370F50297700000E78020E92246B245A2
:10CEF00009ED11478146228597000000E78060E632
:10CF000041011753FFFF6700C31F01478346F50127
:10CF1000DDB71753FFFFE702E31A01113C003ECAD9
:10CF2000B7070A003ECC3C003ECE83C79500AA89D5
:10CF3000328593F7F707A384F5002E8497F0FFFF5F
:10CF4000E78000098567637DF504A165AA84938560
:10CF50008504480897D0FFFFE780600F268597700B
:10CF60000000E78080E12A8929E19145480897F08F
:10CF7000FFFFE78020F6A685480897F0FFFFE780CF
:10CF800060F7CA85480897F0FFFFE780A0F40147E3
:10CF900081465008A2854E8597D0FFFFE7808030FC
:10CFA00005611753FFFF670023158145480897F077
:10CFB000FFFFE78020F20349090275BF1753FFFF07
:10CFC000E702431079711C103ECAB7070F003ECC30
:10CFD000404D1C10AA84AE894808994532C636894E
:10CFE0003ECE97D0FFFFE780800632464808B285E4
:10CFF00097F0FFFFE78000EE630C0902A5454808A3
:10D0000097F0FFFFE780C0E62546CA85972001001C
:10D01000E78020A4500801478146CE85268597D019
:10D02000FFFFE780202845611753FFFF6700C30C0F
:10D030008355C402480897F0FFFFE780A0EB035533
:10D04000E402814505C5854785456301F502C16751
:10D05000FD179305F00F630BF5007D159770000029
:10D06000E780208E9305150093F5F50F480897F09B
:10D07000FFFFE78020E683450403480897F0FFFFA1
:10D08000E78040E583451403480897F0FFFFE780F9
:10D0900060E483552403480897F0FFFFE78080E5AC
:10D0A00083554403480897F0FFFFE780A0E49DB74D
:10D0B0001753FFFFE702A30283C79500814601468D
:10D0C00093F7F707A384F50097000000E78040EF8F
:10D0D0001753FFFF6700E3021753FFFFE702230028
:10D0E00079713E841C103ECA2E89B7070F00A165D6
:10D0F0003ECCFD051C10AA84480842C03AC23ECE70
:10D1000036C432C697D0FFFFE78060F43246480845
:10D11000B28597F0FFFFE780E0DBA2464808B685BE
:10D1200097F0FFFFE78000DD12474808BA8597F0C7
:10D13000FFFFE78020DC0248630C080291454808A5
:10D1400097F0FFFFE780C0D21146A285972001002B
:10D15000E7802090500801478146CA85268597D0F0
:10D16000FFFFE780201445611753FFFF670063F955
:10D170008945480897F0FFFFE78080CF8347040088
:10D180002300F50083471400A300F500E1B717530F
:10D19000FFFFE70223F383C7950001112A8A93F763
:10D1A000F707A384F5003285AE8432C697F0FFFFFF
:10D1B000E78000E232462A89328597F0FFFFE78058
:10D1C00000DF85676373F902AA894A8597700000BA
:10D1D000E780A0BA2A8419ED114781464A86A685C0
:10D1E000528597000000E780C0B705611753FFFF25
:10D1F000670083F09387E9FF93F7F70F0547E3662E
:10D20000F7FE8347F50195EB8947E380F9FE8346F6
:10D21000F401528501474A86A68597000000E78001
:10D2200040B4A167D90748083ECC230A010002CECA
:10D2300097000000E780A0B04DBF639EE7008947DC
:10D24000639EF90093071020231FF50097700000DC
:10D25000E780C0B76DBF0947E39BE7FA8D47E398C6
:10D26000F9FA228597700000E78080DF9797FF1F0B
:10D27000938707D89C4399E79797FF1F938707C128
:10D280009C4399C703D5040097800000E780A0CE97
:10D29000231F040022855DBF1753FFFFE70223E42D
:10D2A00001113C003ECAB7070B003ECC3C003ECE0D
:10D2B00083C795002A89328593F7F707A384F50081
:10D2C000AE8497F0FFFFE780A0D093170501C187D8
:10D2D000635AF006A1652A849385E502480897D031
:10D2E000FFFFE780C0D6A285480897F0FFFFE780E0
:10D2F00060C09797FF1F938767B99C43A9EB0144D0
:10D300009375F40F480897F0FFFFE780A0BC935592
:10D31000844093F5F50F480897F0FFFFE78080BB46
:10D320009355044193F5F50F480897F0FFFFE78008
:10D3300060BA014781465008A6854A8597D0FFFF0D
:10D34000E78040F605611753FFFF670083DB416507
:10D3500085460546A2857D1597500000E78060BD93
:10D3600059DD510597000100E780808F13044006C6
:10D370003344850271B71753FFFFE70243D601110B
:10D38000B70706003EC683C7950021642A8993F734
:10D39000F707A384F500AE8428009305A4040AC40B
:10D3A0000AC897D0FFFFE78080CA30000147814656
:10D3B000A6854A8597D0FFFFE780C0EE97E0FFFF84
:10D3C000E780E01113049404480822CC230A0100EA
:10D3D00002CE97000000E780809605611753FFFF9B
:10D3E000670023D21753FFFFE702C3CDC1642A8928
:10D3F00001449799FF1F938929C1130A8002FD14E4
:10D4000097E0FFFFE780E0BD6347A40001451753A5
:10D41000FFFF670063CEB307440303A7C90ABA97A7
:10D4200003D707006306970083D72700638427018B
:10D430000504F9B70545E1BF1753FFFFE70283C8AD
:10D440002A8A2E8999C123A0050081498144979A8F
:10D45000FF1F938A2A9B614B97E0FFFFE780A0BEE6
:10D4600063C7A4004E851753FFFF6700E3C83384EA
:10D47000640383A70A003E948357040099E763047A
:10D480000900232089008504C1BF4146D2851305C8
:10D49000440097100100E780605975F5A289E5B74F
:10D4A0001753FFFFE70203C239717C083ED4B70768
:10D4B0000A003ED67C083ED883C795002A8A32856A
:10D4C00093F7F707A384F5002E8932C697F0FFFF84
:10D4D000E78000B085676373F5083246AA84328519
:10D4E00097F0FFFFE780A0AC8547AA8963E8A7060D
:10D4F000A16593858504281097D0FFFFE78020B5AC
:10D50000268597700000E78040872A8429ED9145A1
:10D51000281097F0FFFFE780E09BA685281097F082
:10D52000FFFFE780209DCE85281097F0FFFFE78062
:10D53000609A014781463010CA85528597D0FFFF17
:10D54000E78040D6A1679387770448183EDC230A1A
:10D55000010202DE97F0FFFFE780607E2161175332
:10D56000FFFF670063B98145281097F0FFFFE78050
:10D570006096A685281097F0FFFFE780A097979701
:10D58000FF1F9387E7DE9C4381CB228563890900D7
:10D5900097D00000E78040248345040271B797D0FC
:10D5A0000000E780C022CDBF1753FFFFE70283B121
:10D5B00083C795004111AA8993F7F707A384F50063
:10D5C0003285AE84328A97F0FFFFE78060A08567DE
:10D5D000637FF5022A8997600000E780007A2A8439
:10D5E000914631C58347F50105476387E70291C737
:10D5F0000D476366F704AD461DA893050503032593
:10D600000A00414697100100E78040420DE94101C0
:10D610001753FFFF670043AE9305950803250A00E3
:10D62000414697100100E7806040814669F54A86CF
:10D63000A6854E8597000000E780C081C9BF83257D
:10D640000A001305940897700000E780A02919C10B
:10D65000C146F1BF9797FF1F938787999C4399E72E
:10D660009797FF1F938787829C4399C7228597804E
:10D670000000E780208A69FD8547A30FF40022851A
:10D6800097B00000E7806084228597600000E78003
:10D69000E0734E8581464A86A68597F0FFFFE780B6
:10D6A000607BA1679387570448003EC423020100B2
:10D6B00002C697F0FFFFE780806891BF1753FFFF16
:10D6C000E702639F83C795004111AA8993F7F70783
:10D6D000A384F50032852E89B28A97F0FFFFE78098
:10D6E000208F85676374F50EAA8497600000E78039
:10D6F000C0682A840DED416B014A979BFF1F938BF5
:10D70000AB90130C400E7D1B19A833048A0383A72A
:10D710000B0B3E948357C40163836705050A97E0AA
:10D72000FFFFE780008BE342AAFE95460DA08357DA
:10D73000C501639697029305050303A50A004146B8
:10D7400097100100E780802E994611E181462686D8
:10D75000CA854E8597F0FFFFE780C06F85A883A537
:10D760000A001305040397700000E780A017C14664
:10D7700079FD2285231E940097A00000E780E074C5
:10D78000228597600000E78060649797FF1F93876A
:10D7900027BE9C43A9C323000402228597D0000022
:10D7A000E78040F04E8581462686CA8597F0FFFFC8
:10D7B000E780406AA1679387070448003EC42302BC
:10D7C000010002C697F0FFFFE78060574101175341
:10D7D000FFFF6700C39189472300F402E1B7397165
:10D7E00006DE22DC4AD8800052D456D25AD026DA3D
:10D7F0004ED65ECE2E8A32892A8B97D0FFFFE780E5
:10D80000407A0605710541998A8A3301A140232295
:10D8100024FC231404FC97D0FFFFE7808078834723
:10D820009A000605350593F7F7072315A4FCA30412
:10D83000FA004A85232624FC97E0FFFFE780407921
:10D8400093170501C1876340F0025681130104FC60
:10D85000F2506254D2544259B259225A925A025B3F
:10D86000F24B21618280AA844A8597E0FFFFE7801E
:10D870002076AA894A8597E0FFFFE7806075A16559
:10D880009385C5022A89130544FC97C0FFFFE780F2
:10D89000007C268597C0FFFFE7804070854511C951
:10D8A0004A86CE8597C0FFFFE780C069AA8B21E931
:10D8B0008945130544FC97E0FFFFE780A061A6853A
:10D8C000130544FC97E0FFFFE780C062CE85130597
:10D8D00044FC97E0FFFFE780E061CA85130544FC44
:10D8E00097E0FFFFE780006101478146130644FC93
:10D8F000D2855A8597D0FFFFE780C09AB9B7814596
:10D90000130544FC97E0FFFFE780C05CA685130584
:10D9100044FC97E0FFFFE780E05DCE85130544FC03
:10D9200097E0FFFFE780005DCA85130544FC97E0A0
:10D93000FFFFE780205C814497D0FFFFE7806066AF
:10D94000E3D4A4FA83A70B0113971400BA9783D5E5
:10D95000070099C5130544FC97E0FFFFE780805955
:10D960008504D9BF797106D622D44AD000184ECE8C
:10D9700052CC56CA26D25AC8AE893289AA8A97D0C2
:10D98000FFFFE78000620605690541990A8A3301B5
:10D99000A140232A24FC231C04FC97D0FFFFE7802E
:10D9A000406083C7990006052D0593F7F707231DEF
:10D9B000A4FCA384F9004A85232E24FC97E0FFFFF2
:10D9C000E780006193170501C187634FF000528122
:10D9D000130104FDB250225492540259F249624A92
:10D9E000D24A424B45618280AA844A8597E0FFFF74
:10D9F000E780005EA1659385A5022A89130544FD91
:10DA000097C0FFFFE780A064268597C0FFFFE780EF
:10DA1000E058854509C9CA8597C0FFFFE780805552
:10DA20002A8B29E18945130544FD97E0FFFFE78034
:10DA3000604AA685130544FD97E0FFFFE780804B11
:10DA4000CA85130544FD97E0FFFFE780A04A014720
:10DA50008146130644FDCE85568597D0FFFFE780AB
:10DA60006084B5B78145130544FD97E0FFFFE7806B
:10DA70006046A685130544FD97E0FFFFE7808047D9
:10DA8000CA85130544FD97E0FFFFE780A046814467
:10DA900097D0FFFFE780E050E3DBA4FA83270B0178
:10DAA00013971400BA9783D5070099C5130544FD51
:10DAB00097E0FFFFE78000448504D9BF1743FFFFCD
:10DAC000E702E36183474500404DD5EFFD575DC454
:10DAD0008346940009476363D70A0346B40085462A
:10DAE00063EEC6088306E40063CA06085C45F9567F
:10DAF0002390D7009787FF1F83C7073199E3A304BB
:10DB0000E4009787FF1F938767389C4381E7894725
:10DB1000A306F4009797FF1F938787859C4381E7AF
:10DB200089472306F4009705000093854506AA84DB
:10DB30001305040197F00000E7802010FD57231A19
:10DB4000F40281471CDC01489787FF1F23AA872A1C
:10DB50009787FF1F9387072B232E040304C080435E
:10DB600097D0FFFFE780204E61463306C50281450E
:10DB700022859740FFFFE780805981473E85174304
:10DB8000FFFF67000358FD57D5BF1743FFFFE702AC
:10DB900003552A840355450297600000E780E01D85
:10DBA00019E5231E04001743FFFF670083558357C1
:10DBB000E401F5DB930504FF17450100130585E338
:10DBC00097E00000E780E014F9BF1743FFFFE7028A
:10DBD00003512E89A16541119385E5032A8436C43A
:10DBE00032C6BE843AC297C0FFFFE7804046124764
:10DBF0002285BA8597E0FFFFE780C02D3246228557
:10DC0000B28597E0FFFFE780E02EA2462285B68529
:10DC100097E0FFFFE780002E63030902914522850C
:10DC200097E0FFFFE780C0241146A685971001000A
:10DC3000E78020E241011743FFFF6700834C8945DD
:10DC4000228597E0FFFFE780A02283C7040023001E
:10DC5000F50083C71400A300F500E9BF1743FFFFD9
:10DC6000E702E34783C79500444D054793F7F7075D
:10DC7000A384F5001C42411183C707006367F706C0
:10DC80002E842A89B1C003C7D400630FF702178717
:10DC9000FF1F1307A71F184305C3A386F40097A00F
:10DCA0000000E780404A83C7D40099E741657D15AD
:10DCB00097400000E780403083D72403918B89C7C9
:10DCC00097E00000E780C0134A85A28597F0FFFF28
:10DCD000E7808010A167C10748003EC4230201000D
:10DCE00002C697F0FFFFE780800541011743FFFF61
:10DCF000670023411743FFFFE702633E03D7450058
:10DD00008D47AA8441112E8432892E8563E3E70270
:10DD100097E0FFFFE780C02BAA8523000900268536
:10DD200097C0FFFFE780002541011743FFFF670011
:10DD3000433D97E0FFFFE780A0292AC6228597E0B0
:10DD4000FFFFE780E028B24585472A862300F900D7
:10DD5000268597C0FFFFE780E01EF9B7397106DE20
:10DD600022DC26DA80004ED652D456D24AD85AD077
:10DD70005ECEAE89B284AA8A97D0FFFFE780602189
:10DD800006051305250241990A8A3301A140232281
:10DD900024FC231404FC97D0FFFFE780801F83C777
:10DDA000990006054D0593F7F7072315A4FCA384F6
:10DDB000F9002685232624FC97E0FFFFE780402119
:10DDC00093170501C1876340F0025281130104FCDF
:10DDD000F2506254D2544259B259225A925A025BBA
:10DDE000F24B21618280AA8B03AB040097C0FFFF36
:10DDF000E780C01A51E583D7440001498544F117F3
:10DE000093B71700A301F4FC834734FCA165C9C78D
:10DE10009385E504130544FC97C0FFFFE7802023AA
:10DE2000A685130544FC97E0FFFFE780A00ADE8586
:10DE3000130544FC97E0FFFFE780C00B834734FCE9
:10DE4000114691E30946DA85130544FC97E0FFFF8C
:10DE5000E78060058144630A0900416B7D1B97D010
:10DE6000FFFFE780001363CCA4020147814613063D
:10DE700044FCCE85568597C0FFFFE780A042B1B72E
:10DE8000A685130634FC97000000E780E0E6933493
:10DE900015002A8986048DBF9385C504A5BF8327F5
:10DEA000C90013971400BA9783D5070063886501EA
:10DEB000130544FC97E0FFFFE780C003850445B7E6
:10DEC0001743FFFFE702231F79711C103EC4B707F9
:10DED0000F003EC61C103EC883C79500AA8A328533
:10DEE00093F7F707A384F500AE89328497E0FFFF2C
:10DEF000E780000E93170501C187635AF0062A8A4E
:10DF0000228597E0FFFFE780A00C2A895285032B2A
:10DF1000040097C0FFFFE780600839ED8357440095
:10DF200081440544F11793B71700A303F10083451B
:10DF30007100DA872287CA8652862800970000007F
:10DF4000E780E0C8014781463000CE85568597C0FE
:10DF5000FFFFE7802035A1679387D70348083ECCB1
:10DF6000230A810026CE97F0FFFFE78040DD456160
:10DF70001743FFFF6700A317A285130671009700E0
:10DF80000000E78060D7AA84094455D13544E300F6
:10DF900055FB4A8597F0FFFFE78000450D4441D9C6
:10DFA000014497D0FFFFE780C0FE634DA400C16B22
:10DFB0000144FD1B97D0FFFFE780A0FD634EA40046
:10DFC0001544B5B7DC4413171400BA9783D707007C
:10DFD000638327030504F1B7D84493171400BA9755
:10DFE00003D70700631B770123902701268597A09D
:10DFF0000000E78080DB01441DBF050465BF1743B7
:10E00000FFFFE702230C83C7950041112A8A93F78B
:10E01000F707A384F50032852E89328497E0FFFF4D
:10E02000E78000FB93170501C1876353F006AA89B7
:10E03000228597E0FFFFE780A0F92311A1004E851C
:10E04000832A040097C0FFFFE78040F539E5835736
:10E05000440085440144F11793B71700A300F10071
:10E060000348110003572100D6875285CE862686A5
:10E07000CA8597F0FFFFE7806006A167F1074800B7
:10E080003EC42302910022C697F0FFFFE78020CB19
:10E0900041011743FFFF67002306A2851306110005
:10E0A00097000000E78040C52A84894455D98357EA
:10E0B000210011678544BA97C2071167C18313070E
:10E0C000F7EFE36FF7F89787FF1F938767F29C439B
:10E0D00081CB85451305210097500000E78020750E
:10E0E000835521002285814497C0FFFFE780A0E18E
:10E0F00025D923100500228597A00000E78040CD98
:10E1000085B71743FFFFE70203FB83C79500411163
:10E110002A8B93F7F707A384F50032852E8A328481
:10E1200097E0FFFFE780C0EA93170501C1876351BD
:10E13000F006AA8A228597E0FFFFE78060E92A8936
:10E140005685832B040097C0FFFFE78020E531E56B
:10E150008357440081440544F11793B71700A30186
:10E16000F10003483100DE875A854A87D686228629
:10E17000D28597F0FFFFE78060F6A167ED074800C2
:10E180003EC42302810026C697F0FFFFE78020BB34
:10E1900041011743FFFF670083F5A2851306310095
:10E1A00097000000E78040B5AA8409445DD99167D3
:10E1B000CA97C2071167C1831307F7EF0544E362EB
:10E1C000F7FACA8597C0FFFFE780E0D3014451F911
:10E1D000814997D0FFFFE780C0DC63DBA900984846
:10E1E00093971900BA9703D7070005EF23902701EB
:10E1F00097D0FFFFE780E0DA1544E384A9F626858F
:10E2000097A00000E780C0BC9787FF1F938747DE79
:10E210009C430144B9D74A8597500000E780C05815
:10E2200089B785097DB71743FFFFE702A3E9797135
:10E230003E847C083EC82E8AB7071400A1653ECAFA
:10E24000E5057C08AA89080836C4428932C6BA8A1C
:10E25000C6843ECC97C0FFFFE78060DFCA85080810
:10E2600097E0FFFFE78000C732460808B28597E0D5
:10E27000FFFFE78020C8A246630A09049D450808FD
:10E2800097E0FFFFE780C0BE1D4681459740FFFF36
:10E29000E780E0E763890A089145080897E0FFFFF7
:10E2A000E78000BD1146A68597000100E780607AEF
:10E2B000100801478146D2854E8597C0FFFFE78051
:10E2C00060FE45611743FFFF670003E3B68508085A
:10E2D00097E0FFFFE78000C21C400808D843935531
:10E2E000C701858912075183B205D98D97E0FFFFD9
:10E2F000E78040C01C40080883C5870097E0FFFF07
:10E30000E78040BD1C40080883C5A70097E0FFFFD9
:10E31000E78040BC1C40080883C5970097E0FFFFDA
:10E32000E78040BB85BF8945080897E0FFFFE7808D
:10E3300020B483C704002300F50083C71400A300A2
:10E34000F500BDB71743FFFFE702C3D783C79500AA
:10E350004111AA8993F7F707A384F5003285AE84AB
:10E36000328497E0FFFFE780A0C693170501C187BD
:10E37000635DF0042A89032A040097C0FFFFE78049
:10E38000E0C119E9835744000548F11793B7170016
:10E39000A307F100814631A81306F100A28597007A
:10E3A0000000E78060951DC51C459DC783D64700CA
:10E3B00001480347F10093078500D2884A86A68565
:10E3C0004E8597000000E78040E641011743FFFFBC
:10E3D000670083D209487DBF1D486DBF1743FFFF0B
:10E3E000E70243CE65715C083EC4B7077B013EC6B9
:10E3F0005C083EC883C795002A8A328593F7F707E1
:10E40000A384F500AE8997E0FFFFE78040BA835709
:10E41000E100E1C78945280097C0FFFFE78020C3DE
:10E420008145280097E0FFFFE780C0AA97C0FFFF63
:10E43000E78000C99787FF1F938787F39C43178462
:10E44000FF1F0344649CAA843334800099C313647F
:10E4500024009787FF1F938767A39C4399C3136486
:10E4600044009787FF1F9387A7B89C4399C3136401
:10E47000840083D504002800014997E0FFFFE7806E
:10E4800060A783D52400280097E0FFFFE78080A6DF
:10E4900083D54400280097E0FFFFE780A0A597D030
:10E4A000FFFFE78000AB93150501C181280097E0CD
:10E4B000FFFFE78020A4A285280097E0FFFFE78008
:10E4C00060A39C446360F902014781463000CE8519
:10E4D000528597C0FFFFE780E0DC59611743FFFFDB
:10E4E000670083C1DC441314490028003E9497E080
:10E4F000FFFFE78060968347440003475400890785
:10E500000607BA978607E36AF5FC835524002800BE
:10E51000814A97E0FFFFE780E09D834544002800A3
:10E5200097E0FFFFE780009B83455400280097E0B9
:10E53000FFFFE780209A8347440063C9FA00814ABD
:10E540008347540063C1FA020509A5BF1C44139711
:10E550005A002800BA9783D50700850A97E0FFFF85
:10E56000E7804099C9BF032BC40093975A00280045
:10E570003E9B83552B00850A97E0FFFFE78080973D
:10E5800083550B00280097E0FFFFE780A0964DBF62
:10E590001743FFFFE702A3B45C4993E717005CC988
:10E5A00097A00000E78020B61743FFFF670063B520
:10E5B0001743FFFFE702A3B22E84814597F0FFFFC8
:10E5C000E780C0E705C583570500FD172310F50058
:10E5D00009C4835725002310F40097000000E7804A
:10E5E00060FB01451743FFFF6700A3B131457DD8AC
:10E5F00023100400C5BF1743FFFFE702A3AC83C786
:10E60000950041112A8A93F7F707A384F500328514
:10E610002E89328497E0FFFFE780809B93170501E6
:10E62000C1876356F006AA89C145228597E0FFFF9E
:10E63000E780A0802A8B4E85832A040097C0FFFFC5
:10E64000E780C09531E98357440023110100054458
:10E65000F11793B71700A300F1008144034811009C
:10E6600003572100D6875285CE862286CA8597F029
:10E67000FFFFE780A0A6A1679387170248003EC46A
:10E680002302810026C697E0FFFFE780406B41012F
:10E690001743FFFF670043A613061100A28597F0FA
:10E6A000FFFFE7806065AA8409E5231101000944A2
:10E6B00075B7930521005A8597000000E78080EF29
:10E6C000835721002A84D9DB9787FF1F93874792BE
:10E6D0009C4381CB85451305210097500000E780BE
:10E6E0000015835521002685314497C0FFFFE78040
:10E6F00080812DD523100500268597900000E780A6
:10E70000206D0144A1BF1743FFFFE702439D411164
:10E710002E896C00AA8402C697F0FFFFE78000D222
:10E720000DC10357050005072310E5009700000001
:10E73000E78040E681473E8541011743FFFF6700C0
:10E74000439C3247954765DBCA8526859730000094
:10E75000E780400DC147E34005FE3244854741460E
:10E760002310F40083570900A685130544002311E4
:10E77000F40097000100E780C02D228545BF1743B4
:10E78000FFFFE702239483C795004111AA8A93F7FC
:10E79000F707A384F5003285AE89328497E0FFFF46
:10E7A000E780008393170501C1876356F0062A8A24
:10E7B000C145228597D0FFFFE7802068AA84528553
:10E7C000032B040097B0FFFFE780407D31E98357BA
:10E7D0004400231101008544F11793B71700A300EB
:10E7E000F10001440348110003572100DA875685E0
:10E7F000D2862686CE8597F0FFFFE780208EA16720
:10E800009387070248003EC42302910022C697E086
:10E81000FFFFE780C05241011743FFFF6700C38D30
:10E82000A2851306110097F0FFFFE780E04C2A84D1
:10E8300009E523110100894475B726859305210058
:10E8400097000000E78060ECAA8449FD8355210011
:10E85000228597B0FFFFE780006B49F5014997C01B
:10E86000FFFFE7800074635DA90018489317190043
:10E87000BA9703D707000DEF035721002390E70055
:10E8800097C0FFFFE780E071630625039777FF1FBE
:10E89000938707769C4399C7035521009750000042
:10E8A000E78080F0228597900000E78060521DBFCE
:10E8B000050975B795443DB705C19307F00F630F80
:10E8C000F500C547630CF5009307F5FF05453315C3
:10E8D000F5004205418182800145828041657D15B8
:10E8E0008280B9E91733FFFFE702637F0345060320
:10E8F000328497000000E78060FC9305803EB305FA
:10E90000B502C205C18181CD0357E402854763F892
:10E91000E7001305040197E00000E78020428357D9
:10E92000E40241677D176385E700FD172317F402B2
:10E930001733FFFF6700E37C82801733FFFFE70296
:10E940008377004283C79500444D0349140093F731
:10E95000F707A384F5008347040022091167336990
:10E96000F900A167B347F90041112A8BAE8A63EC25
:10E97000E70E834724001307C00EB91793F7F70F6C
:10E980006373F71003473400C14763EEE70E834714
:10E9900044001307E00793C707086371F70C834926
:10E9A000840083477400A209B3E9F900856763F71F
:10E9B000F90A034A6400834754004E85220A336AE9
:10E9C000FA0097500000E780403B61C12396240382
:10E9D000834B3400137AFA00239A34032388740398
:10E9E0002399440393890401631C090023A60402AC
:10E9F000239804024E8597E00000E78060363DA032
:10EA0000034924004A8597000000E78020EB239704
:10EA1000A402834744004E85A388F402E38D0BFCD7
:10EA2000E30B09FC97E00000E780202F979000009F
:10EA3000E780007381460146D6855A8597E0FFFF3F
:10EA4000E7800058A167938797033EC42302010023
:10EA5000480002C697E0FFFFE780602E41011733B0
:10EA6000FFFF6700C3688544A2862686D6855A853F
:10EA700097E0FFFFE780C054A167938797033EC4E8
:10EA800023029100F1B7BD44C5B79144F1BF1733DC
:10EA9000FFFFE702236301111C08404D3EC2B70788
:10EAA0000F003EC41C083EC62A89AE8997C0FFFFEE
:10EAB000E78000D7585C1C5C6346B70E6394E500A2
:10EAC00063E2A70E3385A740B3B7A700B305B740ED
:10EAD0001306803E81469D8D97000100E78080B738
:10EAE00093140501C180A1659385C503480097B0C3
:10EAF000FFFFE780C0558145480097D0FFFFE780C2
:10EB0000603D83550404480097D0FFFFE780803EB6
:10EB100083552404480097D0FFFFE780A03D81453E
:10EB200089CCC167FD179305F00F6388F400268533
:10EB300097500000E780E0E0AA85480097D0FFFFEB
:10EB4000E780403903554404814501CDC167FD1775
:10EB50009305F00F6307F50097500000E78060DE33
:10EB6000AA85480097D0FFFFE780C036834564043C
:10EB7000480097D0FFFFE780E035834574044800E4
:10EB800097D0FFFFE7800035500001478146CE85D2
:10EB90004A8597B0FFFFE780E07005611733FFFFFC
:10EBA00067008355814481B71733FFFFE702235382
:10EBB00083C7950093F7F707A384F500970000003B
:10EBC000E78020ED1733FFFF6700A3531733FFFFE4
:10EBD000E702434F83C795004111404D93F7F70774
:10EBE000A384F5002A8A3285B284AE8997D0FFFFCC
:10EBF000E780003E2A8B268597D0FFFFE780403DC7
:10EC00002A89268597D0FFFFE780603A93170B018A
:10EC100063CA0702E177CA97C207C183116763E33A
:10EC2000E70293070910C207C1831307B00F637B84
:10EC3000F70093170901C187AA8A634AF000C54704
:10EC400063FE570141011733FFFF6700E34A97B0A6
:10EC5000FFFFE7802025E31725FFD5B763080B02E8
:10EC600063060902814463890A02B7077F00231003
:10EC70006405231124057CC0568597000000E780B9
:10EC8000E0C39304803EB304950239A0B7077F0028
:10EC9000232004047CC081440355240497E0000031
:10ECA000E780A0A3A1C497C0FFFFE78060B72695C7
:10ECB00093D7F44133379500AE97BA9708DC5CDC04
:10ECC000CE85528597000000E780A0DC99E02322E2
:10ECD0000404A1679387B70348003EC423020100E0
:10ECE00002C697E0FFFFE7808005A9BF8147014882
:10ECF0001CDC232E0403E9B71733FFFFE702233E92
:10ED000097C0FFFFE7802034E1473305F5029145C6
:10ED100097500000E78000C5E55711C59777FF1FA2
:10ED200023A2A70E81473E851733FFFF6700633D8F
:10ED300085471777FF1F2309F70C82801733FFFFE2
:10ED4000E702E3399777FF1F9387870B80433DC026
:10ED5000835704046390A70683572404639CB70475
:10ED60003689B28497C0FFFFE78080AB5C5C63C3E9
:10ED7000B7046395B7001C5C63EEA7028347640485
:10ED800063F3F400A6872303F4048347740463F356
:10ED90009700A687A303F4048357440441677D17B3
:10EDA0006385E70085072312F4043C4481C7CA85C4
:10EDB000268582971733FFFF6700A3349777FF1FDD
:10EDC000938707049C43014599C303C5870082804C
:10EDD0001733FFFFE702A3300111B70707003EC654
:10EDE00083C79500584D0AC493F7F7070AC8A38450
:10EDF000F5002A89AE8411CB1C4283C70700230487
:10EE0000F70097900000E7800034216493055402D6
:10EE1000280097B0FFFFE780802397000000E7807D
:10EE200020FAAA85280097D0FFFFE780A00A3000CB
:10EE300001478146A6854A8597B0FFFFE780804657
:10EE400013044402480822CC230A010002CE97E0B2
:10EE5000FFFFE780C0EE05611733FFFF6700632AFD
:10EE60001733FFFFE702A32701117C003ECAB70753
:10EE700007003ECC7C003ECE83C795002E84AA843A
:10EE800093F7F707A384F500A16593855502480819
:10EE900097B0FFFFE780A01B97000000E78040F2DB
:10EEA000AA85480897D0FFFFE780C00250080147B5
:10EEB0008146A285268597B0FFFFE780A03E0561C9
:10EEC0001733FFFF6700E3239777FF1F938747F30D
:10EED0009C43094599C303C5970082809777FF1F1C
:10EEE000938707F29C43094599C303C5D7008280E5
:10EEF0009777FF1F9387C7F09C43014599C303C5CC
:10EF0000A70082801733FFFFE702C31B0111B70779
:10EF100008003EC683C79500404D0AC493F7F70723
:10EF20000AC8A384F5002A89AE8429C414428547FF
:10EF300003C7060063E0E70A834794000946814956
:10EF40006380C702B307F740A304E400B339F000BD
:10EF500083C716002305F40097900000E780A01EE9
:10EF600003572403058B19C76386090097D0000057
:10EF7000E78000E9216493058402280097B0FFFF31
:10EF8000E780E00C97000000E78040F4AA852800A5
:10EF900097D0FFFFE78000F497000000E78080F53E
:10EFA000AA85280097D0FFFFE780C0F2014781467D
:10EFB0003000A6854A8597B0FFFFE780A02E130496
:10EFC0007402480822CC230A010002CE97E0FFFF1A
:10EFD000E780E0D605611733FFFF6700E3111733C1
:10EFE000FFFFE702C30F01117C003ECAB70708000C
:10EFF0003ECC7C003ECE83C795002E84AA8493F736
:10F00000F707A384F500A16593858502480897B0AA
:10F01000FFFFE780C00397000000E78020EBAA8590
:10F02000480897D0FFFFE780E0EA97000000E780FC
:10F0300060ECAA85480897D0FFFFE780A0E9500858
:10F0400001478146A285268597B0FFFFE78080258E
:10F0500005611733FFFF6700C30A9777FF1F938788
:10F0600027DA9C43014599C303C5B7008280173353
:10F07000FFFFE702C3060111B70707003EC683C7BB
:10F080009500404D0AC493F7F7070AC8A384F5001A
:10F090002A89AE8405C81C42054783C707006368F8
:10F0A000F7060347B400630FF700A305F400979039
:10F0B0000000E78040098347B400B9CF97D0FFFF35
:10F0C000E78040BE21649305B400280097B0FFFF9D
:10F0D000E780E0F797000000E78060F8AA85280045
:10F0E00097D0FFFFE78000DF014781463000A6850B
:10F0F0004A8597B0FFFFE780E01A2904480822CC30
:10F10000230A010002CE97E0FFFFE78040C30561BC
:10F110001733FFFF6700E3FE97D0FFFFE78020BFB4
:10F1200055B71733FFFFE70283FB01117C003ECA8E
:10F13000B70707003ECC7C003ECE83C795002E84E7
:10F14000AA8493F7F707A384F500A165AD054808E5
:10F1500097B0FFFFE780A0EF97000000E78020F066
:10F16000AA85480897D0FFFFE780C0D6500801471E
:10F170008146A285268597B0FFFFE780A012056132
:10F180001733FFFF6700E3F79777FF1F938747C7A2
:10F190009C43094599C303C5C70082801733FFFF0D
:10F1A000E702E3F301117C00AE843ECAA165B70714
:10F1B00007002A843ECCD1057C0048083ECE97B09B
:10F1C000FFFFE780C0E897000000E78020FCAA85E9
:10F1D000480897D0FFFFE780E0CF500801478146FD
:10F1E000A685228597B0FFFFE780C00B0561173326
:10F1F000FFFF670003F11733FFFFE70243EE83C70A
:10F20000950093F7F707A384F50097000000E780C7
:10F2100020F91733FFFF6700C3EE1733FFFFE70244
:10F2200063EA83C795000329C501411193F7F707E6
:10F23000A384F5001C4283C90700854763E63707AE
:10F240009777FF1F9387C7129C432E84AA8485CF8C
:10F2500097000000E78080F389476306F5026304A6
:10F2600009028347C9006380370323063901979059
:10F270000000E78040ED83572903898B89C797D029
:10F280000000E780E0B72685A28597000000E780B0
:10F2900020F1A167CD0748003EC42302010002C649
:10F2A00097E0FFFFE780A0A941011733FFFF670048
:10F2B000A3E49777FF1F9387A7B49C431D4599C389
:10F2C00003C5E70082801733FFFFE70243E1011126
:10F2D000B70707003EC683C79500584D0AC493F789
:10F2E000F7070AC8A384F5002A89AE8415C71C4213
:10F2F00083C7070093968701E18663C406068546A7
:10F300006381D7068346E7006388F6002307F7008A
:10F3100097900000E78020E321649305E400280033
:10F3200097B0FFFFE780A0D297000000E780A0F829
:10F33000AA85280097D0FFFFE780C0B90147814622
:10F340003000A6854A8597B0FFFFE780A0F5350419
:10F35000480822CC230A010002CE97E0FFFFE78095
:10F36000009E05611733FFFF6700A3D91733FFFF26
:10F37000E702E3D601117C003ECAB70707003ECC86
:10F380007C003ECE83C795002E84AA8493F7F707AE
:10F39000A384F500A165B905480897B0FFFFE78091
:10F3A00000CB97000000E78000F1AA85480897D0BD
:10F3B000FFFFE78020B2500801478146A2852685DD
:10F3C00097B0FFFFE78000EE05611733FFFF67008E
:10F3D00043D31733FFFFE702E3CEAA840144177932
:10F3E000FF1F130929A2E14997C0FFFFE780A0C5CD
:10F3F0006344A400014519A8330534038327090099
:10F400003E95835725006397970011051733FFFF3B
:10F41000670083CE0504C9BF032E8500630A0E1260
:10F420001773FF1F1303C3BC0323030063150300FB
:10F4300029436390061203234E01631503001D4305
:10F44000639907101733FFFFE702E3C6C689428AB4
:10F450003E89BA8AB684328BAE8B2A84B5E10355D5
:10F460004E0019E501431A851733FFFF670023C8D3
:10F47000A167A98F116763FBE70097000000E78091
:10F4800080F5814597F0FFFFE780C0120844B70779
:10F4900000E05841F98F18455CC1B707001FF98F8C
:10F4A0001CC55C4991C7610597E00000E780408B6F
:10F4B000E38A09FA228597900000E78060C65DB76D
:10F4C000328597C00000E78040430D4349DD1C446E
:10F4D000116703D54700A167A98F63FBE700970079
:10F4E0000000E78040EF814597F0FFFFE780800C48
:10F4F0000323840093164B01D1828347B300035644
:10F5000063008588FD8BA305F300FD777D8E558E06
:10F51000FD76FD16B204F18E83274301C58E2312BA
:10F5200073012313D3002304530123052301A304F0
:10F530004301BDDF228597B0FFFFE78080C9AA8520
:10F540000844B5D1610597D00000E780207F8DB7D2
:10F550001D431A8582801733FFFFE702A3B60569B2
:10F56000AA84AE89328A0144FD5A7D1997C0FFFFF3
:10F57000E78020A26347A40001451733FFFF67001F
:10F58000A3B7D84493171400BA9703D70700631F93
:10F5900037032390570163070A00268597900000E0
:10F5A000E780A0809C449DC383D76700B3F7270101
:10F5B000639E3701D2880148814701478146014651
:10F5C0008145268597000000E78040E5050479BF66
:10F5D0001733FFFFE70203AF79711C103EC4B70772
:10F5E0000F003EC61C103EC883C79500AA8A32850C
:10F5F00093F7F707A384F5002E89328497D0FFFF95
:10F60000E780009D93170501C187635AF006AA8918
:10F61000228597D0FFFFE780A09B2A8A4E85032B87
:10F62000040097B0FFFFE780609739ED83574400EF
:10F6300081440544F11793B71700A303F1008345F4
:10F640007100DA872287D2864E86280097E0FFFF76
:10F65000E780E057014781463000CA85568597B05C
:10F66000FFFFE78020C4A1679387F70348083ECCDB
:10F67000230A810026CE97D0FFFFE780406C4561CA
:10F680001733FFFF670043A7A2851306710097E0B9
:10F69000FFFFE7806066AA84094455D1528597E050
:10F6A000FFFFE78060D40D4459D90546D2852685F1
:10F6B00097000000E78060EA2A8451B71733FFFF04
:10F6C000E702E3A1835507000346270041112A847E
:10F6D0002E8532C62EC497E0FFFFE780E0D001C937
:10F6E0003246A245228597000000E78000E74101ED
:10F6F0001733FFFF6700E3A01733FFFFE702A39B69
:10F7000083C795004111AA8A93F7F707A384F500F0
:10F710003285AE89328497D0FFFFE780608B9317E4
:10F720000501C1876357F00AC1452A8A228597C01F
:10F73000FFFFE78080702A8D228597D0FFFFE7804A
:10F7400020892A89228597D0FFFFE780408693078A
:10F7500005F893F7F70F1307E007AA8B637BF7060B
:10F76000228597D0FFFFE78080842A8C228597D05E
:10F77000FFFFE780C083AA8C5285032B040097B05B
:10F78000FFFFE780A08139E983574400231101007E
:10F790008144F11793B71700A300F1000544034714
:10F7A000110083562100938784005685DA882288C9
:10F7B0005286CE8597F0FFFFE78020A7A167E90773
:10F7C00048003EC42302810026C697D0FFFFE78091
:10F7D000005741011733FFFF6700639113061100C3
:10F7E000A28597E0FFFFE7802051AA8409E5231155
:10F7F000010009446DB7930521006A8597F0FFFF6A
:10F80000E780A0F02A8441FD835521009356C9006A
:10F810001316490185486688E2875E87858A51828A
:10F82000268597000000E78060BF2A848DBF1733CC
:10F83000FFFFE702438883C7950041112A8B93F7A6
:10F84000F707A384F5003285AE89328497C0FFFFA5
:10F85000E780007893170501C1876352F00A2A8A6E
:10F86000228597C0FFFFE780A076AA8A228597C0ED
:10F87000FFFFE780E0752A89228597C0FFFFE780B8
:10F880000073930705F893F7F70F1307E0072A8C27
:10F890006377F706228597C0FFFFE7804071AA8C47
:10F8A000228597C0FFFFE78080702A8D5285832BC9
:10F8B000040097A0FFFFE780606E39E5835744009E
:10F8C00085440144F11793B71700A301F1000347E2
:10F8D0003100930784005A85DE882688D6865286B2
:10F8E000CE8597F0FFFFE78040948D4748003EC4E7
:10F8F0002302910022C697D0FFFFE78040444101D8
:10F900001723FFFF6700A37EA2851306310097E04F
:10F91000FFFFE780603E2A84894455D99356C90089
:10F920001316490185486A88E6876287858A51826D
:10F93000D68597000000E78060AEAA8449BF1723F0
:10F94000FFFFE70223782A8981440144617A916AA2
:10F95000176BFF1F130BCB6997B0FFFFE780606445
:10F9600063C7A40022851723FFFF6700E37883277E
:10F97000090093991400CE9703D50700330745017A
:10F98000420741836364570305C103270B0019C76E
:10F9900085453E8597400000E78060E983270900A0
:10F9A0000504CE972390070085047DB797000000DB
:10F9B000E78060A2832709000504CE972390070003
:10F9C00065D5814597F0FFFFE780C0BEF1BF1723E3
:10F9D000FFFFE702236F83C7950041112A8A93F73F
:10F9E000F707A384F50032852E89328497C0FFFF84
:10F9F000E780005E93170501C187635AF004AA8966
:10FA0000832A040097A0FFFFE780405931E5835720
:10FA1000440085440144F11793B71700A301F10096
:10FA200003483100D68752850147CE862686CA858F
:10FA300097D0FFFFE780806AA167F50748003EC4C2
:10FA40002302910022C697D0FFFFE780402F41019B
:10FA50001723FFFF6700436AA2851306310097E072
:10FA6000FFFFE78060292A8489445DD99767FF1FDB
:10FA7000938707589C4381CF044997B0FFFFE780E5
:10FA80004052AA85268597400000E78040DA13059A
:10FA9000040197000000E780C0EA228597800000FB
:10FAA000E78000338144ADBF1723FFFFE702A36067
:10FAB00083C795004111AA8A93F7F707A384F5003D
:10FAC0003285AE8932842311010097C0FFFFE780A1
:10FAD000205093170501C1876354F0062A8AC14557
:10FAE000228597C0FFFFE7804035AA8B5285032B04
:10FAF000040097A0FFFFE780604A21E98357440094
:10FB000085440144F11793B71700A300F10003489F
:10FB1000110003572100DA875685D2862686CE85C6
:10FB200097D0FFFFE780805BA1679387270248009B
:10FB30003EC42302910022C697D0FFFFE780202019
:10FB400041011723FFFF6700835AA28513061100A6
:10FB500097E0FFFFE780401A2A8489444DD99767D0
:10FB6000FF1F9387E74898433E8901CF044997B028
:10FB7000FFFFE7800043AA85268597400000E780C5
:10FB800000CB1305040197000000E78080DB97B0ED
:10FB9000FFFFE780004195443DD9930521005E8534
:10FBA00097F0FFFFE78060B6AA8435F11C48035741
:10FBB000210022852390E70097800000E780402104
:10FBC00083270900A9D70355210097400000E7804B
:10FBD000A0BD35BF1723FFFFE702E34D83C79500A4
:10FBE0004111AA8A93F7F707A384F5003285AE89FD
:10FBF000328497C0FFFFE780A03D93170501C187BE
:10FC00006351F0062A8A228597C0FFFFE780403CB7
:10FC10002A895285032B040097A0FFFFE780003854
:10FC200031E58357440085440144F11793B7170029
:10FC3000A301F10003483100DA8756854A87D2864E
:10FC40002686CE8597D0FFFFE7804049A167F90758
:10FC500048003EC42302910022C697D0FFFFE780F0
:10FC6000000E41011723FFFF67006348A2851306BA
:10FC7000310097E0FFFFE78020082A8489445DD99E
:10FC80009167CA97C2071167C1831307F7EF8544CD
:10FC9000E362F7FA9767FF1F938787359843BE8B18
:10FCA00001CF044997B0FFFFE780A02FAA852685E2
:10FCB00097400000E780A0B71305040197000000FB
:10FCC000E78020C897B0FFFFE780A02D95443DD185
:10FCD0001C48228581442390270197800000E780FB
:10FCE000200F83A70B00B9D74A8597400000E78013
:10FCF000A0AB89B71723FFFFE702633E2A844105C3
:10FD0000B28497000000E780C0C311C522859780A8
:10FD10000000E780E00B81460146A685228597809A
:10FD20000000E780C04E1C4C89C7DC4799C3228580
:10FD300082971723FFFF6700C33C9767FF1F9387D6
:10FD4000270C9C43014599C313850701828097675F
:10FD5000FF1F9387E70A884382801723FFFFE7028C
:10FD600003389317C600DD8DC2054111C1812A8475
:10FD700032C697C0FFFFE780E01732462285118226
:10FD80009375F60F97C0FFFFE780C014410117235A
:10FD9000FFFF670003371723FFFFE702A3327971E4
:10FDA0003C083ED2B7070C003ED43C083ED683C781
:10FDB0009500AE842A8993F7F707A384F500A1651F
:10FDC00093853504481097A0FFFFE7804028C16560
:10FDD000FD150144176AFF1F130A0A23930A400EF8
:10FDE000AE892E8B2EC697B0FFFFE780801E42059E
:10FDF000931704014181C183B24563E9A702C1673A
:10FE0000FD176387F500481097C0FFFFE780800E5D
:10FE1000501001478146A6854A8597A0FFFFE780DD
:10FE2000604845611723FFFF6700032D3307540324
:10FE300083270A0BBA9703D6C701630A3601638A80
:10FE40003501481097000000E78060F1DA8505046D
:10FE500051BFB285EDBF1723FFFFE702C3257971BC
:10FE60007C083EC8B70711003ECA7C083ECC83C759
:10FE70009500AA89328593F7F707A384F5002E89A8
:10FE800097C0FFFFE780C01485676378F504A1651C
:10FE9000AA848905080897A0FFFFE780401B2685F4
:10FEA00097400000E78060ED133415000A04A28536
:10FEB000080897C0FFFFE780E001A685080897C003
:10FEC000FFFFE780200325CC014781461008CA8543
:10FED0004E8597A0FFFFE780E03C45611723FFFFB9
:10FEE0006700E320B30754030327CA0ABA9703D76E
:10FEF0000700631C970003D6270063806505080888
:10FF000097000000E780A0E5DE8505042EC697B0C7
:10FF1000FFFFE780000D4205931704014181C18373
:10FF2000B245E3E1A7FCC167FD17E38FF5F80808C8
:10FF300097C0FFFFE78000FC41BFB285F9B7C165FC
:10FF4000FD150144176AFF1F130A0A0C930A800269
:10FF50002E8BAE8B65BF1723FFFFE70243181841B6
:10FF60008347170083460700A207D58FD207D183A6
:10FF70002390F50083472700034717008D45A2070C
:10FF8000D98F91832310F60097C0FFFFE780A0E987
:10FF90001723FFFF6700E3161723FFFFE702831213
:10FFA000C16401441769FF1F130909069309800200
:10FFB000FD1497B0FFFFE780C0026347A40001452E
:10FFC0001723FFFF67004313330534038327C90A50
:10FFD0003E9583570500E38597FE0504D9BF172397
:10FFE000FFFFE702230E2A8AAE89B284B68A9740C1
:10FFF0000000E78080D819E591473E851723FFFF71
:020000040001F9
:100000006700830F2A894E8597C00000E780E08E45
:100010002A84638E0A048D476DD103570500C547B6
:10002000E31D47FD0347F9018546AD47E317D7FCBC
:100030008347450081CF4146A6855D0597F00000C6
:10004000E780C09E814755D9AD4745BF130965017B
:100050002302E500CA85268597100000E7806062CC
:1000600031C1A547E38B0AF82302040079B705C123
:1000700083570500E39247F94146A685190597F095
:100080000000E780A09A81472DD99947BDB74E85DA
:1000900097000000E78080F02A84954739DD130936
:1000A00055004DBF4146A68523104401231134015C
:1000B0001305190097F00000E780A099228597802A
:1000C0000000E780A0EA81470DBF1723FFFFE7028A
:1000D000030179717C003ECCB7070A003ECE7C005C
:1000E0003ED083C79500B2842E8493F7F707A3848C
:1000F000F5001306A1002A892C0026859700000030
:10010000E780A0E5A16528088D0597A0FFFFE7809F
:1001100000F490408355A100035581008546970067
:100120000000E78000ECAA84AA85280897C0FFFF9A
:10013000E78040DA0356A100835581002808970024
:100140000000E780C0C1300801478146A2854A858A
:1001500097A0FFFFE7800015854748103ED4230293
:10016000910202D697D0FFFFE78060BD456117235B
:10017000FFFF670003F91723FFFFE70243F67971DA
:100180007C003ECCB7070A003ECE7C003ED083C741
:100190009500B2842E8493F7F707A384F500130625
:1001A000A1002A892C00268597000000E780E0DA6C
:1001B000A16528088D0597A0FFFFE78040E99040E2
:1001C0008355A10003558100814697000000E78018
:1001D00040E1AA84AA85280897C0FFFFE78080CF66
:1001E0000356A10083558100280897000000E7808E
:1001F00000B7300801478146A2854A8597A0FFFFD6
:10020000E780400A48102302910202D402D697D018
:10021000FFFFE780C0B245611723FFFF670063EE71
:100220001723FFFFE702A3EB97000000E78060DBE6
:100230001723FFFF6700E3EC9767FF1F938787BCD7
:10024000884382801723FFFFE70263E98357250075
:100250004111AE842A842307B10017F5FFFF13056F
:1002600025466C002316F10097A0FFFFE78080452C
:1002700091C4228597800000E780E0D6FD572310C7
:10028000F400130620028145130554009720FFFF58
:10029000E780E0E741011723FFFF670083E61723AC
:1002A000FFFFE70223E279717C003ECCB7070A002A
:1002B0003ECE7C003ED083C79500AA89AE8493F7DA
:1002C000F7073285A384F5001306A1002C009700E0
:1002D0000000E78080C8035581001144974000006A
:1002E000E780A0A915C50355A100014497B00000FF
:1002F000E780A06011CD0357050083578100454476
:100300006318F700854597000000E780E0F301449B
:10031000216993053900280897A0FFFFE78020D3C3
:10032000A285280897C0FFFFE780C0BA0356A10046
:1003300083558100280897000000E78040A230081C
:1003400001478146A6854E8597A0FFFFE78080F58F
:1003500048104AD42302810202D697D0FFFFE780DB
:10036000009E45611723FFFF670003D91723FFFF96
:10037000E70243D59767FF1F938787A82A8488439E
:100380002E8915C5035745038357C4016311F7022E
:100390002326050223180502410597D00000E780B7
:1003A000209C6306090097800000E78060DB8144A1
:1003B0009769FF1F938949C5130A800297B0FFFF11
:1003C000E78020C263C4A4049767FF1F938707AC2C
:1003D0009C4399C70355C40197200000E780C0BD26
:1003E00063070900228597800000E780C0A01306FC
:1003F000400E814522859720FFFFE78040D1FD57C1
:10040000231EF4001723FFFF670003CF3385440347
:1004100083A7C90A3E95035705008357C401631794
:10042000F700CA8597000000E78000E2850479B7ED
:100430001723FFFFE70203C983C795004111AA896B
:1004400093F7F707A384F5003285AE8497C0FFFFCA
:10045000E78000B885676378F5042A899740000033
:10046000E780A091014401CD83D704003144638823
:100470002701854597000000E78080EF01444E8505
:10048000A2864A86A68597D0FFFFE780A09CA16739
:100490009387170448003EC42302810002C697D008
:1004A000FFFFE780C08941011723FFFF6700C3C436
:1004B0001723FFFFE70203C19767FF1F9387479446
:1004C000804329C4014597C00000E780002181478F
:1004D0000148C1641CDC232E040323200404176993
:1004E000FF1F130969B201449309400EFD1497B030
:1004F000FFFFE78000AE634FA400814517F5FFFFC3
:100500001305857F97A0FFFFE780C01B1723FFFF20
:10051000670083BE330534038327090B3E95835759
:10052000C50163879700854597000000E78040E498
:10053000050475BF9357050113D78700A380F50005
:1005400093170501C183A1832380E5002381F50072
:10055000A381A50082801723FFFFE70243B8230091
:10056000050083C71500A300F50083C725002301FC
:10057000F50083C73500A301F50083C745002302BA
:10058000F50083C75500A302F50083C765009305F6
:100590009500A30305002303F5002304050032851D
:1005A00097000000E78040F91723FFFF670063B55D
:1005B0001723FFFFE70203B14111E9540DCD85CDAB
:1005C00093F9C5FF2E842A89AA84338AA900B7EA41
:1005D000040063189A020D88854411CCB7E7040023
:1005E0009C5F82972AC622866C003305390197E00A
:1005F0000000E7800046268541011723FFFF6700C2
:10060000A3AF83A78A039104829793170501C1833F
:10061000A183A38EF4FE93570501238FF4FEA183DB
:10062000238EA4FEA38FF4FE6DB763E6D5021723D5
:10063000FFFFE702C3AAB28741113686BE8536C6E0
:1006400097E00000E780E040B2464101368517237D
:10065000FFFF670003AB81463685828083870500F4
:100660001387F5003D05FD8793F77708834607005C
:100670007D158606B58FA300F5006307B7007D17CB
:10068000834717009D83DDB782801723FFFFE702B2
:1006900003A5B7E7040083A7070932872A863A85AE
:1006A0008297133515001723FFFF670083A515C137
:1006B00081478DC11723FFFFE70263A2414697E000
:1006C0000000E780003985473E851723FFFF67005C
:1006D00043A381473E8582801DCD1723FFFFE7029C
:1006E00003A0414681452A849720FFFFE78020A28E
:1006F00041468145130504039720FFFFE78020A1B1
:100700000147C1672322040438C87CC80545172364
:10071000FFFF6700039F0145828081473DCDB5CD36
:100720001723FFFFE702A39BB2842E8913068005DF
:1007300081452A849720FFFFE780609DCA8524C4F5
:10074000268597000000E780C0F641468145228556
:100750009720FFFFE780A09B3044A2852285970069
:100760000000E780C0F293040401A285268597006B
:100770000000E780E0EEA685130504029700000064
:10078000E78000EE228597000000E78020F585478E
:100790003E851723FFFF6700C3963E85828017239F
:1007A000FFFFE70223924111E9540DCD85CD93F966
:1007B000C5FF2E842A89AA84338AA900B7EA0400D7
:1007C000639844030D88814411CCB7E704009C5F13
:1007D00082972AC622866C003305390197E0000013
:1007E000E7802027268541011723FFFF6700C3907C
:1007F00083A78A039104829793170501C183A1837C
:10080000A38EF4FE93570501238FF4FEA183238E5C
:10081000A4FEA38FF4FE6DB765CD1723FFFFE7029B
:10082000638AB28411E605451723FFFF6700C38C76
:100830002A842E890145EDD93C487848B3E6E70083
:10084000E5D69386F7FFB3B7F6007D17032A440475
:10085000BA9734C87CC863050A06C14913050A0360
:10086000B38949412295637D3601B2862E86A685DD
:1008700097000000E780A0DB7C40BE9464C065B7B1
:10088000CE862E86CE8597000000E78040DAC11420
:10089000D2944E9923220404A2879306040103C72D
:1008A000070003C607038507318FA38FE7FEE39890
:1008B000F6FE3044A285228597000000E78020DD07
:1008C0002699C1493306994063EC9900A9DCA686B4
:1008D000A6851305040397000000E78040D579BF83
:1008E0008147B306F4003307F6000347070083C5CA
:1008F000060085072D8F2380E600E39437FF304400
:10090000A285228597000000E78060D8C1145DBFF2
:10091000014582800DC11713FFFFE702437C1306D8
:10092000800581459710FFFFE780607E054517131E
:10093000FFFF6700037D01458280814749C5C1C52E
:100940001713FFFFE702A379FC4141462E84AA84D6
:100950006399C70413860501A2878146C14503C771
:10096000070003C507038507298F3305D600034514
:1009700005008506298FA38FE7FEE392B6FE30447B
:10098000A285268597000000E78060D02285970029
:100990000000E78060F885473E851713FFFF67007A
:1009A0004376138507031D8E814522959710FFFF1F
:1009B000E780E0757C40130700F813060402A29755
:1009C0002388E70251BF3E8582801713FFFFE702AD
:1009D00003716D712E84B284AA8590102800368927
:1009E00097000000E780A0D309EDD55725A050401F
:1009F0000C40280097000000E78040E27DD5FD1400
:100A00002104F5F42C004A8597000000E78020F3CC
:100A1000814761DD3E8551611713FFFF6700636EFB
:100A20001713FFFFE702A36B41112EC432C62C003F
:100A3000054697000000E78080F941011713FFFF8A
:100A40006700236C1713FFFFE702636901112A8413
:100A50002EC602C802CA02CC02CE97E00000E78090
:100A6000C023B2462A86A285080897000000E780C6
:100A700060FB1375F50F05611713FFFF67006368CF
:100A80001713FFFFE702A3657971B2872A84214615
:100A90002308B10013051101BE853AC436C697E09C
:100AA0000000E78000FBB246930591013685970070
:100AB0000000E78060A82285141035460C089700D6
:100AC0000000E78020F62A84224701E921460C1025
:100AD0003A8597E00000E780C0F72285456117134B
:100AE000FFFF670003621713FFFFE702435F7171A7
:100AF000AE84AA850A85328497000000E78060BB37
:100B000011C90A86A685228597000000E78020B8D3
:100B1000814711E1C5473E854D611713FFFF67000F
:100B2000435E1713FFFFE70283581D712A8AB289BB
:100B3000BE8435468547130511012E8CB68A3A8B43
:100B4000C28C468D2308F10097E00000E78060F03A
:100B500010100C085285231F010097000000E78049
:100B6000C0F82A843DEDA1476313FD089307900563
:100B700091E0E5473546E2851305110113990A0115
:100B80002308F1001359090197E00000E78060ECA9
:100B90001357890093978A00D98F90080C085285C3
:100BA000231FF10097000000E78020F42A8415E954
:100BB000A1E49387FA0091831379F9003EC6631389
:100BC00009004149668B8144C14B854DB247639F03
:100BD000970C6A868C0033855C0197E00000E78003
:100BE00040E7228525611713FFFF67000350930735
:100BF0009004C9F0A547BDBF834701050947C14B14
:100C00002308F10083471105A58FA308F1009387FE
:100C10002400814463E1FB04014714083386E600A5
:100C20008C08B386E400BA95DA9683C6060083C5BD
:100C300005000507AD8E2300D600E390E7FE41478F
:100C4000639CE70490080C08528597000000E78039
:100C5000C0E925D181A0B3069B00BA871008B3056F
:100C6000F60090083E9603C5060003460600850779
:100C70008506298E2380C500E39277FF998F90081F
:100C80000C085285BE9497000000E78000E6894773
:100C9000014749D12A84B1B790083E960346060021
:100CA0001408BE962380C600850759BFB247850445
:100CB0006387971481471808B306F70098083E9792
:100CC0003386F90003470700034606008507318F86
:100CD0002380E600E39177FF90080C085285970087
:100CE0000000E78080E05DF53546E28513051101DF
:100CF0002308B10197E00000E780A0D51397040115
:100D00004183939784002183D98F10180C08528552
:100D1000231FF10097000000E78020DD25FD8147BB
:100D200010183387F9003E96034707000346060074
:100D3000B306FB008507318F2380E600E39277FF3F
:100D400065A81808B306F70098083E973386F9009F
:100D500003470700034606008507318F2380E6001E
:100D6000E3E127FFCA87639E770990080C08528544
:100D700097000000E78060D711FD81479800B30617
:100D8000F700900818103E973E9603470700034669
:100D900006008507318F2380E600E39177FF354613
:100DA000E285130511012308B10197E00000E780F7
:100DB00040CA139704014183939784002183D98FFC
:100DC00010180C085285231FF10097000000E780DF
:100DD000C0D1E31105EC814710183387F9003E9626
:100DE0000347070003460600B306FB008507318F63
:100DF0002380E600E3E227FFC109410BC1BB814725
:100E000085B79408BE9683C6060018083E9723004F
:100E1000D700850789BF638006321713FFFFE702FB
:100E2000032959712A84BE89B28B8547354613053B
:100E300011022E8B468C4289BA8A368A2300F1022F
:100E400097E00000E780E0C010180C1022852317FF
:100E5000010297000000E78040C963180512A1470E
:100E6000631FFC069307900563930900E547354629
:100E7000DA851305110293140A012300F102C180DF
:100E800097E00000E780E0BC93178A0013D7840046
:100E9000D98F90080C1022852317F10297000000CB
:100EA000E780A0C47DE1639209049307FA00BD883E
:100EB000918391E0C144C207C183DE8C814A3EC662
:100EC000414DB24763E2FA0E6286B3854B0188104A
:100ED00097E00000E78080B54DC93D557DA09307A0
:100EE0009004E39609F8A54759B7834701050947D8
:100EF000C14C2300F10283471105B3C7F900A300D9
:100F0000F10293872900814963E1FC0481461810AE
:100F10003306D7008C083387D900B6955697034718
:100F2000070083C5050085062D8F2300E600E390AA
:100F3000D7FE41476390E70690080C102285970082
:100F40000000E78080BA35D189A0B3863A01BA871C
:100F50001010B305F60090083E9603C50600034640
:100F6000060085078506298E2380C500E39297FF3A
:100F70003387EC4090080C102285BA999700000046
:100F8000E780A0B68947014741D165611713FFFF8C
:100F90006700A31590083E96034606001410BE96FF
:100FA0002380C600850779B7B247850A93990A015D
:100FB000939D8A0093D909016391570F8547354660
:100FC000DA85130511022300F10293D9890097E015
:100FD0000000E78000A8B3ED3D0190000C102285D1
:100FE0002317B10397000000E78020B059FD814727
:100FF000A68963EA970626860C084A8597E00000D2
:10100000E78020A581471810B306F700100898085C
:101010003E973E9603470700034606008507318F3B
:101020002380E600E3E197FE639FA90590080C107A
:10103000228597000000E78040AB21F98147981096
:10104000B306F700900818183E973E96034707002E
:10105000034606008507318F2380E600E391A7FF52
:101060004109C10CB9BD18089000B306F7003E96BF
:101070003387FC0003470700034606008507318FCE
:101080002380E600B5B798084E97034707001C1069
:10109000CE972380E700850941BF85473546DA852D
:1010A000130511022300F10293D9890097E0000093
:1010B000E780209AB3ED3D0190000C1022852317A4
:1010C000B10397000000E78040A2E31005EC8147E0
:1010D00018089000B306F7003E963387FC000347DC
:1010E0000700034606008507318F2380E600E39161
:1010F000A7FF41460C084A8597E00000E78060950D
:1011000081471810B306F700100898083E973E96DE
:1011100003470700034606008507318F2380E6005A
:10112000E391A7FF90080C10228597000000E7804C
:10113000C09B1DD599BD7D5582801713FFFFE70227
:1011400003FA01112A842E8593055100328902C0C9
:1011500002C202C402C69304740097F0FFFFE78046
:10116000A03D1D46A6851305910097E00000E7808D
:10117000408E10088A854A8597000000E780E09637
:1011800019ED93071400180883C6070003460700EB
:1011900085070507B18EA38FD7FEE397F4FE05619F
:1011A0001713FFFF6700E3F51713FFFFE70283F153
:1011B0002E848C414111AA8983871500328991447C
:1011C00063D30700A1449757FF1F9387671A9C4377
:1011D000A1C7C1CA8D472310F10083C725004A85E6
:1011E0002301F10083C73500A301F10083C7450047
:1011F0002302F10083C75500A302F10083C76500F5
:1012000093059100A30301002303F10023040100CF
:1012100097F0FFFFE78040320C404A860A8597F03E
:10122000FFFFE78080330328040083564400A6882C
:101230001D0881470147E51642868A854E8597003D
:101240000000E780408E2A8919E5A685228597B09F
:10125000FFFFE780E0C14A8541011713FFFF6700E8
:10126000A3E94A860A8597F0FFFFE780002F6DB754
:101270001713FFFFE70203E52E848C414111AA8971
:10128000838715003289914463D30700A14497579F
:10129000FF1F9387E70D9C43A1C7C1C68D4723104D
:1012A000F10083C725004A852301F10083C735007B
:1012B000A301F10083C745002302F10083C7550055
:1012C000A302F10083C7650093059100A303010009
:1012D0002303F1002304010097F0FFFFE780C025FE
:1012E0000C404A860A8597F0FFFFE7800027835667
:1012F0004400032804008A85858EC2061D08C18229
:101300002312D400A68881470147E51642864E8500
:1013100097000000E78060B041011713FFFF6700EE
:10132000A3DD4A860A8597F0FFFFE78000234DBFC3
:101330001713FFFFE702A3DAB335B00001118505EB
:101340002A891315F601336515012308B1009305A9
:10135000110136843AC632C03EC442C297F0FFFF44
:10136000E780801DA2471248425593D68700230B81
:10137000F1009305910193578800A30AD100A30BB4
:10138000F100230C010197F0FFFFE780E01A3247DC
:10139000024603280400B337E00083564400920756
:1013A000914411C2A1444A85A68842860C0897F050
:1013B000FFFFE78040772A8919E5A685228597B047
:1013C000FFFFE780E0AA4A8505611713FFFF67006A
:1013D00043D31713FFFFE702E3CE01113EC6864752
:1013E000B335B0008505AA891315F6015D8D230874
:1013F000B1009305110136843A89B28442C446C2D1
:1014000097F0FFFFE7804013224892481645935714
:101410008800A30AF1009305910193D78800230B5C
:101420000101A30BF100230C110197F0FFFFE780EE
:10143000A0103247104083564400B337E0009207B3
:1014400003280900914891C0A1480C084E859700D7
:101450000000E780809CAA8401E9835544004A8506
:1014600097B0FFFFE780C0A0268505611713FFFF37
:10147000670083C8AA959307F00F170701001307A9
:10148000E75A6317B50013C5F7FF1375F50F828090
:1014900005058346F5FFB58FBA9783C70700D5B713
:1014A0000357450014419307F00F17060100130678
:1014B000E657369742074183139506014181631B26
:1014C000E500AD8FB29703C50700130515F313357B
:1014D00015008280850603C5F6FFA98FB29783C7E2
:1014E0000700D9BF1713FFFFE70263BFB287368437
:1014F0002E86BA86AA853E85BA8497F0FFFFE780DC
:101500006052634F0500228597D00000E780E078A5
:101510002A86A686A285268597F0FFFFE780805061
:101520001713FFFF6700E3BD1713FFFFE70283B93F
:101530005D712A8BAE8A170501001305A54C2C009E
:10154000B284368ABA893E8997F0FFFFE780C04FA0
:101550002A845DE134104146DA85280097F0FFFFC8
:10156000E780404C2A8449E98547A303F100A6C2DD
:10157000930771002408BEC4A68685470D462C1823
:10158000281002DC02DED6C0BEC697F0FFFFE7805F
:1015900000442A8435E183477102A6860D4693F7FD
:1015A000F7072300FA00C1473EDE2C1889472810B0
:1015B00026DCA303F10097F0FFFFE78040412A8477
:1015C00005ED4146A6854E8597D00000E78060482E
:1015D0008D47A6860D462C182810A303F10097F01E
:1015E000FFFFE780C03E2A8401E94146A6854A857F
:1015F00097D00000E780E045228561611713FFFF67
:10160000670083AF1713FFFFE70263AD97F7000092
:101610009387C7A0984383C7470079712A89AE840E
:10162000170501001305853E0C083AC42306F10096
:1016300097F0FFFFE78040412A8405ED14104146F2
:10164000CA85080897F0FFFFE780C03D2A8415E1AE
:10165000140815462C00081097F0FFFFE780803C27
:101660002A8401E921462C08268597D00000E780CE
:10167000403E228545611713FFFF670083A81713BB
:10168000FFFFE702C3A597F70000938727999C47C0
:101690007971AA842E84170501001305A5370C085B
:1016A0003EC697F0FFFFE780203A0DE9141041464F
:1016B000A685080897F0FFFFE780C03605E114080B
:1016C00011466C00081097F0FFFFE780A03519E580
:1016D0008347F10193F7F7032300F40045611713E3
:1016E000FFFF670003A21713FFFFE702439F36883F
:1016F000A14881470147E54697F0FFFFE780A042F8
:101700001713FFFF6700E39F1713FFFFE702239DF7
:101710003688A14881470147E54697F0FFFFE780FB
:10172000C06F1713FFFF6700C39D1713FFFFE7028A
:10173000039B01112A842E850C0832C697F0FFFF07
:10174000E780803009ED3247970601009386062B2B
:101750001008C145228597000000E780E0D80561A8
:101760001713FFFF6700E3991713FFFFE7022397A3
:101770004111C1472EC032C48A8509463EC23EC6C9
:1017800097F0FFFFE780A02441011713FFFF6700D8
:1017900043971713FFFFE70283944111AE861306A8
:1017A0001009AA850A8502C002C202C402C697F0C7
:1017B000FFFFE780202741011713FFFF67006394B5
:1017C0001713FFFFE702A391328797060100938664
:1017D000E6242E869305000297000000E780C0D023
:1017E0001713FFFF6700E3911713FFFFE702238F33
:1017F0007971C1472ACC2ED032D42C080D4628004E
:101800003ECE3ED23ED602C402C602C802CA97F0FD
:10181000FFFFE780C01B45611713FFFF6700638E62
:101820001713FFFFE702A38B0111AA842E8417056B
:1018300001001305251F8A8597F0FFFFE780C02070
:1018400015E514084146A6850A8597F0FFFFE78055
:10185000601D09ED8347E1010347F101A207D98F1C
:10186000CA07C9836177D98F2310F4000561171364
:10187000FFFF6700038915CD1713FFFFE7022386DB
:101880009747FF1F9387875C90439745FF1F93857A
:10189000255C1745FF1F1305655797D00000E780AB
:1018A00000C51745FF1F130565561713FFFF670097
:1018B00043851745FF1F1305655582808DCD17138E
:1018C000FFFFE702C3819747FF1F93872758944381
:1018D00001112E840A869745FF1F9385655797D07F
:1018E0000000E78040C60A85029401450561171390
:1018F000FFFF670003817D5582801703FFFFE7022A
:10190000037E97D00000E78080D19747FF1F23AF69
:10191000A75217F5FFFF1305E5C997B00000E78050
:10192000C0741703FFFF6700C37D1747FF1F13072E
:1019300027549317150008433E95FD572310F500D3
:1019400082801703FFFFE70283792A84084009E5B4
:101950001703FFFF6700E37A1C4158401CC0631364
:10196000E5005CC08347550023200500F99BA302D6
:10197000F50097A0FFFFE780207CC9BF1703FFFF9A
:10198000E70243749747FF1F9387875098432A8441
:1019900011CB8347350093F7070289C7035505002C
:1019A000894502971305440197B00000E780403B4A
:1019B000835504000355E40097300000E780A00C35
:1019C000485819C597A0FFFFE7800077232A040233
:1019D0001305840397000000E780E0F68144B149D5
:1019E0009790FFFFE780206A63CBA402834734000F
:1019F0002320040493F727FCA301F40000489790E8
:101A0000FFFFE78040691316150081452285970086
:101A1000FFFFE780C06F1703FFFF6700E36DB38729
:101A200034030329040385043E994A859700000086
:101A3000E78060F12304090065B78347350093F719
:101A4000070299E3014582808357E500E39CB7FED6
:101A5000C167FD176316F60005458280054599A804
:101A60001703FFFFE702A36793170601C187B2843C
:101A70002A8401496359F002835705009DCB014533
:101A80006367F600034584003E953325A600137571
:101A9000F50F0DA01C4813171900BA9783D707003C
:101AA000E38E97FA05099790FFFFE780C05EE34356
:101AB000A9FE01451703FFFF6700A3641703FFFF9B
:101AC000E7024360AE89AA849790FFFFE7806052E7
:101AD0002A8497D0FFFFE780A02EAA86014713062D
:101AE000840197050000938585E41745FF1F1305C2
:101AF00065389790FFFFE780E0182A8925C98C4454
:101B00001304C50022859E0593F5050897A0FFFFE5
:101B1000E780403CCC4083877400E18163DD0704AB
:101B200093E50508228597A0FFFFE780A03A0D46C0
:101B300093854400228597A0FFFFE780C03683D5B8
:101B40000400228597A0FFFFE780E03D83D52400B5
:101B5000228597A0FFFFE780003D03D6490083A5BB
:101B60000900228597A0FFFFE780E0334A8517032D
:101B7000FFFF6700635893F5F5076DB71703FFFF85
:101B8000E702E35501112A84328532C697A0FFFF90
:101B9000E780E0279780FFFFE780C030835704008D
:101BA0001747FF1F130747463246231BF1009307D1
:101BB00000F8A30DF1001C471843231AA1008983E4
:101BC000858BB307F740B28548083ECE231C010041
:101BD000230D010097000000E78080EE05611703E8
:101BE000FFFF670003521703FFFFE702A34D004109
:101BF00001453DC49304C40026853289AE8997A06F
:101C0000FFFFE780C02495452A8A2685035B0401EF
:101C100097A0FFFFE7802021268597A0FFFFE780A0
:101C2000603E8D45AA8A268597A0FFFFE780A01F0A
:101C3000268597A0FFFFE780E03C5C48420A135AE4
:101C40000A01D2975CC423186401814763983A0162
:101C500046054D81330625419337160013F5F70FDE
:101C60001703FFFF670043491703FFFFE702A34481
:101C700089692A8BAE8B328AB68A81440144314C01
:101C8000FD199790FFFFE780004063CDA400979077
:101C9000FFFFE7804042018D33B5AA001703FFFF25
:101CA0006700E3443389840383270B003E9963175D
:101CB0000A008347890085043E94E1B703560A0071
:101CC000DE854A8533F6C90097000000E780E0F121
:101CD0006DD10545E1B71703FFFFE702434001114E
:101CE0002A847C000355E5003ECAB70707003ECCB6
:101CF0007C003ECE97200000E78020082A89854599
:101D0000480897A0FFFFE78020399945480897A029
:101D1000FFFFE780E015AA844A8597200000E7804E
:101D2000A0082380A4009747FF1F9387E72D9C43BB
:101D30004166130606F09396870113D78701558FE6
:101D400093D68700F18E558FA207B706FF00F58F57
:101D5000D98F11462C00138514003EC497D0000083
:101D6000E78020CF5008A382040089452285970090
:101D70000000E780E0E019C9AA851305840397A055
:101D8000FFFFE780E0313C4085073CC00561170359
:101D9000FFFF670003371703FFFFE7024334979005
:101DA000FFFFE78040312A8405049790FFFFE7801A
:101DB000802F3305A402F14791453305F5029720A2
:101DC0000000E78020BA11E565551703FFFF6700A3
:101DD00043339747FF1F23A5A70A9790FFFFE7808C
:101DE000802D2A8405049790FFFFE780C02B3305E0
:101DF000A4028945060597200000E780A0B669D5B2
:101E00009747FF1F23A6A7069790FFFFE780A02A0A
:101E10002A8405049790FFFFE780E0283304A4029A
:101E20009747FF1F239887049790FFFFE780A0281C
:101E30002A849790FFFFE7800027930714003385DB
:101E4000A7029747FF1F2398A702970701009387D0
:101E500027811747FF1F2323F7020145BDB717034B
:101E6000FFFFE7022326AA842E8901449749FF1F1A
:101E700093898919130A80069790FFFFE780A022B3
:101E80006347A40001451703FFFF6700E3263305FE
:101E9000440383A709024A86A6853E959700000061
:101EA000E780E0B919E10504C1BF0545E9BF1703A3
:101EB000FFFFE7024320AA8A2E8BB28B368C3A8A28
:101EC000814401448149974CFF1F938CEC13130DFF
:101ED00080069790FFFFE780001D63C9A40011E012
:101EE00085494E851703FFFF670063203389A403EC
:101EF00083A70C025E86D6853E994A85970000002E
:101F0000E780E0B31DC19790FFFFE780C01A05444A
:101F1000636D4501D2866286DA8513050903970051
:101F20000000E780A0D411C1854985045DB717037F
:101F3000FFFFE7022319C16441112A89014497492F
:101F4000FF1F9389690C130A8006FD1436C632C43C
:101F50002EC29790FFFFE780001592452246B246B9
:101F60006348A400014541011703FFFF6700C31840
:101F70003305440383A709023E9509C6834735000C
:101F8000C18B9DC791C68347350093F707028DC368
:101F9000630699008357E500639C270103570500FA
:101FA00001CB63E7E50083478500BA97E3CDF5FAF7
:101FB000050469BF1703FFFFE702C310C1642A8944
:101FC00001449749FF1F93892904130A8006FD14D1
:101FD0009790FFFFE780200D6346A4001703FFFFE3
:101FE000670083113305440383A709023E95835795
:101FF000E500638A970063049900639627019700C0
:102000000000E780E0970504E1B71703FFFFE70250
:10201000030A89692A8AAE8A328BB68B8144174CAF
:10202000FF1F130C6CFE930C8006314DFD19979029
:10203000FFFFE780400763C6A4001703FFFF6700A8
:10204000C30A3389940383270C028355CA015A8635
:102050003E994A8597000000E780609E31C1814D1E
:1020600015A03384AD038327090303D60B00D6855F
:1020700033F6C9003E94228597000000E780E0B661
:1020800009E9850D9790FFFFE780E0FFE3CBADFC0A
:1020900001A8228597000000E780E08A230404005D
:1020A000850471B71703FFFFE702E3004169AA8ABD
:1020B000014A174BFF1F130B2BF57D19C14B054C24
:1020C0009790FFFFE78020FE6346AA001703FFFFFB
:1020D0006700E30193098006B3073A0383290B02E3
:1020E000BE9983D7E900638E270163842A01639A2E
:1020F000570103A4890301E84E8597000000E7809B
:10210000C0BD050A75BF835704016399770993041D
:10211000C400268597A0FFFFE78060D385452A8D00
:102120002685835C040197A0FFFFE780C0CF26854A
:1021300097A0FFFFE780A0E762056185635905046A
:102140008D45268597A0FFFFE780E0CD8945268550
:1021500097A0FFFFE78020CD8945268597A0FFFF48
:10216000E78060CC8545268597A0FFFFE780E0CC1F
:1021700083470500094793F7F707639AE7009945F6
:10218000268597A0FFFFE78040CBA3028501484842
:10219000337D2D01231894016A9548C40040A1BFE6
:1021A0001703FFFFE702A3F337E404008327041DAE
:1021B00082979747FF1F83C727D21715FF1F130565
:1021C000E536A300F5008327441C82978327841CEF
:1021D00081461306F00F8145014582971703FFFFE3
:1021E000670023F21747FF1F130707BF18439745E0
:1021F000FF1F83C565CE9747FF1F938767CC834634
:102200008703034697036397D5009747FF1F2385EE
:10221000C7CC828083C587010347A7036317B60035
:102220009747FF1F238AE7CA828003C68701631787
:10223000C7009747FF1F2381D7CA828083C68701C3
:10224000130750026319D700930760021747FF1F57
:102250002304F7C8828083C68701130660026315D2
:10226000D60093077002DDB783C7870155BF974734
:10227000FF1F9387E7C4D44B0947638DE608170314
:10228000FFFFE702C3E51749FF1F1309A9C03E84FA
:1022900083470900918B9DCFB7E4040083A7041DF9
:1022A000829783A7441C1745FF1F130525BF8297FC
:1022B00083A7841C81461746FF1F034626C081451D
:1022C0000145829721C583470900ED9B1747FF1FF2
:1022D0002302F7BC8347040093F7F70F85CB9147A0
:1022E0001747FF1F2328F7BE97000000E78080EB09
:1022F00097000000E78040EFB7E70400BC4F41467D
:1023000091451745FF1F034525BC82971703FFFF23
:10231000670023DF82801703FFFFE70243DC8D475E
:1023200041116306F504C5476308F502854763104C
:10233000F5029747FF1F2383A7BAB7E70400BC4BFA
:10234000930500101745FF1F034505B8829741010B
:102350001703FFFF6700E3DA85471747FF1F230FC7
:10236000F7B6B7E70400BC4B93050020E1BF9747E1
:10237000FF1F9387E7B4D44B1147638DE600B7E79F
:10238000040083A7071D8297B7E70400BC4B9305A1
:1023900000044DBF05491747FF1F232D27B383C7EF
:1023A000070032C62E8493F7F70FD5D3B7E40400A5
:1023B00083A7041D7D141374F40F8297E37689FCC0
:1023C000B245994703C61500E3F0C7FCFC44090673
:1023D0001745FF1F1305C5B08297BC489305000839
:1023E0001745FF1F034545AE829779BF1703FFFFCF
:1023F000E702E3CE1747FF1F130787AC4047184B90
:102400001C409746FF1F23A3F6AC6316E400174752
:10241000FF1F232FF7AA130584FE9790FFFFE78085
:1024200060A6035564FF9780FFFFE780E06E97A0EA
:10243000FFFFE78060D01703FFFF670083CC17031F
:10244000FFFFE702C3C99747FF1F938767A7D84BD2
:10245000DC4789C797000000E78080F98547174768
:10246000FF1F2329F7A69747FF1F9387E7969C43F3
:10247000930500021745FF1F034505A583C7870382
:102480001747FF1F230AF7A4B7E70400BC4B829746
:102490001703FFFF6700E3C69747FF1F23A4A7A208
:1024A00082801703FFFFE702E3C137E404007C4C9E
:1024B000A1451745FF1F034525A182977C48A145EB
:1024C0001745FF1F034545A09744FF1F9384449F72
:1024D0008297DC4489EB97000000E78080D91703DE
:1024E000FFFF670063C103D567FF9780FFFFE780A9
:1024F000A062AA896DD1D84891476310F7027C4C3D
:1025000091451745FF1F0345259C82977C489145BF
:102510001745FF1F0345459B829703A9490103D433
:1025200009018947B7E904001747FF1F2324F79AD9
:1025300083A7091D21044204829783C784011715CC
:10254000FF1F1305A5FE61191717FF1FA300F7FE54
:1025500083A7491C418082979747FF1F23800798D4
:1025600083A7C91C814609469375F40F4A85829753
:1025700011E99747FF1F83C7A7A689C79700FF1FC9
:10258000E7804067B7E70400BC4F2146A1451745E7
:10259000FF1F03456593829799B71703FFFFE70273
:1025A00003B493F7052001112E8481CF970000001A
:1025B000E78020E91345042005611703FFFF67004A
:1025C00043B493F70510A9CF9744FF1F9384448F1A
:1025D000DC4897000000E78020C11737FF1F130772
:1025E000A77F184383C78401034787036318F70055
:1025F000DC4489C797000000E78080DF85471747E4
:10260000FF1F2329F78CB7E70400BC4B930500029A
:102610001745FF1F0345458B82971345041069BF7B
:1026200093F70508BDC79747FF1F83C7778BE91747
:1026300019469745FF1F9385C58A1305D10093F46A
:10264000F70F1749FF1F0349A98997C00000E780CA
:10265000404093970401C1831747FF1F1307C788A2
:10266000231DF100231CF1009747FF1F9387478527
:102670003ACE3ACAD8432306010009CBDC4393156E
:10268000890154080D46E1856800829713450408C6
:1026900025B793F72500A5C39747FF1F9387478268
:1026A000D84B89476306F7029737FF1F83C7877E9A
:1026B00013F7270011EF918B99CFB7E70400BC4FB8
:1026C0001306000A89451735FF1F0345E57F8297EA
:1026D00013452400D5B59737FF1F9387E76F9C43B9
:1026E00083C787031737FF1F2308F77E9700000073
:1026F000E78060DBF1BF93F7050281CB9700000014
:10270000E78060DA1345040245BD93F7850081CB6D
:1027100097000000E780E0D21345840071BD93F775
:10272000150081CB97000000E780A0B4134514008A
:1027300061B593F7450081CB97000000E78060B357
:102740001345440095BD93F7050495C39737FF1FC4
:1027500083C7077791CB97000000E780A0A491473B
:102760001737FF1F2328F77613450404B1B593F7F5
:1027700005010145E38207E49737FF1F93874774FC
:10278000D84B91476310F7049737FF1F93878770E3
:102790009C4313D727008583D98F858B91E7B7E7B3
:1027A000040083A7071D8297B7E70400FC4F9145FB
:1027B0001735FF1F03454571829785471737FF1F60
:1027C000232AF77013450401C5BB9747FF1F2389D0
:1027D000A78082801703FFFFE70263909737FF1FF0
:1027E00023A6076E9737FF1F23A4076E854717346C
:1027F000FF1F1304645E1737FF1F232DF76C1C4067
:1028000083C787031737FF1F2308F76C9790FFFFD5
:10281000E780A08F29C59717FF1F23ADA7D01C40C5
:10282000170500001305A5D783C787031737FF1FB8
:102830002304F76A1717FF1FA30AF7CE9737FF1F66
:10284000A3800768B7E7040083A707088297973734
:10285000FF1F238BA7661703FFFF6700838AB7C795
:10286000898E938767ED1717FF1F2325F7CC45BF88
:102870001737FF1F0347C764795555E79737FF1F81
:102880009387076403C7170005079736FF1FA389BF
:10289000E66203C717008D463377D7029736FF1FCE
:1028A000A380E66283C617001737FF1F1307C752BE
:1028B000184393F6F60FA9EE834787031737FF1FD8
:1028C000230CF76085471737FF1F230BF75E9737F9
:1028D000FF1F9387275C9C430145998BA9E717F35A
:1028E000FEFFE702C37F37E404007C48C14517358B
:1028F000FF1F0345655D82973C4885451735FF1FDF
:102900000345855C8297014517F3FEFF6700637FEF
:1029100083C7170085466395F6008347970379BF01
:102920008347A70361BF82809737FF1F83C747593B
:10293000A1CF17F3FEFFE702837A37E4040097374D
:10294000FF1F238F07567C4885451735FF1F03451A
:10295000A55782977C4C91451735FF1F0345C556F7
:1029600082977C4891451735FF1F0345E5558297AF
:102970003C48C1451735FF1F034505558297014562
:1029800017F3FEFF6700E3777955828017F3FEFFA8
:10299000E702E3742A84035565FF9780FFFFE78011
:1029A000A0179737FF1F9387A751D847BE841DEF05
:1029B0009790FFFFE78080779C48232004009DEBE1
:1029C0009737FF1F23A687509737FF1F23A08750F5
:1029D000B7E70400BC4B89451735FF1F0345C54EBB
:1029E0008297014517F3FEFF6700A371630A870012
:1029F000184375BF80C39737FF1F23AB874CC9BFF0
:102A00007955CDB717F3FEFFE702636D9737FF1FC8
:102A10009387475D8843232605002324050051053D
:102A200097A00000E780C03317F3FEFF6700636DD7
:102A300017F3FEFFE702A36A1734FF1F1304845A3B
:102A40001C40411199CF9C472302B5002AC61CC1E6
:102A500097000000E78040FB1C409C4B99C3324527
:102A60008297410117F3FEFF6700A36917F3FEFF8A
:102A7000E702E3664111444D328532842EC69790B9
:102A8000FFFFE780C0522AC422859790FFFFE780AE
:102A9000205403A84400630C0800B2458357440047
:102AA0001840224683D54500AA8626850298410112
:102AB00017F3FEFF6700E36417F3FEFFE7022362EC
:102AC000404D1DC808C09705000093856503130598
:102AD000440197A00000E78040169737FF1F9387B7
:102AE00067509C43014589E79737FF1F23AC874E0A
:102AF00017F3FEFF6700E3607D55DDBF17F3FEFFB0
:102B0000E702E35D011168009305F00F02C602C8F9
:102B100002CA02CC02CE97000000E780A0F1056156
:102B200017F3FEFF6700E35D9737FF1F9387874B1F
:102B30009C43D847A1679D076319F70217F3FEFF6F
:102B4000E702E359011132859790FFFFE7802046A5
:102B5000230AA1008145680097000000E78080ED0E
:102B6000056117F3FEFF6700C35982809737FF1F87
:102B7000938747479C43D847A16793877703631997
:102B8000F70217F3FEFFE702835501113285979094
:102B9000FFFFE780C041230AA1008145680097003C
:102BA0000000E78020E9056117F3FEFF6700635529
:102BB00082809737FF1F9387E7429C43D84795470A
:102BC0006316F70417F3FEFFE70263510111328524
:102BD00032849790FFFFE780803D230AA100228581
:102BE0009790FFFFE780C03E83574400231BA1005E
:102BF00081453ECC1C4068003ECE97000000E78037
